:020000040800F2
:10000000C8820020690200083D5200087D440008B3
:100010003952000881190008BD6E00080000000078
:1000200000000000000000000000000071610008F6
:10003000B11F000800000000A1540008D9610008A9
:10004000830200088302000883020008830200087C
:10005000830200088302000883020008830200086C
:1000600083020008B51F0008C11F000883020008B2
:10007000951E0008A51E00088302000883020008E0
:10008000830200088302000883020008830200083C
:10009000830200088302000883020008CD1F0008C5
:1000A000830200088302000883020008830200081C
:1000B000830200088302000883020008830200080C
:1000C00083020008830200088302000883020008FC
:1000D00083020008830200088302000883020008EC
:1000E00083020008830200088302000883020008DC
:1000F00083020008830200088302000883020008CC
:1001000083020008830200088302000883020008BB
:1001100083020008830200088302000883020008AB
:1001200083020008B51E0008C51E0008D51E000881
:10013000830200088302000883020008830200088B
:10014000830200088302000883020008830200087B
:1001500083020008E51E000883020008A56E00085F
:10016000830200088302000883020008830200085B
:1001700083020008830200088302000800000000D8
:10018000830200088302000800F002F800F05CF827
:100190000AA090E8000C82448344AAF10107DA45E2
:1001A00001D100F051F8AFF2090EBAE80F0013F0D8
:1001B000010F18BFFB1A43F00103184738C80000AD
:1001C00058C800000A444FF0000C10F8013B13F02F
:1001D000070408BF10F8014B1D1108BF10F8015BA0
:1001E000641E05D010F8016B641E01F8016BF9D193
:1001F00013F0080F1EBF10F8014BAD1C0C1B09D1EA
:100200006D1E58BF01F801CBFAD505E014F8016B5B
:1002100001F8016B6D1EF9D59142D6D370470000ED
:100220000023002400250026103A28BF78C1FBD8FF
:10023000520728BF30C148BF0B6070471FB50CF094
:1002400040F91FBD10B510BD00F062F91146FFF76F
:10025000F5FF06F0FDFE00F080F903B4FFF7F2FFB2
:1002600003BC00F083F900000948804709480047B3
:10027000FEE7FEE7FEE7FEE7FEE7FEE7FEE7FEE756
:10028000FEE7FEE704480549054A064B70470000B3
:100290009162000889010008C87C0020C882002003
:1002A000C87E0020C87E002053EA020C00F069805E
:1002B0002DE9F04B4FF00006002B1FBFB3FA83F57A
:1002C00003FA05F424FA05F65E4012BF1643B2FAAB
:1002D00082F502FA05F4C5F120051EBF22FA05FCDD
:1002E00044EA0C04203556EA044C4FEA144418BF83
:1002F000641C4FF000084FF00009904271EB030CB2
:1003000039D3002919BFB1FA81F701FA07F6B0FA1B
:1003100080F700FA07F6C7F120071EBF20FA07FC96
:1003200046EA0C062037B6FBF4FCA7EB0507103FA6
:1003300007F01F0BCBF120062CFA06F60CFA0BFB8C
:1003400044BFB3460026202FA4BF5E464FF0000BEB
:100350005BEA060C08BF4FF0010B19EB0B0948EBE9
:100360000608ABFB027C06FB02CC0BFB03CCC01BDC
:1003700071EB0C01C1E70B46024641464846BDE819
:10038000F08B13B5084318BF4FF0FF300146AFF3B1
:100390000080BDE81C407047032A40F2308010F016
:1003A000030C00F0158011F8013BBCF1020F624410
:1003B00098BF11F801CB00F8013B38BF11F8013BA1
:1003C000A2F1040298BF00F801CB38BF00F8013B4E
:1003D00011F0030300F02580083AC0F0088051F8BE
:1003E000043B083A51F804CBA0E80810F5E7121DC9
:1003F0005CBF51F8043B40F8043BAFF30080D207E8
:1004000024BF11F8013B11F801CB48BF11F8012BB3
:1004100024BF00F8013B00F801CB48BF00F8012BD6
:10042000704710B5203AC0F00B80B1E81850A0E832
:100430001850B1E81850A0E81850203ABFF4F5AFB2
:100440005FEA027C24BFB1E81850A0E8185044BF0E
:1004500018C918C0BDE810405FEA827C24BF51F87B
:10046000043B40F8043B08BF7047D20728BF31F86F
:10047000023B48BF11F8012B28BF20F8023B48BFC0
:1004800000F8012B704702F0FF0343EA032242EA1F
:10049000024200F002B84FF0000200B51346944645
:1004A0009646203922BFA0E80C50A0E80C50B1F1CC
:1004B0002001BFF4F7AF090728BFA0E80C5048BFE0
:1004C0000CC05DF804EB890028BF40F8042B08BF7E
:1004D000704748BF20F8022B11F0804F18BF00F87A
:1004E000012B704770477047704710B500F008F84F
:1004F000006810BD10B5044600F002F8046010BD9D
:10050000004870474001002000487047400100202B
:100510007546FFF7F9FFAE4605006946534620F0E1
:100520000700854618B020B5FFF7ACFEBDE82040B7
:100530004FF000064FF000074FF000084FF0000B9F
:10054000AC46ACE8C009ACE8C009ACE8C009ACE80E
:10055000C00921F007018D46704710B50446AFF37E
:1005600000802046BDE81040FFF777BE0149182003
:10057000ABBEFEE72600020070470000B0B52DEDCF
:10058000028B044600284FF0FF0061D00D46002981
:100590005ED095ED000A95ED011A95ED022A95EDD4
:1005A000033A20EE010A22EE033A21EE011A22EE6E
:1005B000022A31EE021A30EE030A31EE011AB7EECA
:1005C000008A30EE000A78EE410A09F079FDB0EEBB
:1005D000401A95ED000A95ED012A95ED023A95ED48
:1005E000034A20EE030A24EE022A30EE420A30EEDD
:1005F000000AB0EEC02AB4EE482AF1EE10FA84EDFB
:10060000011A02DA09F05AFA01E006F0C7FC84ED9B
:10061000020A95ED000A95ED011A95ED032A95ED74
:10062000023A20EE020A21EE031A30EE010A23EE0E
:10063000031A22EE022A32EE011A31EE011A30EECE
:10064000000A78EE410A09F03BFD002084ED000A23
:1006500040B2BDEC028BB0BD70B52DED028B002811
:100660004FD0B7EE001A81EE000A0D4604464FF057
:100670007E51002D80ED040A4FF00000C4E9001007
:10068000A060E06000F09F80D5E900600BF078FE8C
:1006900041EC180B30460BF073FE41EC110BB0EE41
:1006A000480AF0EE680A09F00BFC51EC100B0BF055
:1006B00025F895ED000AB5EE400AF1EE10FA22D1C8
:1006C00095ED010AB5EE400AF1EE10FA1BD195ED59
:1006D000020AB5EE400AF1EE10FA14D140F2C560FC
:1006E000C3F64D7044F62D214AF2564244F2AD73E2
:1006F000C3F60D41CBF63932C3F619730FC400208F
:1007000061E0FF205FE09FED321A00EE100AB4EEC8
:10071000410AF1EE10FA1EDCB5EE400AF1EE10FAD5
:1007200019DB9FED2C2AB4EE420AF1EE10FA25DC1B
:10073000B4EE410AF1EE10FA20DB9FED271AB4EE79
:10074000410AF1EE10FA2CDCB4EE420AF1EE10FA96
:1007500027DB002037E045F66E10C3F67F7045F2C8
:100760000C3148F6AB0249F28553C3F6B011CBF613
:10077000BB32C3F697530FC4002024E040F2C5609B
:10078000C3F64D7044F62D214AF2564244F2AD7341
:10079000C3F60D41CBF63932C3F619730FC40020EE
:1007A00011E040F2C560C3F64D7044F62D214AF2C7
:1007B000564244F2AD73C3F60D41CBF63932C3F65F
:1007C00019730FC4002040B2BDEC028B70BD00BF96
:1007D000DB0FC9BFDB0F49C00000B4C2B0B52DEDBF
:1007E000108B8EB0044600284FF0FF0018BF002980
:1007F00004D140B20EB0BDEC108BB0BD002AF8D0D1
:1008000040F204054EF69E70C2F20005C3F6275072
:100810002860C3B193ED00EA93ED01FAD3ED028AAB
:10082000B5EE40EAF1EE10FA11D1B5EE40FAF1EE74
:1008300010FA0CD1F5EE408AF1EE10FA07D12046FD
:1008400000F094FAD5E7204600F090FAD1E792ED57
:10085000000A92ED011A94ED014A94ED025A92EDCC
:10086000022A94ED036A94ED003A24EE407A61EE98
:10087000050A37EE607A62EE060A37EE607A60EEBD
:10088000030A62EE051A71EEA00A61EE061A70EE16
:10089000E10A61EE031A62EE042A22EE032A21EE37
:1008A000041A91ED00DA71EEE21A20EE066A31EEDA
:1008B000021A20EE050A36EE216AD1ED019AD1ED39
:1008C00002AA31EE400AB6EE001AB5EE40DA27EE83
:1008D000015A60EE810A26EE017AF1EE10FA20EE5E
:1008E000016A0AD1F5EE409AF1EE10FA05D1F5EE63
:1008F00040AAF1EE10FA00F0EC812DEE0D0A29EE7F
:10090000A91A30EE010A2AEEAA1A30EE010A8DED7C
:100910000D6A8DED0C7ACDED0B0A8DED0A5A03F0C0
:10092000FDFF2DEE001A8DED071A29EE801A2AEE32
:10093000800A8DED081A8DED090A2EEE0E0A2FEEB3
:100940000F1A30EE010A28EEA81A30EE010A03F061
:10095000E5FF94ED001A6EEE00DA6FEE00AA94ED5A
:10096000034A31EE01EA68EE808A94ED012A94EDA3
:10097000023A2AEE8E6A61EE01EA8DED026A28EEF5
:100980008E0A2DEEAE5A26EE046A62EE02BA35EEFB
:10099000465A20EE036A36EE055A2DEEAB6A32EE69
:1009A00002FA36EE055A2AEE8F6A23EE066A36EE12
:1009B000055A28EE8F6A26EE046A63EE03FA36EED5
:1009C000055A2DEEAF6A24EE048A35EE465A2DEE16
:1009D000886A2DEE8E9A35EE465A29EE046A2AEE82
:1009E000AE7A37EE066A22EE000A2DEE8FAA36EEB8
:1009F000400A23EE0A6A36EE000A2AEEAB6A30EEAF
:100A0000460A2AEEAF6A73EE039A36EE000A28EE23
:100A1000A96A24EE066A36EE000A2AEE886A30EEEB
:100A2000460A25EE055A20EE000A35EE000A21EEB0
:100A300002BA21EE035A21EE041A8DED051A22EEB8
:100A4000031A8DED031A23EE041A8DED041A34EE09
:100A5000041A8DED015A22EE04CA6EEE03CA8DED22
:100A6000061A29EE84DA03F059FF94ED013A94ED69
:100A7000022A9DED021A29EE024A21EE031A31EEF6
:100A8000444A94ED031A28EEAE5A35EE044A2AEE93
:100A9000015A35EE044A28EEAB5AF7EE001A34EE4E
:100AA000454A2AEEA95A81EE800A25EE015A35EE12
:100AB000044A28EEAF5A34EE454A28EE885A75EEBD
:100AC000042A3CEE0C4A9DED075A34EE6C4A34EE93
:100AD000454A3BEE0B5A9DED086A35EE0D5A35EE50
:100AE000465A2FEE056A29EE847AF6EE007A76EE03
:100AF000470A37EEEF6A36EE486A9DED018A20EE2E
:100B0000066A3CEE487A27EE227A36EE076A36EE1F
:100B10006D7A22EE226A66EE073A70EEE33ADDED78
:100B2000050ADDED034A60EE015A74EEE00ADDEDE0
:100B3000044A60EE200A7BEE244A64EEA24A70EE7C
:100B4000A40A63EE224A70EEEA0A74EEE56A66EEE3
:100B5000A06A77EEEB7A76EEA33A78EE0C6A77EE3F
:100B6000EF7A60EE266A67EEA27A76EEA76A76EEF4
:100B7000E86A60EE027ADDED068A27EEA68A38EE94
:100B800023CA68EE843A2EEE058A78EE233A3BEECD
:100B9000AB8A71EEC81A3FEEAF8A71EEC81A9DEDAE
:100BA000098A21EE22AA71EEC81AB1EE008A23EE5C
:100BB000089A21EE899A73EEC93A94ED009A2AEECA
:100BC00007BA73EE8B3A29EE22BA77EE8B7A67EE8C
:100BD000A07A72EEA22A77EEA33A63EE227A75EE3D
:100BE000E75A65EEA65A35EEA3DA68EE853A6EEE60
:100BF000045A73EEE53A62EE085A65EEA11A73EEF6
:100C0000E11AF8EE003A60EE233A62EE235A75EEEE
:100C1000CB5A65EE875A20EE033A71EEA51A73EEB1
:100C20000A5A20EE090A22EE222A65EEA05A30EE78
:100C3000422A75EEA11A22EE262A23EE811A32EEFE
:100C4000218A2FEE042A29EE854A31EE241A34EE49
:100C5000022A21EE071A36EE400A32EE011A20EE81
:100C6000200A30EE010A23EE261A31EE009A2CEE0D
:100C70000C0A2DEE0D1A30EE010A28EE081A31EE9C
:100C8000000A29EE091A31EE000A03F047FE95ED3D
:100C9000004A9DED0A5A20EE0C1ADDED0B0A20EEFB
:100CA0000D2A24EE011A9DED0C7A9DED0D6A20EEC1
:100CB000083A20EE090A35EE415A24EE021A70EE87
:100CC000C10A24EE031A24EE000A37EE417A36EE0A
:100CD000406A94ED043A94ED000A94ED011A25EE71
:100CE000035A94ED022A30EE050A20EE835A94ED61
:100CF000034A35EE011A27EE035A35EE022A26EE94
:100D0000033A84ED000A84ED011A20EE000A21EE78
:100D1000011A33EE043A30EE010A22EE021A30EEE6
:100D2000010A23EE031A30EE010A84ED022A84ED53
:100D3000033A03F0F3FD94ED001A94ED012A94EDCB
:100D4000023A94ED034A20EE011A20EE022A20EE28
:100D5000033A20EE040A002084ED001A84ED012AF3
:100D600084ED023A84ED030A43E50000B0B52DEDB1
:100D7000108B044600284FF0FF0018BF002900F038
:100D80006981002A00F0668140F2040542F60230D3
:100D9000C2F20005C3F60750286092ED000A92EDFA
:100DA000011A94ED014A94ED025A92ED022A94ED53
:100DB000036A94ED003A24EE407A61EE050A37EEBC
:100DC000607A62EE060A37EE607A60EE030A62EE3F
:100DD000051A71EEA00A61EE061A70EEE10A61EEE4
:100DE000031A62EE042A22EE032A21EE041A91ED80
:100DF00000CA71EEE21A20EE066A31EE021A20EE07
:100E0000050A36EE216A91ED01DA91ED02EA31EE42
:100E1000400AB6EE001AB5EE40CA27EE01BA20EE3F
:100E200081AA26EE019AF1EE10FA20EE018A0AD18B
:100E3000B5EE40DAF1EE10FA05D1B5EE40EAF1EE8A
:100E400010FA00F0BC802CEE0C0A2DEE0D1A30EEDC
:100E5000010A2EEE0E1A30EE010A03F05FFD94ED4A
:100E6000003A94ED025AF1EE001A2CEE001A94EDBD
:100E7000014A75EE050A63EE212A65EE053A62EE37
:100E8000A34A61EE205A74EEA54A64EE045A2DEE90
:100E9000002A94ED036A34EE047A62EEA52A72EE1B
:100EA000A42A62EE074A32EEE4CA76EE062A64EE1F
:100EB000214A66EE066A64EEA67A21EE22DA77EE21
:100EC000CD7A23EE03DA2DEE21DA2EEE000A24EE9F
:100ED0000DEA33EE033A7EEE277A22EE03EA77EE4E
:100EE000CE7AB2EE00EA24EE0E4A77EEE47A24EEF1
:100EF00025FA7FEE277A24EE234A34EE274A60EE65
:100F0000244A34EE84FA2DEE054A21EE033A33EEFC
:100F1000043A25EE0E4A25EE215A65EE264A33EEB6
:100F2000243A62EE222A33EE623A33EE453A65EE17
:100F3000842A32EE833A24EE234A34EE033A20EE3A
:100F4000050A30EE03DA21EE070A25EEA11A21EE9A
:100F5000061A31EE400A23EEA11A26EE011A30EEEF
:100F6000010A22EE201A30EE41EA2CEE0C0A2FEE96
:100F70000F1A30EE010A2DEE0D1A31EE000A2EEE98
:100F80000E1A31EE000A03F0C9FC95ED004A20EE7E
:100F90000C1A20EE0F2A24EE011A20EE0D3A20EE54
:100FA0000E0A3BEE41BA24EE021A3AEE41AA24EEB2
:100FB000031A24EE000A39EE419A38EE408A94ED85
:100FC000043A94ED000A94ED011A2BEE035A94EDC5
:100FD000022A30EE050A2AEE035A94ED034A35EE52
:100FE000011A29EE035A35EE022A28EE033A84ED5F
:100FF000000A84ED011A20EE000A21EE011A33EEF8
:10100000043A30EE010A22EE021A30EE010A23EE13
:10101000031A30EE010A84ED022A84ED033A03F04C
:101020007DFC94ED001A94ED012A94ED023A94EDC2
:10103000034A20EE011A20EE022A20EE033A20EEA7
:10104000040A002084ED001A84ED012A84ED023A9E
:1010500084ED030A40B2BDEC108BB0BDB1EE601A56
:10106000B4EE600AF1EE10FAB4EE401AC8BFB0EE6A
:10107000600AF1EE10FAC8BFB0EE410A70470000F6
:1010800000214FF07E524DF20A734CF28F2CC3F6C2
:101090002343C3F6F54CC0E90011C0E90221016108
:1010A0004FF07A5142618361C0F81CC00162704701
:1010B00090ED056A90ED035A66EE011AD0ED042A10
:1010C000D0ED063A31EE855A75EE224A63EE813A4A
:1010D00090ED024A74EEA33A63EE813A34EE234A6D
:1010E000D0ED083A71EEA21A74EE232AC4EE223A29
:1010F000C1EEA22AF6EE004A90ED013A60EE244AD3
:1011000064EE814A90ED002A23EE017A64EE814A72
:1011100034EE877A32EE072A90ED077A20EE010A44
:1011200030EE030A27EE011A30EEC23A36EE011A0B
:1011300023EE236A32EE062A80ED002A23EE222ACD
:1011400030EE020A80ED010A24EE230A34EE400A52
:1011500080ED020A25EE230A35EE400A80ED030AEF
:1011600024EE220A31EEC00A80ED040A25EE220A9E
:1011700031EE400A80ED050A7047000080B541F26B
:101180003430C2F200000068042106F00FF980BD7F
:1011900080B540F21832C2F200020020122113235F
:1011A00000F086F9002080BD80B5012001214FF0BC
:1011B000FF3206F03BF980BD9FED010A704700BF8A
:1011C0000000C84380B541F23430C2F2000000682C
:1011D000082106F0EBF880BD80B540F21830C2F26D
:1011E0000000C21D01200221062300F061F9002049
:1011F00080BD000080B5022001214FF0FF3206F0D3
:1012000015F980BDF0B581B000284FF0FE0700F061
:1012100097800C46002900F0938040F67406C2F2D5
:1012200000060546307808B1FD2789E006F05CF934
:1012300041F23431C2F20001002808607BD0002066
:101240007E21B622EC6200F085F901201421B6223D
:1012500000F080F91E2000F0E7FA00201E2100F0C7
:1012600049F90020002100F045F91E2865D1012030
:101270000021012400F03EF90F2860D1022000F087
:101280008DF9032000F08AF941F26142C0F60002B4
:1012900000200121002700F09DFA41F27D11C0F6E7
:1012A0000001022000F0C0F941F2C511C0F60001B2
:1012B000032000F0B9F900204021AA2200F04AF9E9
:1012C00000204121012200F045F90020532108228D
:1012D00000F040F900205821042200F03BF90020E2
:1012E0007D21042200F036F9322000F09DFA012021
:1012F0000F21012200F02EF901201021032200F01D
:1013000029F901201621002200F024F901201821DA
:10131000012200F01FF901201521802200F01AF9A6
:101320000A2000F081FA0220347000F04FF9032007
:1013300000F04CF904E0FE2702E0FC2700E0FC2767
:1013400078B201B0F0BD0000002841D040F2183161
:10135000C2F20001B1F901209FED1F3A00EE102A00
:10136000B8EEC00A80EE030AB1F90330B1F905C046
:1013700001EE103A02EE10CAB8EEC11AB8EEC22A57
:1013800081EE031A82EE032A4FF60003CFF6FF73B5
:1013900080ED040A4A7C897CD20042EA5112002185
:1013A000B1EB922F80ED051A80ED062A18BF1A4383
:1013B00000EE102AB8EEC00AB4EE001A20EE010AC0
:1013C000B3EE071A30EE010A80ED0A0A48B2704700
:1013D000FE2148B2704700BF00A0AA45C0B340F24A
:1013E0001831C2F20001B1F90720B1F90930B1F9A1
:1013F0000B1000EE102A01EE103A9FED172A03EEB3
:10140000101AB8EEC00AB8EEC11AB8EEC33A80EEB0
:10141000020A81EE021A83EE022A9FED103AC16A97
:1014200091ED014A91ED025A20EE030A21EE031AD2
:1014300022EE032A91ED003A31EE441A30EE430ACF
:1014400032EE452A80ED070A80ED081A80ED092A60
:101450006FF00100704700BF6F12034235FA8E3CF7
:1014600010B5002000F0CAF841F23434C2F2000492
:1014700038B90020012100F0FDF82068012105F0B5
:1014800095FF012000F0BAF8002818BF10BD012018
:10149000012100F0EFF82068022105F087FF10BD60
:1014A00080B50C2001214FF0FF3205F0BFFF80BD59
:1014B000002A08BF704770B51C4615460E46012825
:1014C00002D8002100F0D6F840F22B3146F080001F
:1014D000C2F20001087000200122002300F08AF906
:1014E000002029462246012300F05AF9BDE8704049
:1014F0007047000070B5044601200D4600F094F9D5
:10150000012C03D82046002100F0B4F845F08000FB
:1015100040F22B35C2F200052E4606F8010B0020E2
:1015200029460122002300F065F900202946022205
:10153000002300F035F92CB1012C08D140F22B36F4
:10154000C2F200062046012100F094F83078C0B2C3
:1015500070BD000010B5044601F07F0040F22B3151
:10156000C2F20001087001204A7000F05DF9012C00
:1015700003D82046002100F07DF840F22B31C2F262
:10158000000100200222002300F034F9012C88BF62
:1015900010BD2046012100F06DF810BD0238C0B228
:1015A000022882BFFF2040B2704780B541F20A7125
:1015B000C000C0F2090121FA00F040B201F096F932
:1015C0000020BDE8804040B2704700000238C0B241
:1015D000022882BFFF2040B2704780B541F20A71F5
:1015E000C000C0F2090121FA00F040B201F082F916
:1015F0000020BDE8804040B270470000052884BF4D
:101600000020704780B54CF62001C0F6000101EBC8
:10161000C002526831F83010104600F099FF0138CE
:10162000B0FA80F0400980BDB9B1052882BFFF2023
:1016300040B270474CF62002C0F6000232F830C0CB
:10164000002000232CFA00F2D20709D10E2B03F15F
:10165000010300F10100F5D908E0FE2040B2704717
:1016600040F2A012C2F2000242F82010002040B264
:1016700070470000052882BFFF2040B2704780B548
:101680000A464CF62001C0F6000101EBC0035B687E
:1016900031F83010184600F061FF0020BDE88040AE
:1016A00040B27047082882BFFF2040B270474CF616
:1016B0005001C0F60001B7EE001A51F83010B4EE38
:1016C000410AF1EE10FAC8BFB0EE410A0A689FED78
:1016D000181AD16AB5EE400A0131F1EE10FAB8BF1E
:1016E000B0EE410A01EE101AB8EE411A20EE010ADE
:1016F000BCEEC00A011F022910EE101A02D802F136
:10170000340010E0072801D0012802D102F138008E
:1017100009E040F2051323FA00F0C0070CBF02F104
:10172000400002F13C000160002040B2704700BF61
:1017300000000000082882BFFF2040B2704780B53B
:101740004CF65001C0F6000101EBC00251F8300028
:10175000918802F023FB0020BDE8804040B2704732
:10176000082882BFFF2040B2704780B54CF6500178
:10177000C0F6000101EBC00251F83000918802F080
:101780009FFB0020BDE8804040B2704740F23061CE
:10179000C2F20001002818BF00210846704700006F
:1017A00070B510B1FF2040B270BD1E4614460D4604
:1017B000FFF7ECFF0028F5D02946224616B101F0CC
:1017C00021FD02E0142301F063FC002818BF012072
:1017D00040B270BD002A0FBFFE2040F20023C2F2CB
:1017E000000303EB40101CBF40F82120002040B252
:1017F0007047000070B510B1FF2040B270BD1E46AA
:1018000014460D46FFF7C2FF0028F5D029462246B0
:1018100016B101F0E5FF02E0142301F08DFD002870
:1018200018BF012040B270BD70B5044605F078FCC9
:101830000546FF2605F056FC411C05290BD8012062
:10184000884010F0310F0BD110F0060F0AD020465F
:1018500000F078FD11E06FF00041884218BF0026CB
:1018600070B270BD4FF47A70B0FBF5F1B4FBF1F0DB
:10187000A14288BF012005F00BFC002670B270BDAC
:1018800070B5044600F00CF805460E4600F008F866
:10189000401BB141001B71F10000F7D3002070BD67
:1018A0002DE9F04105F03CFC044607F04FFE4FF4F3
:1018B0007A784EF21806B8FBF4F4CEF200063768D8
:1018C00004FB00F507F042FE60433168854208BF23
:1018D000394656F8042C01FB08F10132B1FBF2F154
:1018E00000FB08F0401A00F57A700021BDE8F08195
:1018F00040F2F07240F2A871C2F200020128C2F276
:10190000000118BF0022002818BF11460846704782
:1019100080B582B001680A68D20614D5002201920F
:101920000A68019249680191019905F059F940F25C
:10193000202100EBC000C2F2000101EB8000006A30
:10194000002818BF804702B080BD00003AB10128CE
:101950004FF0FF0398BF082904D958B27047FE23FF
:1019600058B2704740F2202300EBC000C2F20003DF
:1019700003EB8000002340F8212058B2704700009C
:10198000FEE7000000284FF0FF0218BF002901D138
:1019900050B2704790ED010A9FED603A90ED021A47
:1019A00030EE030A9FED5E3A9FED5E5A30EE000A7C
:1019B00090ED032A80EE036A31EE050A9FED5A1A74
:1019C0009FED5A5A30EE000A90ED044A80EE011A5B
:1019D00032EE050A9FED562A9FED565A30EE000A68
:1019E00080EE022A34EE050A30EE000A80EE035A39
:1019F000BFEE000A36EE006A81ED016A31EE004A60
:101A000081ED024AB0EEC44A32EE003A9FED4A2A16
:101A100081ED033A35EE001AB0EEC65AB4EE425AE2
:101A2000F1EE10FAB4EE424AB0EEC33A81ED041A78
:101A3000DCBF00224A60F1EE10FAB4EE423AB0EE9A
:101A4000C11ADCBF00228A60F1EE10FAB4EE421A2D
:101A5000DCBF0022CA60F1EE10FADCBF00220A618E
:101A600091ED012AB7EE001AB0EEC23AB4EE413A57
:101A7000F1EE10FA0ADBB5EE402AB0EE402AF1EEA4
:101A800010FAC8BFB0EE412A81ED012A91ED022A79
:101A9000B0EEC23AB4EE413AF1EE10FA0ADBB5EE1E
:101AA000402AB0EE402AF1EE10FAC8BFB0EE412A4B
:101AB00081ED022A91ED032AB0EEC23AB4EE413A2A
:101AC000F1EE10FA0ADBB5EE402AB0EE402AF1EE54
:101AD00010FAC8BFB0EE412A81ED032A91ED042A25
:101AE000B0EEC23AB4EE413AF1EE10FA08DBB5EED0
:101AF000402AF1EE10FAC8BFB0EE410A81ED040AA7
:101B000002780AB1002003E0C07D013818BF01202F
:101B10000A700022487050B2704700BF000051C3E5
:101B20000060AD44000032C30020AC44000052C34A
:101B30000040AD4400005DC3CDCC4C3DB5EE401A35
:101B4000F1EE10FA30EE600AD8BF7047B6EE002A08
:101B500021EE022AB4EE420AF1EE10FAC4BF30EED2
:101B6000410A7047B1EE422AB4EE420AF1EE10FA91
:101B7000B8BF30EE010A704740F21400C2F2000014
:101B800070470000B0B5E8B140F67504C2F2000439
:101B9000207810B1FD2568B2B0BD05F0A5FC41F27A
:101BA0003831C2F20001086060B141F64562C0F60A
:101BB0000002002003210025FFF7C8FE012020704D
:101BC00068B2B0BDFE2568B2B0BD00002DE9F04F8F
:101BD00082B090F802C0C27841F23C234FEADC04A4
:101BE000C2F2000362F34A1490F8019005795C8018
:101BF000C2784679AD0045EA921206F0010542EA44
:101C000085229A80457987796E0867F3CA16DE8047
:101C10008579C7794FEA151E67F30A1EA3F808E015
:101C2000077A90F80780457A7F0047EAD81705F0D1
:101C3000030547EA452BA3F80AB0457A877A4FEAAD
:101C4000950867F38A18A3F80C80C77A857AFF0095
:101C500047EA5515DD8190F80CA0477B009567F3A6
:101C60000A2AA3F810A0477B857BFF0865F34A1773
:101C70005F820197C77B6CF30A2990F80EC0057C40
:101C8000BF0047EA9C1705F0010547EA852CA3F839
:101C900014C0057C477C680800EE104A01EE102A4B
:101CA00002EE106AAEF22D1203EE109A67F3CA101C
:101CB000C72AB8EEC33AB8EEC00AB8EEC11AB8EEF9
:101CC000C22AA3F80090D88281ED012A81ED021A80
:101CD00081ED033A81ED040A01D201220DE0AEF557
:101CE000FA72B2F57A7F01D2032206E0AEF2DC523C
:101CF0000023C82A38BF01235A00ABF22D13DDE9B7
:101D000000679BB2C72B0A7501D201220FE0ABF529
:101D1000FA7292B2B2F57A7F01D2032207E0ABF2F7
:101D2000DC5292B20023C82A38BF01235A00A8F21D
:101D30002D13C72B4A7501D201220DE0A8F5FA72C6
:101D4000B2F57A7F01D2032206E0A8F2DC5200232A
:101D5000C82A38BF01235A00A6F22D13C72B8A7553
:101D600001D202220CE0A6F5FA72B2F57A7F01D216
:101D7000032205E0A6F2DC530022C82B38BF012263
:101D8000AAF22D13C72BCA7501D202220CE0AAF5C4
:101D9000FA72B2F57A7F01D2032205E0AAF2DC538F
:101DA0000022C82B38BF0122A7F22D13C72B0A76B9
:101DB00001D202220CE0A7F5FA72B2F57A7F01D2C5
:101DC000032205E0A7F2DC530022C82B38BF012212
:101DD000ACF22D139BB2C72B4A7601D201220FE041
:101DE000ACF5FA7292B2B2F57A7F01D2032207E023
:101DF000ACF2DC5292B20023C82A38BF01235A0049
:101E0000A0F22D13C72B8A7601D202220CE0A0F596
:101E1000FA72B2F57A7F01D2032205E0A0F2DC5318
:101E20000022C82B38BF0122B0F59670CA7618BFC1
:101E30000120B9F57A7218BF01221040087002B073
:101E4000BDE8F08F80B541F23830C2F20000006882
:101E50004FF4801105F0AAFA80BD000010B50446C9
:101E60000020FFF745FD2146192202F0B5FA0028AF
:101E700018BF4FF0FF3010BD80B502464FF4801000
:101E8000012105F0D3FAA0F58010B0FA80F04009E6
:101E900080BD000080B540F2B840C2F2000000F002
:101EA000F1F880BD80B540F29830C2F2000000F039
:101EB000E9F880BD80B540F21850C2F2000000F091
:101EC000E1F880BD80B540F2F830C2F2000000F0C9
:101ED000D9F880BD80B540F25840C2F2000000F051
:101EE000D1F880BD80B540F27850C2F2000000F019
:101EF000C9F880BDD0F800C06FF00F024AF6AB23DE
:101F000052FA8CF2CAF6AA230146A2FB033000095A
:101F100005A31B5C40F2FF302CEA00005F2A88BF5B
:101F20000430C1E9160370470006101600061016AB
:101F30008269816AB2F5005F06D06AB9022912D0BF
:101F4000012914D0D1B90EE0032917D8DFE801F038
:101F5000020B020F0120704703293CBF012070478C
:101F60001CBF00207047C06AC0F300607047C06AA1
:101F7000A0F1C070B0FA80F04009704700207047AF
:101F800080B5D0F800C0D0F808E0DCF80000BEF161
:101F9000400F20F48020CCF800000846CCF8043034
:101FA00004BF10460A46CCF80800CCF80C2080BDCF
:101FB0007047000080B5082000F0EEF980BD0000F9
:101FC00080B5102000F0E8F980BD000080B5202029
:101FD00000F0E2F980BD000072B600BFFEE700002D
:101FE00070B5866D044600F0BFFA94F835100229EA
:101FF00025D105462068216C026822F01602026095
:10200000426922F08002426109B9A16C19B10168EC
:1020100021F008010160016821F00101016000BFA9
:1020200020680068C0070ED000F09EFA401B06280A
:10203000F6D320206065032084F835000CE0802072
:102040006065012008E0E06D3F2101FA00F0B0601A
:10205000012084F835000020002184F8341070BD80
:1020600090F83510022909D1052180F83510006853
:10207000016821F001010160002070478021416565
:1020800001207047F0B581B004460020009040F276
:102090000000C2F200000268D4E9166048F2B513ED
:1020A00037680821C1F64E3381403942A2FB03252F
:1020B0000CD0226813685B0708D5136823F004036B
:1020C0001360B160616D41F00101616501218140E2
:1020D000394208D022685269120604D5B160616D98
:1020E00041F00201616504218140394208D0226833
:1020F0001268920704D5B160616D41F00401616519
:1021000010218140394215D020680268120711D58C
:10211000B16002680168520306D4C90506D401689B
:1021200021F00801016001E0080342D4216C09B1EB
:1021300020468847E16D202000FA01F23A4244D05F
:1021400020680368DB0640D5B26094F83530026839
:10215000052B1ED122F016020260426922F0800295
:102160004261226C0AB9A26C1AB1026822F008021C
:1021700002603F208840B060012084F83500216D66
:102180000020002984F8340040D02046884701B060
:10219000F0BD0168520310D4C90512D4016821F0C2
:1021A00010010160012084F83500002084F834001B
:1021B00007E0A16C0029BBD1BCE7080301D4616C26
:1021C00000E0E16B09B120468847606DF0B1606DB9
:1021D000C00717D0052084F835002068A90A0268D6
:1021E00022F00102026000BF009A01328A4200928E
:1021F00002D80268D207F7D1012084F83500002008
:1022000084F83400E16C09B12046884701B0F0BD84
:102210002DE9F041044600F0A7F9C4B105460220BB
:1022200084F835000020216884F83400086820F024
:102230000100086026683068C0070BD000F094F9F0
:10224000401B0528F6D903212022032042E001206B
:10225000BDE8F081306848F23F01CFF21001251D42
:1022600000EA010C2ECDD4E9050E41EA0C01114320
:1022700019432943D4E90778084340EA0E01606A0C
:102280003943042841EA080103D1D4E90B2311435F
:10229000194331607169042821F0070141EA000502
:1022A0000CD1D4E90A1045EA010538B12046FFF700
:1022B0003FFE18B10121402201200BE0204675614C
:1022C000FFF718FEE16D3F2202FA01F18160002262
:1022D00001210020626584F83510BDE8F08100001E
:1022E000B0B5044690F83400012828D0012084F8C5
:1022F0003400A56D94F8350001281DD1022084F822
:102300003500002060652046FFF73AFEE26D3F236E
:10231000206803FA02F2216CAA60026842F01602F9
:10232000026019B1016841F008010160016841F0E3
:10233000010101600020B0BD002084F834000220BB
:10234000B0BD0000B0B5044600F00EF9054640F2FD
:102350003410C2F200000078611C18BF044400BFB2
:1023600000F002F9401BA042FAD3B0BD70B540F2B4
:10237000A01604460025C2F2000603E00135102D28
:1023800008BF70BD24FA05F0C007F7D056F8250045
:10239000002818BF8047F1E780B543F61441C4F226
:1023A00001010A68024208BF80BD0860FFF7DEFF36
:1023B00080BD00002DE9F04F83B000F13E4202F1F4
:1023C000FF724FEAB22241F600470192C4F20207BF
:1023D00008224FF0010E00254FF0000A4FF00008D0
:1023E000B84208BF072200920AE000BF08F10108C6
:1023F0000AF1040AB8F1100F05F1020500F0A480FB
:102400000C680EFA08FB14EA0B09EFD04C6804F0D4
:10241000030CACF1010EBEF1010F11D80322876845
:1024200002FA05F6CA68B743AA403A438260426896
:10243000C4F3001722EA0B0207FA08F73A43426096
:10244000BCF1030F1CD0C26803238E6803FA05F7A2
:10245000BA4306FA05F73A43BCF1020FC2600FD146
:102460006FF0030202EA580202440AF01C060F232E
:10247000176A03FA06F40B69A743B3403B431362A0
:10248000026803234F68AB409A4307F00303AB4055
:102490001A4317F4403F4FF0010E0260A6D000220D
:1024A00043F644030292C4F202031A6843F600445E
:1024B00042F480421A601A68C4F2010402F48042B5
:1024C0000292029A28F003024FF6084B2244CFF6FC
:1024D000FF7B52F80B300AF00C070F26BE4023EAB0
:1024E000060C019B009E072B38BF1E4606FA07F715
:1024F00047EA0C0342F80B30A2684B6842EA09072E
:1025000043F60C4CDE0258BF22EA0907A760C4F26A
:10251000010CDCF800209E0242EA090758BF22EABB
:102520000907CCF8007062689E0342EA090758BFA9
:1025300022EA090767602268DB0342EA090358BF01
:1025400022EA0903236051E703B0BDE8F08F0000E1
:102550000069084018BF012070470000002A08BF2A
:10256000090481617047000047F2EC40C2F20000AC
:1025700000687047F0B581B0B0B3044690F83D00F4
:1025800028B9002084F83C00204600F0BFF8242041
:1025900084F83D002068016821F0010101600168B4
:1025A00041F400410160016821F40041016000F044
:1025B0006FFA48F28041C0F21E0140F600126568D1
:1025C00088424FF00001C0F23D0248F2A16C4FF08A
:1025D000000338BF01219042C0F2010C38BF012333
:1025E000654538BF0B4613B1012001B0F0BD4DF673
:1025F0008361C4F21B31A0FB011221684FEA924EA5
:102600004B684FF4967623F03F0343EA92434B60C6
:1026100044F6D3530F6A0EFB06F6C1F26203A6FB23
:10262000033627F03F03B709654538BF970C7A1C7E
:102630001A430A62CA6948F2A0674CF6FF73C0F2F7
:102640000107BD4222EA030C0AD801386A00B0FB38
:10265000F2F001306FF31F30042898BF04202BE004
:10266000A368A0F1010E9BB119206843BEFBF0F0F6
:102670000422013062F31F30000512D09BB11920F3
:102680006843BEFBF0F00422013062F31F3011E01A
:1026900005EB4500BEFBF0F001306FF31F30000585
:1026A000ECD1012008E005EB4500BEFBF0F0013065
:1026B0006FF31F3040F4004040EA0C00C861086826
:1026C000D4E9072320F0C00010431843086088684D
:1026D00048F2FF3204F10C0790438CCF18431043AB
:1026E000A6698860C86820F0FF0038433043C8609E
:1026F000086840F00100086000202021206484F870
:102700003D10206384F83E0001B0F0BD2DE9F04F8C
:1027100087B0044645F600470068C4F2000700266B
:10272000B8420696CDE904660396029602D007B039
:10273000BDE8F08F43F630050196C4F20205286823
:102740000DF1080840F00400286028684FF01209D5
:1027500000F0040001900198019628684FF0030AE8
:1027600040F00100286028684FF0040B00F00100E1
:10277000019001984FF40070029007F5D630414661
:10278000CDE90396CDF814A0CDF818B0FFF712FEEE
:102790004FF48070CDE9020904A880E8400C07F5E9
:1027A000D2304146FFF706FE019628694FF0C0611E
:1027B00040F400002861286940F2983500F40000D8
:1027C0000190019846F24000C2F20005C4F20200F6
:1027D0004FF4806285E843002846C5E90362C5E9F5
:1027E0000566C5E907666E62FFF712FD002818BF8F
:1027F000FFF7F2FBA563AC6307B0BDE8F08F000004
:1028000040F2341047F2EC41C2F20000C2F2000183
:1028100000780A68104408607047000080B543F6ED
:102820000040C4F20200016841F4007101600168D7
:1028300041F480610160016841F48071016003200E
:1028400000F06CF80F2000F005F800F02BF80020E5
:1028500080BD0000B0B540F23412C2F2000240F276
:1028600000011278C2F200014FF47A730968B3FBD9
:10287000F2F20446B1FBF2F1084601F05DF80F2CCC
:102880004FF001050CD858B94FF0FF302146002217
:10289000002500F033F840F23810C2F20000046066
:1028A0002846B0BD80B582B0002043F640010190BB
:1028B000C4F202014A6842F480424A604A6802F463
:1028C00080420192019A00900868002240F08050F6
:1028D000086008680F2100F08050009000986FF0A9
:1028E000010000F00BF802B080BD000080B504F0DC
:1028F000FFFA80BD80B504F00FFB80BD70B51446B3
:102900000D46064604F018FB2946224602F098FCC4
:102910000146304604F018FB70BD000080B504F09D
:102920002DFB80BD2DE9F041002800F08B8043F69F
:102930000808C4F202080446D8F8F8030D4600F06F
:102940000700884207D288F8F853D8F8F80300F057
:102950000700A84276D12068810717D5410705D521
:10296000D8F8001041F4E051C8F80010010705D56F
:10297000D8F8001041F46041C8F80010D8F80010F1
:10298000A26821F0F0011143C8F80010C0073FD140
:10299000D8F8F80300F00700A84207D988F8F853E0
:1029A000D8F8F80300F00700A8424BD1206841078F
:1029B00007D5D8F80010E26821F4E0511143C8F8B7
:1029C0000010000708D5D8F80000216920F4604005
:1029D00040EAC100C8F8000000F07EF8D8F8001006
:1029E0004CF60802C1F30311C0F60002515C40F23C
:1029F000000220FA01F140F23810C2F20000006833
:102A0000C2F200021160FFF725FF0020BDE8F0814F
:102A10006068811E022907D258F8081C89015CBF32
:102A20000120BDE8F08110E0012807D158F8081C0A
:102A300089035CBF0120BDE8F08106E058F8081C5E
:102A4000890702D40120BDE8F081D8F8001021F0F8
:102A500003010843C8F80000FFF786FD064641F26F
:102A6000883700BFD8F80000616800F00C00B0EBB8
:102A7000810F8DD0FFF778FD801BB842F2D903207B
:102A8000BDE8F08140F20000C2F20000006870472B
:102A900080B5FFF7F7FF43F60801C4F202010968A9
:102AA0004CF61802C1F38221C0F60002515CC84006
:102AB00080BD000080B5FFF7E5FF43F60801C4F2D2
:102AC000020109684CF61802C1F34231C0F6000257
:102AD000515CC84080BD000010B543F60404C4F248
:102AE0000204606800F00C0008280AD0042819BF0E
:102AF00042F20040C0F2F40041F60030C0F2B700EC
:102B000010BD206821682368490241F60031C0F2F7
:102B1000B70100F03F02C3F388105CBF42F20041EE
:102B2000C0F2F401A1FB00010023FDF7BDFB216809
:102B30000222C1F3014102EB4101B0FBF1F010BDF3
:102B40002DE9F04182B0002800F0A2800446007810
:102B500043F60006C007C4F2020643D0B06800F096
:102B60000C00042805D1306880033BD56068C8BBE1
:102B70008EE0B06800F00C00082802D170684002B6
:102B8000F1D46568B5F5A02F0AD0B5F5803F0BD01C
:102B9000306820F480303060306820F4802006E017
:102BA000306840F480203060306840F4803030601D
:102BB000FFF7DAFC002D054611D000BF3068800316
:102BC00010D4FFF7D1FC401B6428F7D922E100BFE5
:102BD000FFF7CAFC401B64284FF0030055D830684B
:102BE0008003F5D4207880071AD5B06810F00C0F58
:102BF00009D0B06800F00C00082840F08A807068A6
:102C0000400200F186803068800702D5E068012824
:102C10003ED13068216920F0F80040EAC100306000
:102C20002078000738D4207840074CD4A5695DB3DC
:102C3000B06800F00C00082840F09E80012D27D0DD
:102C40007068E16900F480028A4221D1216A00F0B3
:102C50003F028A421CD147F6C071626A0140B1EB63
:102C6000821F15D1A26A0023CFF6FF7303EBC23295
:102C700000F440316FF30F02914209D1E16A00F094
:102C80007060B0EB016F03D1002002B0BDE8F081AD
:102C9000012002B0BDE8F0816069002840F2000028
:102CA000C4F2472057D00121C0F8801EFFF75CFC1A
:102CB000054600BF706F8007B5D4FFF755FC401B79
:102CC0000228F7D9A6E0306C10F080580AD1002015
:102CD0000190306C40F080503064306C00F08050D7
:102CE0000190019847F20007C4F200073868C00558
:102CF00024D4386840F480703860FFF735FC05460E
:102D00003868C0051AD4FFF72FFC401B0228F7D9FA
:102D100080E0E068002851D00020C4F24720012163
:102D20000160FFF721FC0546306880073FF571AF71
:102D3000FFF71AFC401B0228F6D96BE0A568052DA9
:102D400050D0012D52D0306F20F001003067306F2D
:102D500020F004004DE00021C0F8801EFFF704FCC5
:102D6000054600BF706F80077FF55DAFFFF7FCFB86
:102D7000401B0228F6D94DE00027C4F24727002067
:102D80003866FFF7F1FB022D05460BD13068800154
:102D900058D5FFF7E9FB401B02284FF00300F5D997
:102DA00073E700BF306880017FF56EAFFFF7DCFB93
:102DB000401B02284FF00300F4D966E70020C4F25C
:102DC000472000210160FFF7CFFB054630688007F0
:102DD0007FF526AFFFF7C8FB401B02284FF003002A
:102DE000F4D952E7306F40F004003067306F40F0A4
:102DF00001003067FFF7B8FB002D054641F2883728
:102E000014D000BF306F800713D4FFF7ADFB401B19
:102E1000B842F7D9032002B0BDE8F081FFF7A4FB68
:102E2000401BB8424FF003003FF62FAF306F8007D2
:102E3000F4D4B8F1000F7FF4F9AE306C20F080507C
:102E40003064F3E604F11C052FCD08430021CFF6D2
:102E5000FF7140EA821001EBC3316FF30F0140EACA
:102E600005600843706001203866FFF77DFB04466B
:102E7000306880013FF508AFFFF776FB001B0228A2
:102E80004FF00300F4D900E780B502F0E9FF022813
:102E900008BF80BD40F20021C2F2000101EB4010EA
:102EA0008069002818BF804780BD000070B538B128
:102EB0000446406A30B10020206104F1140007E0AC
:102EC000012070BD6068B0F5827F03D004F11C0062
:102ED000002101600026A66294F8510020B9204626
:102EE00084F8506000F03CF8022084F8510094E827
:102EF0000F0001F48271056802F4044225F04005D8
:102F00000560114403F400622369114403F00202D6
:102F10006369114403F00102A369E569114403F4F4
:102F20000072114405F03802256A114405F0800250
:102F3000A56A114305F4005211430160626A04213D
:102F400001EA134102F0100211444160C16921F409
:102F50000061C1610120666584F85100304670BD92
:102F60002DE9F04F87B0044643F200070068C4F231
:102F700001070026B8420696CDE90466039602963C
:102F800002D007B0BDE8F08F43F630000196C4F2DE
:102F90000200416902AD41F48051416141694FF045
:102FA000020901F4805101910199019601684FF0E5
:102FB000010A41F00201016001684FF0030B01F0CA
:102FC000020101910199019601684FF0050841F055
:102FD000010101600068294600F00100019001989C
:102FE0001820029007F55440CDF80C90CDF810A0B1
:102FF000CDF814B0CDF81880FFF7DCF9802002A9D5
:1030000081E8010ECDF8188046F2404807F550409F
:103010002946C4F20208FFF7CDF940F2F835C2F2B2
:1030200000054FF0C0674FF480692846C5E9008766
:10303000C5E90266C5E90496C5E90666C5E90866FC
:10304000FFF7E6F8002818BFFEF7C6FFE564AC639B
:1030500040F2584508F11800C2F200054021C5E9C8
:10306000000705F10800002280E806022846C5E9AD
:103070000522C5E907226A62FFF7CAF8002818BFCF
:10308000FEF7AAFFA564AC6307B0BDE8F08F0000AF
:103090002DE9F04182B0044690F85100012815D185
:1030A0000E4600294FF0010060D01746002A5DD07F
:1030B00060681D46B0F5827F02D1A068002858D014
:1030C000FFF752FA94F85010012903D1022002B000
:1030D000BDE8F0818046012084F85000042084F887
:1030E000510000206065A663A787E7872063A0865C
:1030F000E086A1682064B1F5004F606408D12068C3
:10310000016821F040010160016821F48041016003
:1031100020680168490603D4016841F0400101605C
:10312000E168E08F91B3002855D06E1C0BE000BF22
:10313000C068A16B21F8020BA163E08F0138E08722
:10314000E08F002847D020688168C907F0D1FFF7D9
:103150000BFA002EF4D0A0EB0800A842F0D3012017
:1031600084F85100002084F85000032002B0BDE82C
:10317000F081042084F851002046314632463B4617
:10318000009500F09FF902B0BDE8F08118B36E1C05
:103190000BE000BF007BA16B0870A06B0130A06347
:1031A000E08F0138E087E08FA8B120688168C90707
:1031B000F0D1FFF7D9F9002EF5D0A0EB0800A84216
:1031C000F1D3012084F85100002084F8500003203E
:1031D00002B0BDE8F08120462946424602F0B2FD29
:1031E00000281CBF20206065012084F851000020C9
:1031F00084F85000606D002818BF012002B0BDE8BF
:10320000F081000010B5044690F8510001281CBF61
:10321000022010BD13460A4600294FF0010018BFD6
:10322000002B00D110BDA06858B96168B1F5827F4C
:1032300007D1042084F851002046114600F03EFAE0
:1032400010BD94F85010012904BF022010BD0121C7
:1032500084F85010042184F851100021B0F5004F7B
:103260006165A263A387E387C4E91011A186E186A3
:1032700008D12068036823F040030360036823F447
:1032800080430360E06C45F6ED3E45F61143C0F621
:10329000000EC0F60003C0E90F3E45F6C933C0F684
:1032A0000003D4F800C0C0E91331E38F0CF10C0126
:1032B000FFF716F840B1606D40F010006065002027
:1032C00084F85000012010BD21680868400603D42E
:1032D000086840F040000860002084F850004A6808
:1032E00042F020024A604A6842F001024A6010BD82
:1032F00080B502F0B5FD022808BF80BD40F2002174
:10330000C2F2000101EB40104068002818BF80475E
:1033100080BD000080B502F0A3FD022808BF80BD7B
:1033200040F20021C2F2000101EB401000690028C8
:1033300018BF804780BD00002DE9F04182B01D46D6
:1033400016460F460446FFF70FF994F8511001296D
:103350000DD18046002F4FF0010018BF002E02D182
:1033600002B0BDE8F08194F85000012803D102209A
:1033700002B0BDE8F081012084F85000032084F8F9
:103380005100002060652763A686E686A063A087BB
:10339000E087A168C4E91000B1F5004F08D12068AA
:1033A000016821F040010160016841F48041016041
:1033B00020680168490603D4016841F040010160BA
:1033C0006168731EE268B1FA81F1B3FA83F34909C7
:1033D0005B09B2F5006F41EA030124D139B1216BD9
:1033E0000988C160B81C2063E08E0138E086E08E59
:1033F000002846D06E1C09E0216B31F8022BC26018
:103400002163E08E0138E086E08ED0B320688168C9
:103410008907F1D4FFF7A8F8002EF5D0A0EB08003B
:10342000A842F1D323E039B139780173206B013020
:103430002063E08E0138E086E08E10B36E1C0AE057
:10344000216B09780173206B01302063E08E013815
:10345000E086E08EA8B1206881688907F0D4FFF784
:1034600083F8002EF5D0A0EB0800A842F1D301208C
:1034700084F85100002084F85000032002B0BDE819
:10348000F08120462946424602F0A4FC00281CBFD9
:1034900020206065A06838B9002001902068C168CC
:1034A0000191806801900198012084F8510000206A
:1034B00084F85000606D002818BF012002B0BDE8FC
:1034C000F08100002DE9F04381B01E4615460F46FD
:1034D0000446FFF749F894F851108146012909D0B4
:1034E0006068B0F5827F14D104294FF0020007D143
:1034F000A16829B9002F4FF0010018BF002D02D19B
:1035000001B0BDE8F083002EFAD094F850000128F5
:1035100003D1022001B0BDE8F083012084F85000FF
:1035200094F85100002104281CBF052084F85100A4
:103530006165A563E687A6872763E6862068A68679
:10354000216461640168490603D4016841F04001C7
:1035500001606168731EE268B1FA81F1B3FA83F326
:10356000DDF8208049095B09B2F5006F41EA0301EB
:1035700039D139B1216B0988C160B81C2063E08E54
:103580000138E086012608F1010500BFE08E10B980
:10359000E08F00286CD02068816889070CD5E18E07
:1035A000012E09D141B1216B002631F8022BC260F6
:1035B0002163E18E0139E1868168C9070AD0E18F74
:1035C00041B1C068A16B012621F8020BA163E08F15
:1035D0000138E087FEF7C8FF002DD7D0A0EB090027
:1035E0004045D3D33AE039B139780173206B0130CB
:1035F0002063E08E0138E086012608F1010500BF56
:10360000E08E08B9E08F98B32068816889070DD5EE
:10361000E18E012E0AD149B1216B00260978017390
:10362000206B01302063E08E0138E08620688168DD
:10363000C9070BD0E18F49B1C068A16B01260870A2
:10364000A06B0130A063E08F0138E087FEF78CFFAC
:10365000002DD5D0A0EB09004045D1D3012084F83E
:103660005100002084F85000032001B0BDE8F08331
:10367000204641464A4602F0ADFB40B1202060653D
:10368000002084F85000012001B0BDE8F083A0685C
:1036900038B9002000902068C168009180680090CF
:1036A0000098012084F85100002084F85000606DDB
:1036B000002818BF012001B0BDE8F08370B50446B2
:1036C00090F85100012806D100294FF0010018BFE1
:1036D000002A0CD170BD6568B5F5827F0ED1042833
:1036E0004FF00200F6D1A568002DEDD0F2E7002BD7
:1036F00008BF70BD94F85000012801D1022070BDB0
:10370000012084F8500094F85100002604281CBFC2
:10371000052084F8510066652163A386E386A263D1
:10372000A387E387C4E9106694F8510045F6ED31AC
:1037300045F60543C0F60001C0F60003042808BFA3
:103740000B4645F6114045F6E941C0F60000C0F6CB
:10375000000108BF0146E06C2568C0E90F1345F67B
:10376000C931C0F60001C0E91316E38F05F10C0161
:10377000FEF7B6FD38B1606D40F0100060650120C5
:1037800084F8506070BD2268216BA06C536843F0D0
:1037900001035360C0E90F66C0E91366E38E0C3283
:1037A000FEF79EFD40B1606D40F0100060650020A6
:1037B00084F85000012070BD21680868400603D4D9
:1037C000086840F040000860002084F850004A6813
:1037D00042F020024A604A6842F002024A6070BD2C
:1037E00010B5044690F8510001280AD100294FF085
:1037F000010018BF002A00D110BD94F85000012824
:1038000001D1022010BD012084F8500003200023C4
:1038100084F8510063652163A286E286A363C4E94C
:103820001033A387E387A068B0F5004F08D1206864
:10383000026822F040020260026842F480420260A4
:10384000A06C45F6F93C45F67942C0F6000CC0F68E
:103850000002C0E90F2C45F6C932C0F60002D4F8C8
:1038600000E0C0E91323E38E0EF10C02FEF738FDF1
:1038700040B1606D40F010006065002084F8500099
:10388000012010BD21680868400603D4086840F094
:1038900040000860002084F850004A6842F020028E
:1038A0004A604A6842F002024A6010BD80B502F0E8
:1038B000D7FA022808BF80BD40F200214001C2F2C1
:1038C00000010858002818BF804780BD80B502F06D
:1038D000C7FA022808BF80BD40F20021C2F20001F1
:1038E00001EB4010C068002818BF804780BD000071
:1038F00080B502F0B5FA022808BF80BD40F2002171
:10390000C2F2000101EB40108068002818BF804718
:1039100080BD000080B502F0A3FA022808BF80BD78
:1039200040F20021C2F2000101EB40104069002882
:1039300018BF804780BD000080B502F035FC80BD17
:10394000B0B590F83C20012A04BF0220B0BD01F1BF
:1039500008053CCDD1E900CE23F47C5322F470520B
:103960001A432EF4F0431A432CF4E0431A4324F490
:10397000C0431A432A43C96922F4804203681143B1
:103980005964002180F83C100846B0BD10B590F88D
:103990003C20012A4FF0020252D0012380F83C3033
:1039A00080F83D200268D2F804E0D2F808C00C6824
:1039B0002EF07003234341F2FF74C4F20004A242CC
:1039C00053600DDC40F2FF73C4F200039A4215DC31
:1039D000B2F1804F29D040F20043C4F2000322E04C
:1039E00040F2FF33C4F201039A4212DC41F60003B5
:1039F000C4F200039A4218D0002312E040F60003FC
:103A0000C4F200039A4210D040F60043C4F200030F
:103A100009E044F20003C4F201039A4205D040F2E7
:103A20000043C4F201039A4204D149682CF0800398
:103A3000194391600121002280F83D1080F83C205C
:103A4000104610BD002804BF0120704710B5044681
:103A500090F83D0028B9002084F83C00204600F092
:103A60001FF8022084F83D002068211D02F01AFC96
:103A7000012084F8460084F83E0084F83F0084F872
:103A8000400084F8410084F8420084F8430084F840
:103A9000440084F8450084F83D00002010BD00007B
:103AA00081B0006844F20041C4F20101884201D0B3
:103AB00001B070470020009043F64400C4F20200B9
:103AC000016841F400310160006800F400300090AA
:103AD000009801B07047000080B586B000684FF6CE
:103AE000FF71C4F2000188424FF000010591CDE959
:103AF0000311CDE9011129DC40F60001C4F20001F7
:103B000088424AD040F60041C4F20001884240F0A9
:103B100082804FF0000C43F63000CDF800C0C4F2B4
:103B200002000268002342F0800202600068022264
:103B300000F08000009000984FF4E050019040F6B3
:103B40000040C4F2020000F580505CE044F2004105
:103B5000C4F2010188423BD00021C4F20101884235
:103B600059D14FF0000C43F63000CDF800C0C4F23C
:103B70000200026842F0100202600068012200F0B8
:103B80001000009000984FF4D440019040F600409F
:103B9000C4F2020000F5806034E04FF0000C43F600
:103BA0003000CDF800C0C4F202000268002342F0E9
:103BB000080202600068022200F0080000900098ED
:103BC0004FF48040019040F60040C4F202001AE039
:103BD0000020009043F63000C4F202000168032286
:103BE00041F02001016000684FF0020C00F020005D
:103BF000009000984020019040F60040C4F202007E
:103C000000F5006002230221CDE9021C01A9CDE9E3
:103C10000432FEF7CFFB06B080BD0000B0B504460D
:103C200090F83C00012804BF0220B0BD0D464FEAC9
:103C3000B2010120032984F83C0037D8DFE801F005
:103C4000020A12222068294602F0D4FB206850F8AC
:103C5000181F0EE02068294602F0FEFB206850F88D
:103C6000181F16E02068294602F02CFC206850F846
:103C70001C1F41F008010160016821F0040101608E
:103C800029690FE02068294602F050FC206850F8AE
:103C90001C1F41F400610160016821F48061016032
:103CA000296909020268114301600020002184F89B
:103CB0003C10B0BD002804BF0120704710B5044679
:103CC00090F83D0028B9002084F83C00204600F020
:103CD0001FF8022084F83D002068211D02F0E2FA5E
:103CE000012084F8460084F83E0084F83F0084F800
:103CF000400084F8410084F8420084F8430084F8CE
:103D0000440084F8450084F83D00002010BD000008
:103D100083B0006840F60001C4F2000188421BD065
:103D200040F60041C4F20001884226D00021C4F2CE
:103D30000101884230D10020029043F64000C4F2D5
:103D40000200416841F001014160406800F001005B
:103D50000290029803B070470020019043F64000A3
:103D6000C4F20200016841F004010160006800F043
:103D700004000190019803B070470020009043F6C2
:103D80004000C4F20200016841F0080101600068CF
:103D900000F008000090009803B0704710B504468A
:103DA00041B1082909D0042914BF04F1410004F1EC
:103DB0003F0004E004F13E0001E004F1400000781F
:103DC00001281CBF012010BD022041B1082909D0E3
:103DD000042914BF84F8410084F83F0004E084F80B
:103DE0003E0001E084F840002068012202F0F0FA71
:103DF000206841F2FF71C4F2000188420FDC40F2FA
:103E0000FF71C4F20001884217DCB0F1804F49D045
:103E100040F20041C4F20001884243D049E040F240
:103E2000FF32C4F20102904214DC41F60003C4F2F6
:103E30000003984236D0002314E040F60001C4F29B
:103E4000000188422ED040F60041C4F200018842B1
:103E500028D02EE044F20003C4F20103984221D09E
:103E600040F20043C4F20103984222D1436C8842DD
:103E700043F400434364C2DD904207DC41F6000195
:103E8000C4F2000188420DD0002107E044F2000195
:103E9000C4F20101884205D040F20041C4F20101A0
:103EA000884206D1816801F00701062904BF00207D
:103EB00010BD016841F001010160002010BD00004B
:103EC000B0B50446006800220D4602F081FA206871
:103ED00040F2004240F48061C4F2010291420DD1EF
:103EE000016A41F21112114208D1016A40F24442C2
:103EF000114203D1416C21F400414164016A41F255
:103F00001112114208D1016A40F24442114203D118
:103F1000016821F0010101600120082D09D0042D64
:103F20000BD0002D14BF84F8410084F83E0000201F
:103F3000B0BD84F840000020B0BD84F83F000020F0
:103F4000B0BD00007047000080B502F049FE0328B4
:103F500008BF80BD40F2202100EBC000C2F200018A
:103F600001EB80000069002818BF804780BD000079
:103F7000B0B582B0036804461868D9685A6900F081
:103F80002F05202D01F0200505D125B1204602F096
:103F900037FE02B0B0BD5FEA007C1EBF02F0010E2A
:103FA00001F4907212EB0E024AD1226B0840C10656
:103FB0003DD5012A3BD10020019018680190586836
:103FC000019001985869400642D4A08DE18DE28DA0
:103FD000002A1CBF401A5FEA004101D102B0B0BD07
:103FE000216851E8031F226821F4907142E803130D
:103FF000002BF5D1216851E8051F226821F001014D
:1040000042E80513002BF5D1202184F8421000214D
:10401000216300BF216851E8031F226821F01001CD
:1040200042E80313002BF5D10221616354E001063D
:1040300054D44006D2D5204602F0B8FD02B0B0BD3F
:10404000C20718BF11F480725DD1420761D467E0E6
:10405000E06B016849688AB2002A44D0A38D9A4275
:1040600041D2E185C069B0F5807F30D0206850E84A
:10407000030F216820F4807041E80302002AF5D183
:10408000206850E8050F216820F0010041E8050292
:10409000002AF5D1206850E8050F216820F0400083
:1040A00041E80502002AF5D1202084F842000020D2
:1040B000206300BF206850E8030F216820F0100043
:1040C00041E80302002AF5D1E06BFDF789FF0220E9
:1040D0006063A08DE18D401A81B20FE0204602F0AE
:1040E000B7FE02B0B0BDA18D91427FF477AFC06939
:1040F000B0F5807F7FF472AF022060632046FFF747
:1041000021FF02B0B0BD626C42F00102626442075E
:1041100006D5BEF1000F03D0626C42F00202626469
:10412000820706D5BEF1000F03D0626C42F0040294
:104130006264BCF1000F06D55EEA050203D0626C32
:1041400042F008026264626C002A3FF447AF084004
:10415000800602D5204602F053FD20684069616C5C
:1041600000F0400001F00801401827D0204602F07E
:10417000F5FC2068406940061BD500BF206850E868
:10418000050F216820F0400041E80502002AF5D122
:10419000E06B70B146F65D21C0F600010165FDF7E8
:1041A0005FFF00283FF41AAFE06B016D884702B053
:1041B000B0BD2046FFF7C8FE02B0B0BD2046FFF7F5
:1041C000C3FE0020606402B0B0BD0000002804BF40
:1041D0000120704710B5044690F8410028B900202E
:1041E00084F84000204600F021F8242084F84100A3
:1041F0002068C16821F40051C160204602F064FDCE
:104200002068016921F490410161416921F02A018E
:104210004161C16841F40051C16000202021606407
:1042200084F8411084F84210606310BD2DE9F0431A
:1042300087B00446006841F20041C4F20101002643
:104240008842CDE90566CDE90366029651D044F671
:104250000001C4F20001884240F0BB80002643F612
:1042600030000196C4F20200016941F4802101612D
:10427000016901F48021019101990196016841F0E1
:1042800004010160006802A900F004000190019897
:104290004FF4406002900220CDE903060320059010
:1042A0000720069040F60000C4F20200FEF782F8F4
:1042B00040F2B84546F22800C2F20005C4F20200FE
:1042C0004FF000614FF4806285E843002846C5E95D
:1042D0000362C5E90566C5E907666E62FDF798FFEA
:1042E000002818BFFDF778FEE563AC6307B0BDE8B2
:1042F000F08343F630000196C4F20200416946F2B1
:10430000280841F0200141614169C4F2020801F02E
:104310002001019101990196016841F0400101607D
:10432000006802A900F04000019001984FF4844019
:1043300002900220CDE90306032005900820069094
:1043400040F60000C4F2020000F58050FEF732F89B
:1043500040F2185508F58060C2F200054FF0206762
:104360004FF48069C5E900072846C5E90266C5E93A
:104370000496C5E90666C5E90866FDF749FF002809
:1043800018BFFDF729FEE563AC6340F2785508F5E8
:104390008F60C2F200054021C5E9000705F1080061
:1043A000002280E806022846C5E90522C5E9072261
:1043B0006A62FDF72DFF002818BFFDF70DFE4720AC
:1043C00005210022A563AC63FEF798FA4720FEF7AB
:1043D00091FA07B0BDE8F08380B590F84230202B09
:1043E0001CBF022080BD00294FF0010318BF002A26
:1043F00001D1184680BD0023036302F0D3FC0346BD
:10440000184680BD80B502F0EBFB032808BF80BDD5
:1044100040F2202100EBC000C2F2000101EB80005D
:10442000C068002818BF804780BD000080B502F03A
:10443000D7FB032808BF80BD40F2202100EBC0005D
:10444000C2F2000101EB80008068002818BF80479D
:1044500080BD000080B502F0C3FB032808BF80BD0B
:1044600040F2202100EBC000C2F2000101EB80000D
:104470004068002818BF804780BD0000FEE70000AC
:10448000F0B581B02DED028B0C46054600F0C8F862
:10449000FDF706FA07F09FFF9FED238A00EE100A52
:1044A00080EE080A10EE100A08F062F840F2F012EE
:1044B000C2F20002C2E90001FDF7F2F940F2E8168B
:1044C000C2F20006D6E90023801A994107F083FF63
:1044D00000EE100A80EE080A40F2E017C2F2000770
:1044E00087ED000AFDF7DCF940F26822C2F2000213
:1044F00092ED000A41F26822C2F20002C6E9000110
:1045000040F29826D2ED000A97ED001AC2F200069A
:104510003046FCF7CDFD30682860716800202160CE
:10452000BDEC028B01B0F0BD00247449F0B581B040
:104530002DED028B82B0B0EE408A01F04DFD64207B
:10454000FDF772F940F27020C2F20000F3EE0E0A9D
:10455000B0EE480A00F0B4FA41F26C20C2F200005A
:10456000F1EE040AB0EE480A00F0AAFA40F29820F0
:10457000C2F20000FCF784FD40F67C06C2F20006A1
:10458000308863281AD841F2303440F68C0540F662
:104590007807C2F20004C2F20005C2F2000700BFB1
:1045A0002046294601F04CFD286801F0D5FC3188F1
:1045B0003860481C81B264293080F1D39FED168A9F
:1045C00041F2BC250020C2F2000501AC3080019010
:1045D000A86921460022002302F00CFE30889DEDE0
:1045E000010A01303080142038EE008A02F050FDBC
:1045F00030886428ECD39FED090A40F2943188EEAC
:10460000000AC2F20001002081ED000A02B0BDECF8
:10461000028B01B0F0BD00BF000000000000C842E6
:1046200010B52DED028B40F68C0441F23030C2F211
:104630000004C2F200002146B0EE408A01F000FD05
:10464000206801F089FC40F67801C2F20001096897
:104650009FED211A411A00EE101AB8EEC00A80EE42
:10466000010A40F2D851C2F20001086041F268200C
:10467000C2F2000080ED000A41F26C20C2F200009C
:1046800000F0E0F941F28C20C2F2000080ED000A57
:1046900040F27020C2F20000B0EE480A00F0D2F9F9
:1046A00040F29020C2F2000080ED000A40F2943007
:1046B000C2F2000090ED001A9FED082A30EE410A88
:1046C00040F2682120EE020AC2F20001002081EDD2
:1046D000000ABDEC028B10BD00007A440AE81C41C0
:1046E00010B541F20044C4F2020420460221002227
:1046F000FDF734FF01F056FA204601210022FDF7B4
:104700002DFF0220FDF7BCF8204602210122FDF713
:1047100025FF0220FDF7B4F8204602210022FDF714
:104720001DFF204601210122FDF718FF10BD0000EA
:1047300010B541F20044C4F20204204602210022D6
:10474000FDF70CFF01F02EFA204601210122FDF7B2
:1047500005FF0420FDF794F8204602210122FDF711
:10476000FDFE0420FDF78CF8204602210022FDF713
:10477000F5FE204601210122FDF7F0FE10BD0000EC
:10478000F0B581B041F200450446C4F2020501F0E3
:10479000F7F90026002700BF284602210022FDF776
:1047A000DDFE0220FDF76CF8284602210122FDF70C
:1047B000D5FE28460121FDF7CBFE002818BF0120B9
:1047C00040EA46060120FDF75BF8072F07F10107D5
:1047D000E2D314B1FFF784FF01E0FFF7A9FFF0B2C5
:1047E00001B0F0BD70B541F200450446C4F20205C7
:1047F00001F0D8F92846022100220026FDF7AEFE7E
:10480000E0B2C20928460121FDF7A8FE022064009B
:10481000FDF736F8284602210122FDF79FFE02200F
:10482000FDF72EF8284602210022FDF797FE022010
:10483000FDF726F8072E06F10106E1D370BD000052
:1048400010B501F0AFF941F20044C4F20204204671
:1048500001210122FDF782FE204602210122FDF7FF
:104860007DFE0420FDF70CF8204601210022FDF713
:1048700075FE0420FDF704F8204602210022FDF712
:104880006DFE10BD10B501F08DF941F20044C4F287
:104890000204204602210122FDF760FE204601218C
:1048A0000022FDF75BFE0420FCF7EAFF2046012111
:1048B0000122FDF753FE0420FCF7E2FF10BD0000CB
:1048C000B0B541F20044C4F2020401F059F92046A7
:1048D00001210122FDF742FE0120FCF7D1FF204615
:1048E00002210122FDF73AFE0120FCF7C9FF002555
:1048F00020460121FDF72CFE38B1642D05F101059C
:10490000F6D3FFF7BFFF0120B0BD204602210022F1
:104910000024FDF723FE2046B0BD000045F6DF1160
:1049200010EE100AC5F63771B6EE001AA1EB600062
:1049300020EE011A00EE100A21EE002A22EE002AD3
:10494000B7EE083A33EE422A22EE000A21EE001AB0
:1049500020EE011A33EE411A20EE010A70470000E2
:1049600041F26F2C49F6A6324CF28F23C3F6832C0A
:10497000C3F64432C3F6F5430021C0E900C2C0E9E2
:104980000231C0E90411C0E906110162704700005C
:1049900090ED086A90ED065A90ED077A66EE011ADE
:1049A00090ED002A71EEC52A72EEC72A90ED054AF5
:1049B00032EE822A90ED023A22EE012A34EE022AE9
:1049C00032EE033A37EE617A82EE034A87EE033A1B
:1049D000D0ED043AD0ED012AD0ED034A70EEE30A9F
:1049E00060EE810A74EEA00A22EE811A36EE011AF8
:1049F00030EE606A35EE615A26EE040A26EE036A4E
:104A000033EE866A80ED046A22EE046A32EE466A6C
:104A100022EE032A37EE422A25EE044A80ED072AC9
:104A200025EE032A30EE800A35EE444A31EE421A72
:104A300080ED030A80ED056A80ED064A80ED081AD4
:104A40007047000010B52DED088B88B3B0EE408A9A
:104A500090ED010A90ED069A90ED021A90ED07AAEA
:104A600029EE000A38EE400A2AEE011A30EE41BA69
:104A700004461BEE100A02F033FA002808BFB0EE1D
:104A80004B8A94ED030A94ED041A94ED052A20EE66
:104A9000080A29EE011A30EE010A2AEE021A30EE57
:104AA000010A84ED068A84ED079ABDEC088B10BDDF
:104AB0009FED020ABDEC088B10BD00BF0000000096
:104AC000002808BF704710B5F5EE400A0446C0ED57
:104AD000000A0020F1EE10FAA061E0612EDD80EE08
:104AE000200A9FED1E1A81EE000A06F039FB9FEDA9
:104AF0001C1AB7EE002A20EE011A31EE023A20EE1F
:104B0000000ABFEE005A30EE033A30EE055A32EE9C
:104B1000411A80EE034A35EE055A30EE010A85EE61
:104B2000035A80EE030A34EE041A84ED034A84ED3E
:104B3000041A84ED054A84ED015A07E04FF07E51D6
:104B40009FED050AC4E903106061606084ED020A0C
:104B5000BDE81040704700BF00000000DB0F494077
:104B6000F304B53F10B52DED048B10B3B0EE408AC1
:104B700090ED030A90ED041A90ED052A30EE010A3B
:104B800030EE020A88EE009A044619EE100A02F08E
:104B900097F900282046B0EE480A08BFB0EE489AC0
:104BA00084ED069A84ED079AFFF74CFFBDEC048B69
:104BB00010BD9FED020ABDEC048B10BD000000008B
:104BC00080B582B0002043F630010190C4F20201AA
:104BD0000A6842F400120A600A6802F400120192A4
:104BE000019A00900868002240F48000086008687C
:104BF000052100F48000009000980C20FDF77EFE57
:104C00000C20FDF777FE0D2005210022FDF776FE32
:104C10000D20FDF76FFE392005210022FDF76EFE05
:104C20003920FDF767FE3A2005210022FDF766FED8
:104C30003A20FDF75FFE3B2005210022FDF75EFED6
:104C40003B20FDF757FE452005210022FDF756FECB
:104C50004520FDF74FFE02B080BD000080B546F252
:104C60009D104CF67012C0F60000C0F60002002144
:104C700002F03EFC40F25C31C2F20001086046F2F4
:104C80007D504CF62812C0F60000C0F6000200214C
:104C900002F02EFC80BD00002DE9F04F87B0002708
:104CA00043F630000697CDE90477CDE90277019706
:104CB000C4F20200016841F6000441F040010160C5
:104CC0000168C4F2020401F04001019101990197C9
:104CD0000168A4F5806541F00201016001680022CD
:104CE00001F0020101910199019701684FF0030A57
:104CF00041F001010160016801F001010191019998
:104D00000197016841F004010160016801F00401AC
:104D1000019101990197016841F02001016001684A
:104D200001F02001019101990197016841F0800192
:104D30000160016801F0800101910199019701680A
:104D400041F008010160016801F008010191019939
:104D50000197016841F0100101600068032100F033
:104D60001000019001982846FDF7F8FB20464021ED
:104D700000224FF0400BFDF7F1FBA4F5C059484667
:104D8000102101220126FDF7E9FBA4F5A0584046B9
:104D900001210122FDF7E2FB112003A9C1C102AFED
:104DA00028463946CDF808A0FDF704FB20463946D1
:104DB000CDE902B6CDE90466FDF7FCFA08200290C1
:104DC0004FF4041520463946CDE90356FDF7F2FAB3
:104DD0001020CDE9020648463946CDE90466FDF7C4
:104DE000E9FA302002A961C1A4F580503946FDF7E7
:104DF000E1FA40463946CDE90266CDE90466FDF7A1
:104E0000D9FA092005210022FDF778FD0920FDF7D8
:104E100071FD0A2005210022FDF770FD0A20FDF733
:104E200069FD172005210022FDF768FD1720FDF719
:104E300061FD07B0BDE8F08F80B540F2DC5045F66B
:104E40000041C2F20000C4F2000141F680220023BA
:104E50004FF4804CC0F2060280E80E00C0E9033C2B
:104E6000C0E90533C0E90733FDF784FB002818BF0C
:104E7000FDF7B2F880BD0000B0B540F2306043F2FB
:104E80000001C2F20000C4F201014FF4827200235B
:104E900080E80E0000F10C014FF0020C4FF0010E03
:104EA0004FF40074182581E808500A21C0E906452E
:104EB000C0E90833C0E90A31FDF7F8FF002818BF40
:104EC000FDF78AF8B0BD000080B588B040F2D06030
:104ED00044F200420021C2F20000C4F201024FF687
:104EE000FF730791CDE90511CDE90311CDE901115A
:104EF000C0E90021C0E9021301618161FEF7A2FD52
:104F0000002818BFFDF768F840F2D060C2F2000038
:104F1000FEF7D0FE002818BFFDF75EF86020019074
:104F20000020CDE90200059040F2D060C2F20000FE
:104F300001A90022FEF772FE002818BFFDF74CF809
:104F400040F2D060C2F20000FEF7C6FD08B080BD9E
:104F500010B592B040F2886000210024C2F2000037
:104F6000C4F201014FF6FF731194CDE90F44CDE96E
:104F70000D44CDE90B44CDE90944CDE90744CDE921
:104F80000544CDE90344CDE90144A72280E8160099
:104F9000C0E90334C0E90544FEF78CFE002818BFC1
:104FA000FDF71AF840F28860C2F2000010A9CDE9BE
:104FB0001044FEF7EBFC002818BFFDF70DF8602049
:104FC00009900020CDE90A00CDE90C00CDE90E00E2
:104FD00040F28860C2F2000009A90022FEF71EFE1E
:104FE000002818BFFCF7F8FF40F28860C2F200000A
:104FF00009A90422FEF712FE002818BFFCF7ECFFF7
:1050000040F28860C2F2000009A90822FEF706FEFD
:10501000002818BFFCF7E0FF40F28860C2F20000F1
:1050200009A90C22FEF7FAFD002818BFFCF7D4FFEF
:1050300000200590CDE90300CDE901004FF40051B7
:10504000089040F288600691C2F2000001A9FEF7C4
:1050500077FC002818BFFCF7BFFF40F28860C2F25F
:105060000000FEF739FD12B010BD000010B58AB087
:1050700040F2187040F600010024C2F20000C4F2B1
:1050800000014FF6FF730994CDE90744CDE90544CB
:10509000CDE90344CDE90144A72280E81600C0E928
:1050A00003348461FEF706FE002818BFFCF794FF66
:1050B00040F21870C2F2000008A9CDE90844FEF7DA
:1050C00065FC002818BFFCF787FF602001900020D6
:1050D000CDE90200059040F21870C2F2000001A96B
:1050E0000822FEF79BFD002818BFFCF775FF40F271
:1050F0001870C2F20000FEF7EFFC0AB010BD00000D
:1051000010B58AB040F2607040F600410024C2F24F
:105110000000C4F200014FF6FF720994CDE9074484
:10512000CDE90544CDE90344CDE90144C0E90014CB
:10513000C0E9024204618461FEF7BCFD002818BF8B
:10514000FCF74AFF40F26070C2F2000008A9CDE906
:105150000844FEF71BFC002818BFFCF73DFF602049
:1051600001900020CDE90200059040F26070C2F28B
:10517000000001A90022FEF751FD002818BFFCF72E
:105180002BFF40F26070C2F2000001A90422FEF77A
:1051900045FD002818BFFCF71FFF40F26070C2F207
:1051A000000001A90822FEF739FD002818BFFCF70E
:1051B00013FF40F26070C2F20000FEF78DFC0AB0EF
:1051C00010BD000080B540F2A87044F60001C2F2A4
:1051D0000000C4F2000148F2A06200234FF00C0C62
:1051E000C0F2010280E80E00C0E90333C0E905C344
:1051F000C361FEF7EBFF002818BFFCF7EDFE80BD92
:1052000080B540F2F07041F20041C2F20000C4F2F9
:10521000010100234FF00C0C4FF4E13280E80E0046
:10522000C0E90333C0E905C3C361FEF7CFFF00281F
:1052300018BFFCF7D1FE80BDFEE70000FEE70000CE
:1052400000F0070080F00703042B28BF04234FF071
:10525000FF3C03380CFA03F338BF00209943814028
:105260000CFA00F022EA000008437047B0B52DEDBB
:105270000A8B044610EE100AB0EE618AB0EE419A35
:10528000B0EE60AAB0EE40BA01F022FE002800F0B5
:105290009C801AEE100A01F01BFE002800F0958099
:1052A00019EE100A01F014FE002800F08E8018EEAE
:1052B000100A01F00DFE002800F087806068B0EE53
:1052C0004B0A90ED071AF0EE4A0AFCF737FC6068CB
:1052D000B0EE40BA90ED001A04F11C0020EE01CAB5
:1052E00021EE0A0AFFF7AEFB207888B1012811D120
:1052F00094ED051A94ED022A30EE411AB4EE428A7A
:10530000F1EE10FAC8BFB0EE482A81EE029A01E031
:105310009FED309A19EE100A84ED04BA84ED050A67
:1053200001F0D6FD65689FED2B0A002808BFB0EE9E
:10533000409A95ED010A95ED032A2CEE000A29EE1C
:10534000022A95ED021A30EE42AA94ED030A9FED6F
:10535000229A2CEE082A32EE008AB4EE491AF1EEB7
:1053600010FA28EE01BA1ADD18EE100A01F0B0FDAD
:10537000A8B13AEE0B0A95ED051AB0EEC00AB4EEEC
:10538000410AF1EE10FA0ADC95ED040AB0EEC81AF3
:10539000B4EE401AF1EE10FAD8BF84ED038A3AEE6B
:1053A0000B8A18EE100A01F093FD70B1D5ED050AD5
:1053B000F4EE490AF1EE10FA05DDB0EE480AFBF70B
:1053C0004DFEB0EE408A84ED068A94ED060ABDECEF
:1053D0000A8BB0BD00000000BD37863570B52DEDDD
:1053E000048B90B3044650681646B0EE408A0D46D2
:1053F00001F06EFD58B3B06801F06AFD48B3F06883
:1054000001F066FD38B3306901F062FD28B37069C0
:1054100001F05EFD18B3B7EE000A80EE089A6660F0
:1054200019EE100A01F054FDD8B1D6ED060A04F1C8
:105430001C00B0EE480A84ED029AFFF741FB2046BB
:10544000257000F013F800200CE0FF200AE0FF2098
:1054500008E0FF2006E0FF2004E0FF2002E0FF203C
:1054600000E0FF2040B2BDEC048B70BD10B568B108
:1054700000F11C0100249FED070AC0E90344C0E9C4
:1054800005440846FFF76EFB60B210BDFF2460B212
:1054900010BD00BF00000000000000000000000080
:1054A000EFF30980BFF36F8F154B1A681EF0100FD2
:1054B00008BF20ED108A20E9F04F10602DE90900A7
:1054C0004FF0500080F31188BFF34F8FBFF36F8F01
:1054D00003F050FA4FF0000080F31188BDE8090096
:1054E00019680868B0E8F04F1EF0100F08BFB0EC64
:1054F000108A80F30988BFF36F8F704700BF00BF29
:105500008409002010B52DED028B9FED118AD0ED9E
:10551000021AD0EDF10A90EDF50A04465830B0EECB
:10552000481AFFF7A3FE84EDF80AD4ED021AD4ED71
:10553000F00A94EDF60A04F1D000B0EE481AFFF735
:1055400095FE002084EDF90ABDEC028B10BD00BF72
:1055500000000000B0B52DED028B9FED1A8AD0ED52
:10556000021AD0EDED0A90EDF90A044600F11C058F
:105570009430B0EE481AFFF779FE84EDFF0AD4EDBF
:10558000021AD4EDEE0A94EDF70A04F58670B0EE37
:10559000481AFFF76BFE94EDF81A04F58060D4ED1D
:1055A000021AD4EDEC0A80ED000A2846B0EE410A5A
:1055B000B0EE481AFFF75AFE002084EDFE0ABDEC5B
:1055C000028BB0BD0000000000286FD02DE9F04331
:1055D00081B02DED028B82B0DDE90C981D46164698
:1055E00004460F46FCF75CF906F0F5FE9FED318AA4
:1055F00000EE100A80EE080A10EE100A06F074FFA2
:10560000C4E90001FCF74CF9D4E90423801A99415C
:1056100006F0E1FE00EE100A80EE080A84ED020AB0
:10562000FCF73EF9C4E90401204600F079FA20466F
:10563000394632462B46CDF80090CDF8048000F074
:1056400031FA40F2FC15C2F2000528784CF6CD4143
:105650000130CCF6CC41A0FB0112D10801EB810155
:10566000A0EB4100287040B994ED020AB2EE041A92
:1056700020EE010A204600F0EFF92878800702D1D9
:105680002046FFF73FFF2046FFF764FF204600F06B
:105690004BF904F57D7000F0BFF9002002B0BDECBD
:1056A000028B01B0BDE8F04340B27047FF2040B22A
:1056B000704700BF00247449002900F0EA802DE9FA
:1056C000F0472DED048B0446816100F55770B0EE74
:1056D000408A0D46FFF744F904F56070FFF740F982
:1056E000B3EE0E9AB5F80090B5F80280AF88B5F821
:1056F00006A004F5FE70B0EE480AF0EE490AFFF786
:10570000DFF904F50770B0EE480AF0EE490AFFF73A
:10571000D7F904F50F70B0EE480AF0EE490AFFF72A
:10572000CFF99FED5D9A04F51770B0EE480AF0EEE0
:10573000490AFFF7C5F904F51F70B0EE480AF0EE0C
:10574000490AFFF7BDF904F52770B0EE480AF0EEFC
:10575000490AFFF7B5F9B3EE049A04F52F70B0EEDD
:10576000480AF0EE490AFFF7ABF904F53770B0EEDE
:10577000480AF0EE490AFFF7A3F904F53F70B0EECE
:10578000480AF0EE490AFFF79BF904F54770F2EE7C
:10579000040AB0EE480AFFF793F904F54F70F2EEF1
:1057A0000E0AB0EE480AFFF78BF900EE107AB8EE59
:1057B000408A04F5A47005F14C020121B0EE480ABC
:1057C00004F11C0605F10C07FFF708FE04F1D000F8
:1057D0000121B0EE480A3A46FFF700FE04F15800F6
:1057E00005F12C020121B0EE480AFFF7F7FD00EEAB
:1057F00010AAB8EE408A04F5867005F1AC020121CA
:10580000B0EE480AFFF7EAFD04F1940005F16C02DE
:105810000121B0EE480AFFF7E1FD05F18C023046A8
:105820000121B0EE480AFFF7D9FD00EE109A04F509
:10583000C270B8EE400A05F1CC020121FFF7CEFD9F
:1058400000EE108A04F5E070B8EE400A05F1EC02B3
:105850000121FFF7C3FD04F56F730BCBD4F8C82308
:10586000C4E9F4030420C4F8F023C4F8D813FBF708
:1058700061FF0120FBF75EFF0220FBF75BFF0320C7
:10588000FBF758FF0020BDEC048BBDE8F04740B2A9
:105890007047FF2040B270470000A04290ED001A10
:1058A000B4EE401AF1EE10FA02DA80ED000A704709
:1058B000B4EE601AF1EE10FAB0EE600AC8BF80EDE7
:1058C000000A704790ED000A91ED001A92ED002A4F
:1058D00030EE011A93ED003A31EE021A31EE031A5E
:1058E000B7EE002AB4EE421AF1EE10FAD8BF7047B4
:1058F00082EE011A20EE010A80ED000A91ED000A05
:1059000021EE000A81ED000A92ED000A21EE000A64
:1059100082ED000A93ED000A21EE000A83ED000AF1
:1059200070470000000000002DE9F04F81B000F545
:10593000806400F57D75064600F57E7100F57F7286
:1059400028462346FFF7BEFF96EDFD0A96EDFE1AA8
:1059500096EDFF2A30EE013A94ED004A30EE410A0E
:1059600030EE421A30EE020A30EE040A84ED030AE9
:105970009FED230B31EE441A33EE425A33EE022AE6
:1059800084ED021A5AEC109B9FED1F0B9FED201B1C
:1059900035EE045A32EE442A009684ED015A84ED25
:1059A000042A05F120044FF004085BEC107B56EC50
:1059B000115B00BF0098806990ED460AD0ED470A60
:1059C000A4F11000FFF76AFF54F8100C06F0D8FCA1
:1059D0004A46534606F0DAF93A465B4606F0D6F9EF
:1059E0002A46334605F0BCFE05F088FE2060B8F17B
:1059F000010804F10404DDD1002001B0BDE8F08FFE
:105A00009A9999999999E93FE17A14AE47E1CA3F89
:105A10009A9999999999D13FD0B110B590ED080A0A
:105A200004460420FBF73EFE94ED090A0120FBF733
:105A300039FE94ED0A0A0220FBF734FE94ED0B0ABE
:105A40000320FBF72FFE0020BDE8104040B2704756
:105A5000FF2040B27047000010B5F0EE401AD0EDC4
:105A6000F30A90EDFA0A9FED0E1A044600F5E07075
:105A7000FFF7FCFB04F57B7084EDFB0ABFEE000A28
:105A8000F7EE000AFFF70AFFA06994EDFB1A90ED0C
:105A9000020A002030EE010A84EDFD0A10BD00BFAD
:105AA0000000000070B50446A1699DED040A94ED64
:105AB000F12A9DED051A94EDF03AD1ED430A32EE4C
:105AC000000AC0F8E82300F5777033EE011A84ED80
:105AD000F50AB1EE600AC4F8DC3304F5757604F516
:105AE000767584EDF61AFFF7D9FEA06994EDF51AE4
:105AF00090ED442A304631EE420A71EE020AFFF779
:105B0000CDFEA06994EDF61A90ED452A284631EEB7
:105B1000420A71EE020AFFF7C1FE002070BD0000CC
:105B2000B0B590EDEA0AD0EDEB0A044600F55775E2
:105B300004F0C6FA94ED021AD4EDEC0A2846FEF7FA
:105B400027FF84EDF10A94EDE90AD4EDEB0AB1EEFA
:105B5000400A04F5607504F0B3FA94ED021AD4ED2E
:105B6000ED0A2846FEF714FF84EDF00A94EDEB0AE7
:105B700004F5727004F57371FEF782FC0020B0BD6D
:105B800080B586B00020CDE90400CDE902000120F7
:105B9000019041F20040C4F2020001A9FCF70AFCA6
:105BA00006B080BD80B586B000200590CDE9030029
:105BB0000120CDE9010041F20040C4F2020001A938
:105BC000FCF7F8FB06B080BD80B5806B01684A68C1
:105BD00022F003024A60416D41F01001416501214C
:105BE00080F85110FDF750F980BD000080B5806B42
:105BF000FDF790FB80BD000080B5806BFDF766FE71
:105C000080BD000080B5806BFDF784FE80BD000084
:105C1000B0B5846B0546FCF7A7FC29680968C9057F
:105C200026D402462068A168436823F0200343601D
:105C300031B96168B1F5827F02D16FF0030101E0F3
:105C40006FF001014368194041602046642100F073
:105C500079F800281CBF202060650020E087012023
:105C600084F85100606D18B12046FDF70DF9B0BD04
:105C70002046FDF73DFBB0BDB0B582B0846B054654
:105C8000FCF772FC29680968C90528D40246206817
:105C9000416821F020014160416821F0020141602A
:105CA0002046642100F096F818B1606D40F02000A5
:105CB0006065A06838B9002001902068C168019132
:105CC0008068019001980020E086012084F851004E
:105CD000606D20B12046FDF7D7F802B0B0BD204678
:105CE000FDF7E4FD02B0B0BDB0B5846B0546FCF72E
:105CF0003BFC29680968C9051FD402462068416831
:105D000021F0200141602046642100F063F818B1C1
:105D1000606D40F0200060652068416821F003015B
:105D200041600020E086E087012084F85100606D2A
:105D300018B12046FDF7A8F8B0BD2046FDF7D8FD04
:105D4000B0BD0000B0B582B0044640680B46B0F567
:105D5000827F20D1A168B1F5004F02D0B1F5806FEC
:105D600004D121680D6825F040050D60B0F5827FF3
:105D700011D1A068B0F5806F1DD10092204601219D
:105D80000022002500F076F890B1606D032540F008
:105D9000200060650CE000922046012100220025D1
:105DA00000F068F820B1606D032540F020006065C8
:105DB000284602B0B0BD0092204680210022002576
:105DC00000F058F80028F3D0606D032540F0200063
:105DD0006065EDE770B582B00D46164602210122DE
:105DE0002B460446009600F045F838B1606D032557
:105DF00040F020006065284602B070BD40F200000F
:105E0000C2F20000006849F68171C1F25E61A0FB38
:105E10000101480D4FF47A71484301906068B0F574
:105E2000827F0FD12046802100222B46009600253C
:105E300000F020F80028DED0606D032540F020003F
:105E40006065D8E7019840B1019801380190206859
:105E500080680006F6D40025CDE70025CBE70000DA
:105E6000006843F20001C4F20101401A18BF01208A
:105E7000400070472DE9F04782B00A9C98461546CD
:105E80000E468146FCF770FB201A00EB0804FCF775
:105E90006BFB40F20001C2F200010968C1F3CB3193
:105EA00061430191D9F8001089683140891BB1FA2A
:105EB00081F14909A94203D1002002B0BDE8F08771
:105EC000824608F101070CE0019801380190D9F8E9
:105ED000000080683040801BB0FA80F04009A84282
:105EE000EAD0002FF3D0FCF73FFBA0EB0A00A04262
:105EF00004D201980028E7D10024E8E7D9E900019D
:105F00004268B1F5827F22F0E00242600BD1D9F8FD
:105F10000810B1F5004F02D0B1F5806F03D10168D0
:105F200021F040010160D9F82810B1F5005F07D1D8
:105F3000016821F400510160016841F400510160E1
:105F4000012089F85100002089F85000032002B098
:105F5000BDE8F0870000000080B500EE100AB8EE42
:105F6000C00A10EE100A06F00BFA9FED110B53EC6D
:105F7000102B05F0B1FC41EC100B9FED0F1B04F052
:105F8000F7F953EC102B9FED0E0B51EC100B06F0B4
:105F900009F99FED0D0B53EC102B05F0F7FE9FED6B
:105FA0000C0B53EC102B05F0F1FE05F02BFE80BD21
:105FB00000000000D0BCF8406C45D9CC955BC83FD0
:105FC000000000000000F03F0000000040A5E54098
:105FD0000000000000408F4080B50C20892102F0B5
:105FE000A3F900281CBF012080BD6420FBF71CFC26
:105FF00002F044F940B2B0F1FF3FF9DC02F0BAF828
:1060000002F03CF94006FBD50D2002F069F941F29F
:10601000902100F0F002C2F20001102A08701CBFAB
:10602000022080BD7020032102F046F87020032179
:1060300002F070F8072002F071F9002080BD000026
:106040002DE9F04F81B02DED048B8846824602F099
:1060500031F941F29024C2F2000494ED041A00EEEA
:10606000100AB8EEC00AB8EEC11A80EE018A02F03A
:106070000BF994ED031A41F2A424C2F2000400EEDD
:10608000100AB4F90000B8EEC00AB8EEC11AB4F9AB
:106090000250B4F90C90B4F90EB080EE019A05F0FC
:1060A0000EFE9FED310B53EC102B05F06FFE00EE52
:1060B000105AB8EEC00A28EE000A064610EE100A82
:1060C0000F4606F05DF902460B463046394605F0AC
:1060D00047FB05F097FDCAF80000B4F9100094EDF5
:1060E000021A02EE100AB4F91400B8EEC22A03EE46
:1060F000100AB8EEC33A29EE033A33EE022A94EDC1
:10610000010AB8EEC11A29EE022AB4F9120032EEE1
:10611000011A04EE100AB8EEC00A29EE011A03EEC5
:1061200010BAB8EEC44A31EE000A01EE109AB8EE89
:10613000C33A29EE044AB8EEC11A28EE092A34EE11
:10614000033A28EE011A22EE032A31EE000A32EE5B
:10615000000ABDEEC00A002088ED000ABDEC048BE9
:1061600001B0BDE8F08F00BF000000000000E03F7C
:10617000074B19680868B0E8F04F80F30988BFF34F
:106180006F8F4FF0000080F31188704700BF00BF91
:106190008409002080B500F0E9FE80BD80B501F0E3
:1061A000A3F901F0FFF980BDB0B501380024B4EBCC
:1061B000106F1CBF0120B0BD4EF21005CEF20005DD
:1061C00068604FF0FF300F2100F0BEFE0720AC608A
:1061D00028602046B0BD000080B5FCF711FB03F03D
:1061E000A1F9012818BF02F0B5FC80BD70B592B0CE
:1061F00006AC20463021FAF74EF9002543F6400060
:106200000595CDE90355CDE901550095C4F202008D
:106210000168022641F080510160006800F0805062
:106220000090009847F200000095C4F20000016859
:1062300041F480410160006800F4804000900098C3
:10624000012006904FF4803007904FF480000D90AD
:1062500006200E90A820CDE90F06042011902046BC
:106260000C96FCF76DFC88B90F20CDE901064FF4C0
:10627000A05004904FF48050059001A8052103958B
:10628000FCF750FB002804BF12B070BDFBF7A4FE62
:106290004EF68850CEF20000016841F470010160B2
:1062A00070470000B0B540F6FF3E0568C4F2000E2E
:1062B00040F2004C7045C4F2010C0FDCB0F1804F8D
:1062C00019D040F20043C4F20003984213D040F6C4
:1062D0000003C4F2000398420DD011E040F60043E1
:1062E000C4F20003984206D0604504D00023C4F2F3
:1062F0000103984204D14B6825F0700243EA02057D
:1063000041F6FF73C4F2000398420DDC70451FDCB8
:10631000B0F1804F41D040F20043C4F200039842F4
:106320003BD040F6000321E043F6FF73C4F20103C3
:10633000984220DC42F20003C4F2000398422CD0C1
:106340000023C4F20103984227D0604525D029E0FC
:1063500040F60043C4F2000398421ED041F6000309
:10636000C4F20003984218D041F60043C4F200037F
:10637000984212D016E044F20003C4F2010398429E
:106380000BD044F60003C4F20103984205D044F256
:106390000043C4F20103984204D1CB6825F4407253
:1063A00043EA02050A688C684B69C46240F4806461
:1063B0008262644504BF09690163026825F08001B7
:1063C00042F0040219430260012242610160B0BD43
:1063D00080B501F01F014FF0010CD0F820E00CFA5D
:1063E00001F32EEA03030362036A02FA01F119437F
:1063F000016280BDB0B5026A036A40F2004523F035
:1064000001030362D0F804E0D0F818C08C6822F0D1
:10641000020240F48063C4F20105AB4242EA040286
:1064200005D1CC6822F00C0224F0040422430C684D
:10643000AB4207D1D1E905532EF4407E45EA0E0563
:1064400045EA030E2CF073032343C0F804E0836194
:10645000496841630262B0BD70B5026A036A40F2E6
:10646000004423F010030362D0F804E0D0F818C011
:106470008D6822F0200240F48063C4F20104A3423C
:1064800042EA051207D1CD686FF0400622F0C00243
:1064900006EA05152A430D68A34207D1D1E9056430
:1064A0002EF4406343EA860343EA840E2CF4E64369
:1064B00043EA0523C0F804E083614968816302620E
:1064C00070BD000070B5026A036A40F2004423F414
:1064D00080730362D0F804E0D0F81CC08D6822F409
:1064E000007240F48063C4F20104A34242EA052230
:1064F00007D1CD6840F2FF462D0222F44062B54339
:106500002A430D68A34207D1D1E905642EF4405314
:1065100043EA061343EA041E2CF073032B43C0F82E
:1065200004E0C3614968C163026270BD70B5D0F810
:1065300020C0026A40F2004622F4805202624268A1
:10654000C3690C68D1F808E040F48065C4F2010624
:10655000B54204D14D6922F4804242EA851223F407
:10656000E64343EA04234260C3612CF400564968C1
:1065700046EA0E320164026270BD000010B500F000
:10658000E7FD46F251604CF69802C0F60000C0F6F6
:106590000002002100F0ACFF41F2BC24C2F2000472
:1065A000206046F2C1704CF6BC02C0F60000C0F696
:1065B0000002002100F09CFF606046F6F9004CF6F6
:1065C0000412C0F60000C0F60002002100F090FFA7
:1065D000A06046F699104CF64C12C0F60000C0F6CA
:1065E0000002002100F084FFE06046F649004CF60E
:1065F000E002C0F60000C0F60002002100F078FFC3
:10660000206105200421002200F038FEA061032053
:106610000C21002200F032FEE06103200421002260
:1066200000F02CFE206203200421002200F026FE50
:10663000606203201421002200F020FEA06200F01E
:10664000B7FD00F051FF00F0ADFF10BD00000000ED
:1066500082B000F065FD05F049FB9FED550B53EC52
:10666000102B05F039F905F0FDFA0646002000F080
:106670000FFD00F04BFD40F2E825C2F2000540F2AC
:1066800008010446C2F200012846FAF7BBFD28467D
:10669000FAF792FD40F2803040F68001C2F200002D
:1066A000C2F20001F9F7D8FF2846FAF785FDB7EEE8
:1066B000001A81EE000A40F638004CF69412C2F23D
:1066C0000000C0F600020021FEF788FE0520FBF75F
:1066D00031F8A71940F2743840F2942940F2683A30
:1066E0009FED358A9FED359A41F2BC2B40F2803404
:1066F000019605F1100005F11C06C2F20008C2F275
:106700000009C2F2000AC2F2000BC2F200040090BB
:10671000FAF7C6FEFAF73CFDFAF746FDFAF75CFD1C
:10672000FAF768FD00F014FD2846FAF70DFE28463A
:10673000FAF754FE009940F6800320463246C2F232
:106740000003FAF74BF840462146F9F717FF00F02F
:106750002FFDA8690023C9F8000098E80700CAF8CF
:106760000820CAE90001DBF818004946002200F0C1
:10677000D5FDDBF81C0051460022002300F0CEFDC1
:10678000D5ED0A0A40F63800C2F20000B0EE480A21
:10679000B0EE491AF0EE491AFEF768FD0520FAF747
:1067A00081FF384600F084FC01980744B0E700BF41
:1067B0000000000000408F40000020420000000068
:1067C00000F0AEFC05F092FA9FED1B0B53EC102B82
:1067D00005F082F805F046FA0446002000F058FC67
:1067E00000F094FC05460820FAF7BAFF0620FAF7F5
:1067F000B7FF9FED130A0720FAF754FF0720FAF7B7
:1068000099FF9FED108A2544B7EE009AB6EE00AAD4
:1068100000EE105AB8EE400A20EE080A04F0D8FB49
:1068200030EE090A20EE0A0A0720FAF73BFF284655
:1068300000F03EFC2544EBE700000000000059405A
:1068400000000000A69B443B00F06AFC05F04EFAF5
:106850009FED270B53EC102B05F03EF805F002FAE4
:106860000446002000F014FC00F050FC40F2BC286C
:10687000C2F2000805464046FBF784F940F22D3984
:10688000C2F200094846FBF7E9FA2F1941F25425F4
:1068900040F2483641F2BC2AC2F20005C2F20006BC
:1068A000C2F2000A13E000BF28882B1D30800FCBF6
:1068B000F260C6E90110DAF828003361314600229F
:1068C000002300F02BFD384600F0F2FB27440A209D
:1068D000FBF7D2FA0028E7D048464146FBF776F9A5
:1068E00040462946FBF74EF84846FBF7B7FADBE788
:1068F0000000000000407F4000F012FC05F0F6F9B7
:106900009FED210B53EC102B04F0E6FF05F0AAF9E4
:1069100080464FF4967000F0BBFB00F0F7FB9FED54
:106920001C0A0446FDF702FE04EB080541F2BC26F2
:1069300040F26C2940F2603740F26434C2F2000643
:10694000C2F20009C2F20007C2F20004B06949466F
:106950000022002300F04EFC99ED000A3846214643
:10696000FDF78EFD306A39460022002300F0D6FC88
:10697000706A21460022002300F0D0FC284600F077
:1069800097FB4544E2E700BF0000000000407F4065
:106990000000FA430000000082B000F0C1FB05F0E7
:1069A000A5F99FED2B0B53EC102B04F095FF05F090
:1069B00059F98146002000F06BFB00F0A7FB04466C
:1069C000FBF7DAF840F60067C2F200079FED220AF3
:1069D00001463846FEF770FE41F2BC2507F56F7A96
:1069E00007F5727B07F5737841F2282704EB090657
:1069F000C2F20005C2F20007E869514600220023F6
:106A000000F0F8FB286A59460022002300F0F2FB50
:106A1000686A41460022002300F0ECFBA86A394670
:106A20000022002300F0E6FBD7E9030497E80E00FC
:106A3000009040F60060C2F200000194FEF7C4FD31
:106A4000304600F035FB4E44D6E700BF00BF00BF24
:106A50000000000000408F4000007A4480B5806B49
:106A60000021C185FDF770FA80BD000010B5846B70
:106A70002068406994F84110212907D110F0800066
:106A800004D00020E084204600F09CF82068406993
:106A900094F84210222907D110F0400004D00020C1
:106AA000E085204600F05AF8606C40F01000606409
:106AB0002046FDF749FA10BD80B50168806B096872
:106AC000C9052FD40021C185016851E8031F026860
:106AD00021F4807142E80313002BF5D1016851E8DD
:106AE000051F026821F0010142E80513002BF5D1D2
:106AF000016851E8051F026821F0400142E80513D2
:106B0000002BF5D1202180F84210016B012909D119
:106B1000016851E8031F026821F0100142E80313E5
:106B2000002BF5D100214163016B012903D1818D37
:106B3000FDF708FA80BDFDF765FC80BD80B5806B70
:106B400001214163016B012904D1818D4908FDF7C1
:106B5000F9F980BDFDF76AFC80BD0000016851E8CD
:106B6000031F026821F4907142E80313002BF5D152
:106B7000016851E8051F026821F0010142E8051390
:106B8000002BF5D1016B01290AD100BF016851E842
:106B9000031F026821F0100142E80313002BF5D116
:106BA000202180F8421000210163704780B5016800
:106BB000CA6822F04002CA60202180F84110FDF727
:106BC00049FC80BD016851E8031F026821F0C00143
:106BD00042E80313002BF5D1202180F841107047C3
:106BE00044F600010068C4F2000101F54C420323A1
:106BF000904208BF0123401A18BF18467047000092
:106C000080B582B090F8421022291ED18268B2F578
:106C1000805F02D1016900294AD0816AB2F5805FA4
:106C200007D00AB9026922B10268526802F07F02F5
:106C300001E0026852680A700121826A114481628F
:106C4000C18D01390A04C18501D002B080BD01683F
:106C5000CA6822F02002CA60CA6822F48072CA6040
:106C60004A6922F001024A61202180F84210002185
:106C70004163026B012A23D1016300BF016851E81F
:106C8000031F026821F0100142E80313002BF5D125
:106C900001680A68D20606D5002201920A680192AC
:106CA000496801910199818DFDF74CF902B080BDD1
:106CB0000168826A49686FF35F2111800221BCE795
:106CC000FDF7A0FB02B080BD10B504460068D4E912
:106CD00002C22369016921F44051114301616269D3
:106CE00043EA0C01E3691143C268194349F20C639A
:106CF0009A431143C1604169A26921F4407141F294
:106D00000043114340F48062C4F201039A4241619E
:106D100002D1FBF7CFFE01E0FBF7BAFEE169636841
:106D20001922B1F5004FA0FB02011CD15A00DB0F64
:106D3000F9F7BAFA48F21F51C5F2EB11A0FB012393
:106D40005A096FF0630302FB0300322303EBC00018
:106D5000A0FB01014FF4F87000EA111000EB0210E3
:106D6000C1F342111AE09A009B0FF9F79DFA48F21D
:106D70001F51C5F2EB11A0FB01235A096FF0630309
:106D800002FB0300322303EB0010A0FB0101F02003
:106D900000EA511000EB0210C1F3431122680843CE
:106DA000906010BDF0B581B01346002704468162A3
:106DB00083854764222084F84200E06B46F6B925BB
:106DC00046F63D360A462168C0F60005C0F60006C4
:106DD000C0E90F5646F66D26C0F600060431C0E93C
:106DE0001367FBF77DFA38B110206064202084F827
:106DF0004200012001B0F0BD0097206801680091B9
:106E0000406800900098206950B100BF206850E8A9
:106E1000030F216840F4807041E80302002AF5D195
:106E2000206850E8050F216840F0010041E80502A4
:106E3000002AF5D1206850E8050F216840F0400095
:106E400041E80502002AF5D1002001B0F0BD0000A4
:106E500090F84110212923D18168B1F5805F01D1DB
:106E6000016931B1016A02684B1C03620978516003
:106E700007E0016A036831F8022B6FF35F225A6062
:106E80000162C18C01390A04C18418BF70470068CF
:106E9000C16821F08001C160C16841F04001C1605A
:106EA0007047000010B540F2F074C2F200042046B2
:106EB000FDF75EF82046FAF72BFD10BDFEE7000057
:106EC00000F0FF40B0F1FF4018BF01207047000004
:106ED00000F0FF40B0F1FF4018BF012070470000F4
:106EE00020F00040A0F1FF40B0FA80F04009704768
:106EF000002848BF704700F01F01012202FA01F18B
:106F00004EF280124009CEF2000242F82010BFF388
:106F10004F8FBFF36F8F7047002848BF704700F056
:106F20001F01012202FA01F14EF200124009CEF2D5
:106F3000000242F8201070474EF60C50CEF20000CE
:106F40000068C0F3022070474EF6145300F00F02A1
:106F5000CEF2000309011A4400F16043B0F1FF3F93
:106F6000C8BF03F564421170704700004EF61F5011
:106F7000CEF2000000210170704700004EF60C5167
:106F8000CEF200010A684FF6FF031A4060F30A22AE
:106F900042F0806040F0FD700860704740F6DB71A1
:106FA00010EE100AC3F6C97161F31E0000EE100A5C
:106FB00070470000F0B581B0F0B1044640F684108F
:106FC000C2F200000068A0421FD001F045FA40F66E
:106FD0008C10C2F200006569076840F69410C2F296
:106FE0000000066801F05CFABD424FF0020018BFD5
:106FF000B5420DD101B0F0BD4FF0500080F31188C3
:10700000BFF36F8FBFF34F8FFEE7002001B0F0BDDD
:1070100047F69040C2F2000085420CD047F6A441EA
:107020000120C2F20001002D08BF04208D4208BFDC
:10703000042001B0F0BDA06A10B1022001B0F0BD83
:1070400094F858100320012908BF022001B0F0BDB8
:10705000FBF7E4FBFFF7CAF8FDF71EFEFDF7B0FDF6
:10706000FDF7EAFEFDF774FFFEF700F8FEF748F8BB
:10707000FDF72AFFFDF700FFFEF7C2F8FEF7A2F8C2
:1070800000F052F8FDF7EAFD00F078F8FEE70000A6
:10709000EFF3058100291CBF6FF005007047002841
:1070A00004BF0020704780B501F0DAFA002080BDEF
:1070B00010B582B0EFF3058119B16FF0050002B091
:1070C00010BD044602F042FA211A0129019005DBA5
:1070D00001A801F0EFFA002002B010BD6FF003002C
:1070E00002B010BD80B502F01DFA022808BF80BDB5
:1070F00008B9032080BD40F2F810C2F20000006819
:107100000138B0FA80F0400980BD000080B5EFF38F
:10711000058010B102F020FA80BD02F017FA80BDA0
:107120004FF47A7070470000EFF3058000281CBF11
:107130006FF00500704740F2F810C2F200000168DD
:10714000002911BF4FF0FF3001210160002070477E
:1071500080B5EFF3058000281CBF6FF0050080BDEF
:1071600002F0E0F928B1022805D101F0FBFB002074
:1071700080BD012080BD4FF0FF3080BD10B5EFF322
:10718000058000281CBF6FF0050010BD40F2F81408
:10719000C2F20004206801281CBF4FF0FF3010BD70
:1071A000FEF7F8FF0220206001F08AFB002010BDEE
:1071B00010B5EFF3058018B16FF00504204610BD3F
:1071C00002F0B0F902280ED080B902F053FB01287A
:1071D0004FF001040CD002F0A5F9002808BF4FF0D1
:1071E000FF34204610BD0024204610BD4FF0FF3470
:1071F000204610BD10B582B01C46B0FA80F3B1FA3B
:1072000081F25B095209EFF3058CBCF1000F42EAF1
:10721000030219D0002C18BF0124224315D10022EB
:10722000019201AA01F05AFF01281AD10198A8B1D0
:107230004EF60450CEF200004FF080510160BFF3D3
:107240004F8FBFF36F8F09E01AB16FF0030002B0E8
:1072500010BD224601F080FE012806D1002002B0B8
:1072600010BD6FF0020002B010BD6FF00100002CE5
:1072700008BF6FF0020002B010BD0000B0B582B0D0
:10728000144600294FF00005EFF3058218BF0028CF
:1072900002D1284602B0B0BD002AFAD19CB1A5683F
:1072A000D5B1E268502A16D32269A2B1D4F814C02D
:1072B00001FB00F2002394454FF0000228BF012299
:1072C00010D24DB10EE0012300226AB9E3B10022D1
:1072D00001F058FC0EE01DB9E2680AB92269C2B19A
:1072E00000220023002AF1D0A3682269002500951E
:1072F00001F06CFC054655B1002C14BF216800213B
:10730000284601F077F9C4E70025002DF4D10025C7
:10731000BFE76269B2FA82F25309D5E7B0B582B02D
:107320001C46B0FA80F3B1FA81F5EFF305825B09F0
:107330006D09002A43EA050207D0002C18BF01247A
:10734000224306D06FF003052CE0CAB16FF00305AD
:1073500028E00022019201AA002301F095FD0128F6
:107360001CD10198E8B14EF60450CEF200004FF067
:1073700080510160BFF34F8FBFF36F8F002511E085
:1073800022460023002501F0ADFC01280AD06FF051
:107390000105002C08BF6FF0020503E06FF0020545
:1073A00000E00025284602B0B0BD0000B0B584B0B2
:1073B00048B3B1F1FF3F26DD04464FF0FF300390A4
:1073C000EFF3058018B300250DF1080C20460122CB
:1073D00000230295CDF800C002F008F803AB204668
:1073E00000210022009502F001F80298D0B14EF67B
:1073F0000450CEF200004FF080510160BFF34F8F78
:10740000BFF36F8F0EE06FF0030003900AE0204699
:107410000122002301F06CFF03AB20460021002273
:1074200001F066FF039804B0B0BD00002DE9F04FF5
:1074300083B00C46EFF3058129B16FF0050738469C
:1074400003B0BDE8F08F0546002849D44FF0000B8B
:107450009246A00758BFAB4602F078F800906FF054
:10746000010804F0010054460027BAF1000F08BFDC
:107470006FF00208019002E04746002EDFD00020A6
:10748000594602AA234602F01BF906460128F3D109
:10749000029807EA050140EA01090198002809EA73
:1074A000050007D100286FF0020718BF4F4607D02C
:1074B000C5E700BFA8426FF0020708BF4F46BED025
:1074C000BAF1000FBBD002F041F800994F46401AC4
:1074D000241A4FF0000038BF0446002ECFD1AEE78B
:1074E0006FF00307ABE7000080B502F015F880BD30
:1074F00070B584B08E46002100280391EFF305811A
:1075000046D0002944D1FAB19369002B08BF182353
:10751000382B16D81179C90713D1556994681168A9
:107520004FEA950C002D08BF4FF0800CFCB1D668D7
:107530005C2E1BD3D5B11569C5B10024012555B901
:107540001BE0002004B070BD0124002118234FF07F
:10755000800C00258DB1946812690294CDE9003247
:107560006246734601F088FE039011E00CB9D468BE
:107570009CB100250024002DEDD14CB103AC00934B
:107580001FFA8CF27346019401F042FE012802D1E9
:10759000039804B070BD0020E6E71469B4FA84F4DF
:1075A0006409D6E710B5EFF3058100291CBF6FF021
:1075B000050010BD044660B12046FFF7FBFC04281F
:1075C00004BF6FF0020010BD204601F0C7F8002094
:1075D00010BD6FF0030010BDF0B581B00D4647F649
:1075E000B84140F68416C2F20001C2F200060F68EC
:1075F00031680446081D00F0B9FE601C0AD14DB187
:107600003068011D47F69040C2F2000000F00CFF08
:1076100001B0F0BD3068E41944600AD340F694101C
:10762000C2F2000000683168043100F0DFFE01B0F2
:10763000F0BD40F68C10C2F20000006831680431E1
:1076400000F0D4FE47F61C40C2F2000001688C42F4
:1076500038BF046001B0F0BD70B5044600F0FCFE18
:1076600047F2F040C2F20000016840F68415013193
:107670000160C2F20005296847F68446C2F200069E
:1076800041B1306860B92868E16AC06A884298BF31
:107690002C6005E02C600068012801D100F0C2F9DF
:1076A00047F2FC40C2F200000168013101606164F0
:1076B00047F20051C2F20001E06A0A68904288BFB6
:1076C000086040F69C1100EB8000C2F2000101EB63
:1076D0008000211D00F0A8FE00F0E2FE306880B1BD
:1076E0002868E16AC06A884228BF70BD4EF604501F
:1076F000CEF200004FF080510160BFF34F8FBFF317
:107700006F8F70BD70B582B000F0A6FE47F6BC4624
:10771000C2F20006306850BB47F6BC34C2F2000427
:10772000204600F053FE47F6D035C2F20005284649
:1077300000F04CFE40F68810C2F20000046040F6F3
:107740009810C2F2000040F6900240F63013056037
:107750000025C2F20002C2F200030A2010210095A7
:1077600001F034FA306010B103A100F043FF00F0E3
:1077700097FE02B070BD00BF546D72510000000052
:10778000F0B581B047F2F445C2F200052868E0B1D7
:1077900047F6A44647F2F047C2F20006C2F20007DD
:1077A00000F05AFEF068C468201D00F0DFFD386864
:1077B0000138386028680138286000F071FE2046E2
:1077C00000F058F828680028EAD101B0F0BD0000A8
:1077D00080B5026C002A08BF80BDD0E902C3134403
:1077E000C360634524BF0368C360C3680846194685
:1077F000F8F7D2FD80BD000070B5866B036C0446BF
:10780000E3B115461AB3E0681A46F8F7C5FDE1681A
:10781000206C2268091A9142E16003D2A1684042BB
:107820000844E060A81EB0FA80F040093146002EFE
:1078300018BF01210840361A002516E020680025EF
:1078400098B9A06801F084FFA56005460DE0606866
:107850001A46F8F7A1FD216CD4E90102002508447D
:107860006060904224BF20686060711C2846A1635C
:1078700070BD000010B5044690F85900022808BFFA
:1078800010BD012803D030B9206B00F021FE204646
:1078900000F01EFE10BD4FF0500080F31188BFF3C2
:1078A0006F8FBFF34F8F00BFFEE7000040F68811D7
:1078B000C2F2000109680A68B2FA82F35B09036048
:1078C000002A0EBF0020C8680068704741F23C30B3
:1078D000C2F20000C21D22F0070210F0070CA0EB5C
:1078E000020318BF104647F68842C2F20002002188
:1078F000C2E9000146F2A812BCF1000F18BF1A44F9
:107900000244083A40F6901322F00702C2F2000344
:107910001A60C2E90011111A1A68C0E9002147F67D
:107920001840C2F20000016047F61040C2F20000A9
:10793000016047F6E430C2F2000001210170704797
:1079400040F69C144EF60455C2F20004CEF2000537
:107950004FF08056FFF714FF20680228FAD32E60FC
:10796000BFF34F8FBFF36F8FF4E70000B0B5049DF6
:10797000002914BF2A602D60C5E90F0128460121A6
:107980001C4601F06FF985F84C40B0BD2DE9F04779
:107990000A9C8246206B16460F46DDE90859910085
:1079A000A5229846F8F76FFD206B00EB8600A0F14A
:1079B000040020F007067FB104F13400002100BF6D
:1079C0007A5C42547A5C1AB10F2901F10101F7D3B4
:1079D000002084F8430002E0002084F834000027EF
:1079E000201D372D28BF3725E562C4E9135700F065
:1079F000F9FC04F1180000F0F5FCC5F13800A061B5
:107A000030465146424624616462676584F8587086
:107A100000F03EFBB9F1000F206018BFC9F800402C
:107A2000BDE8F087B0B540F69C150024C2F2000511
:107A3000281900F0CBFC1434B4F58C6FF8D147F65C
:107A4000E834C2F20004204600F0C0FC47F6FC35E2
:107A5000C2F20005284600F0B9FC47F63040C2F2F9
:107A6000000000F0B3FC47F6A440C2F2000000F0B2
:107A7000ADFC47F69040C2F2000000F0A7FC40F6D3
:107A80008C10C2F20000046040F69410C2F20000B4
:107A90000560B0BD80B547F68842C2F2000200BF63
:107AA000114612688242FBD3D1F804C001EB0C03EB
:107AB000834203D14068604448600846D0F804C05F
:107AC00000EB0C03934201D013460BE040F69013F9
:107AD000C2F200031B689A4204D0D2E9003E0EEBCA
:107AE0000C0242608142036018BF086080BD000044
:107AF00080B58C46014641F804CF9445006108D911
:107B00009A4201D29C4511D240F68810C2F2000080
:107B100007E08069D21A824208D240F69810C2F279
:107B20000000006800F062FC002080BD012080BDE4
:107B300010B5044600F090FCA06BB0FA80F0440948
:107B400000F0AEFC204610BD10B5044600F084FCE9
:107B5000A06BE16B401AB0FA80F0440900F0A0FC81
:107B6000204610BD08480068006880F308884FF080
:107B7000000080F3148862B661B6BFF34F8FBFF385
:107B80006F8F00DF00BF00BF08ED00E070B582B06E
:107B900040F68812C2F2000212680546D2680E460C
:107BA000D468201D00F0E2FB94F82800410704D4BB
:107BB00000F0FE0084F8280010E0A0693246411968
:107BC00020462B46FFF794FF40B1002620460021B7
:107BD0002A460023009601F011FF20B1216A2046B9
:107BE000884702B070BD4FF0500080F31188BFF39A
:107BF0006F8FBFF34F8F00BFFEE700002DE9F0410C
:107C000086B047F6BC47C2F20007386802A90022D6
:107C10004FF0000801F0A0F900286AD001AC02ADD5
:107C20000BE000F0FE0086F8280000BF3868294607
:107C3000002201F091F900285BD00298B0F1FF3FDB
:107C400003DCDDE903200599904702980028EDD474
:107C5000049E706910B1301D00F088FB204600F0D2
:107C6000B3F802990929E1D80246DFE801F00808D3
:107C700008052A390808052A96F82800D1E796F859
:107C80002800039BB16940F0010086F828001944E0
:107C90003046FFF72DFF0028C8D0316A30468847AC
:107CA00096F828004007C1D50398B16900230A1847
:107CB00030460021CDF8008001F0A0FE0028B5D1AB
:107CC00023E096F8280040F00101039886F8281078
:107CD000B06188B1811830461346FFF709FFA5E768
:107CE00096F8280081073FF59CAF304600F0F0FB86
:107CF0009CE706B0BDE8F0814FF0500080F311889A
:107D0000BFF36F8FBFF34F8FFEE74FF0500080F34C
:107D10001188BFF36F8FBFF34F8F00BFFEE70000E6
:107D200070B582B00E46044600F01CFE01A800F0BB
:107D30004BF8019919B101F09DFD02B070BD0546E7
:107D40004EB9A54207D301F095FD20462946FFF71D
:107D50001DFF02B070BD4EB140F69810C2F2000097
:107D600000680068B0FA80F0420900E0002247F69F
:107D7000BC40C2F200000068611B00F04FFC01F043
:107D800079FD0028D9D14EF60450CEF200004FF014
:107D900080510160BFF34F8FBFF36F8F02B070BD92
:107DA00040F68C10C2F200000168096821B1006839
:107DB000C068C068406801E04FF0FF3047F61C41E2
:107DC000C2F200010860704770B5044601F0BEFBC6
:107DD00040F68016C2F2000631680546884203D29A
:107DE00000F008F8012000E00020206028463560FF
:107DF00070BD00002DE9F04182B040F68817C2F254
:107E000000073868016891B34FF0000809E000BF2F
:107E1000606038682946246100F0E8FA3868016833
:107E200029B3C068C4680668251D284600F09EFA7C
:107E3000216A2046884794F828004007EED5A069BB
:107E40003044B042E4D82046002132460023CDF829
:107E5000008001F0D3FD0028E0D14FF0500080F306
:107E60001188BFF36F8FBFF34F8F00BFFEE740F65F
:107E70009811C2F200010A6808603A6002B0BDE8D9
:107E8000F081000081B00020009040F23C10C2F26E
:107E9000000000684FF0500181F31188BFF36F8F2D
:107EA000BFF34F8F013001D0FEE700BF00980028DC
:107EB000FCD001B07047000082B001AC2046FFF753
:107EC000F5FC0199FFF72CFFFFF798FEF6E700009D
:107ED000F0B581B0044600F0BFFA94F94560012E78
:107EE0000FDB04F1240500BF286850B1284601F0DB
:107EF00079FC002818BF00F0A1FC70B2013E0128F7
:107F0000F2DCFF2684F8456000F0CAFA00F0A4FA1B
:107F100094F94470012F0EDB04F11005286850B16C
:107F2000284601F05FFC002818BF00F087FC78B2FB
:107F3000013F0128F2DC84F8446000F0B1FA01B09E
:107F4000F0BD00002DE9F04381B0044600F00AFDC9
:107F500040F69016C2F200063068002808BFFFF70E
:107F6000B5FC47F6E438C2F2000898F80000002893
:107F700018BF4FF0004020420DD0002401F07AFCE1
:107F800060071ED04FF0500080F31188BFF36F8F51
:107F9000BFF34F8FFEE7C4B114F0070004F10801EE
:107FA0001EBF081A00F108015FEA41700ED04FF0C1
:107FB000500080F31188BFF36F8FBFF34F8F00BF66
:107FC000FEE7204601B0BDE8F083002147F61049E6
:107FD000C2F20009D9F800004A1E8242CDD247F60B
:107FE0008840C2F2000005682F4657F8042F8A42E5
:107FF00011D22B685BB100BF1F4657F8042F2846EB
:108000001D468A4207D22B68002BF5D103E047F6C4
:108010008840C2F2000033689D42AED004682B68ED
:10802000521A112A036010D36818430709D04FF081
:10803000500080F31188BFF36F8FBFF34F8F00BFE5
:10804000FEE742603960FFF725FD47F618403968C2
:10805000D9F80020C2F200000368511A9942C9F809
:10806000001038BF016098F80000396800284FF010
:10807000000018BF41F00041286047F62440C2F2DA
:108080000000026808343960511C016076E7000086
:10809000034647F68560C0F600004FF0807C21F073
:1080A000010103E903106FF0020043F8240CA3F16F
:1080B000440043F8202C7047B0B50C46042905460F
:1080C00007D3092000F00CF940F00401092000F06A
:1080D0002BF9072C08D860B206A151F8200041F214
:1080E0009021C2F20001C86044EA0501062000F0B8
:1080F0001BF9B0BD000008000000180000003800A7
:108100000000780000E0030000E0070000E00F003E
:1081100000E01F00B0B50C460429054607D309202E
:1081200000F0DEF840F00801092000F0FDF8072C0F
:1081300008D860B207A151F8200041F29021C2F2A4
:108140000001086145EA040040F08001072000F0CA
:10815000EBF8B0BD00000800000018000000380077
:108160000000780000E0030000E0070000E00F00DE
:1081700000E01F00F0B581B0102000F0B1F8044617
:10818000112000F0ADF8210141EA101041F2A426BF
:10819000210648BF00F57040C2F200063080112071
:1081A00000F09EF80446122000F09AF804F00F0147
:1081B00040EA0120210748BF00F57040708013207D
:1081C00000F08EF80446142000F08AF805461520C9
:1081D00000F086F8290141EA043141EA1010002735
:1081E000CFF6F077210648BF38437060152000F0C5
:1081F00077F80446162000F073F80546172000F0C3
:108200006FF8290241EA04410844210748BF384376
:10821000B060182000F064F80446192000F060F8FF
:1082200040EA0420B0811A2000F05AF804461B20CE
:1082300000F056F840EA0420F0811C2000F050F8CD
:1082400004461D2000F04CF840EA042030821E2035
:1082500000F046F804461F2000F042F840EA0420EF
:108260007082202000F03CF80446212000F038F80D
:1082700040EA0420B08201B0F0BD000080B50820C3
:1082800000F02EF880BD0000B0B5002000F028F806
:108290000446012000F024F80546022000F020F8F2
:1082A000290241EA04410844210648BF00F17F4009
:1082B000B0BD0000B0B5032000F012F80446042061
:1082C00000F00EF80546052000F00AF8290241EA00
:1082D00004410844210648BF00F17F40B0BD0000C2
:1082E00010B50446FCF7ACFAEE20FCF77BFAFCF77D
:1082F000E7FA2046FCF776FAFCF7E2FAFCF7A0FA78
:10830000EF20FCF76FFAFCF7DBFA0020FCF738FAF5
:108310000446FCF7B7FA204610BD000080B50146C0
:10832000082000F001F880BDB0B50C460546FCF70A
:1083300087FAEE20FCF756FAFCF7C2FA18B1FCF700
:10834000A1FA0120B0BD2846FCF74CFAFCF7B8FAB8
:108350002046FCF747FAFCF7B3FA0446002818BF9A
:108360000124FCF78FFA2046B0BD0000D0E90132AD
:1083700001699A60D1F804C082688445536008BFDF
:108380004A60002202610868013808600868704786
:1083900047F20473C2F20003036047F20450C2F2D2
:1083A00000000860802010607047000047F66033CE
:1083B000C2F20003036047F26070C2F2000008607E
:1083C0004FF4807010607047704700004FF0FF312D
:1083D000024642F8081F00214260C0E90322016002
:1083E00070470000002101617047000080B5D1F89E
:1083F00000C01CF1010207D000F108039E465B6833
:108400001A686245FAD901E0D0F810E0DEF80420DD
:1084100008614A609160C1F808E0CEF80410016874
:108420000131016080BD0000D0F800C043680861E0
:108430009A684B608A609A68996051600CF10101FA
:1084400001607047DFF80C00016841F470010160C1
:10845000704700BF88ED00E04FF0500080F31188B6
:10846000BFF36F8FBFF34F8F40F23C10C2F200009A
:1084700001684A1C026001B170474EF60450CEF20A
:1084800000000068000608BF70474FF0500080F3FE
:108490001188BFF36F8FBFF34F8F00BFFEE700005F
:1084A00040F23C10C2F20000016839B101390160AC
:1084B00018BF7047002080F3118870474FF05000BC
:1084C00080F31188BFF36F8FBFF34F8FFEE700007B
:1084D000B0B5002808BFB0BD044647F6E430C2F28C
:1084E0000000007854F8041C002818BF4FF000402A
:1084F00008420CD0A4F108052A6892B14FF0500050
:1085000080F31188BFF36F8FBFF34F8FFEE74FF0FB
:10851000500080F31188BFF36F8FBFF34F8F00BF00
:10852000FEE721EA000044F8040C00F01BFA47F6CD
:108530001041C2F2000154F8040C0A6810440860AB
:108540002846FFF7A7FA47F62840C2F20000016864
:108550000131016001F08EF9B0BD00004EF2100053
:10856000CEF2000000210160816040F20001C2F201
:108570000001096844F6D352C1F26202A1FB021263
:108580004FF0FF3101EB921141600721016070470C
:10859000EFF30580102814D34EF2F031CEF2000133
:1085A000405C47F2E441C2F200010978884208D2F7
:1085B0004FF0500080F31188BFF36F8FBFF34F8FE0
:1085C000FEE74EF60C50CEF2000047F2E84100689C
:1085D000C2F20001096800F4E060884298BF704769
:1085E0004FF0500080F31188BFF36F8FBFF34F8FB0
:1085F000FEE7000047F6444C0022C2F2000C00BF28
:108600005CF8323023B10132082A08BF7047F7E71F
:108610000CEBC2034CF832105860704770B5154629
:108620000E460446FFF718FF94F84400FF2804BFE5
:10863000002084F8440094F84500FF2804BF00207F
:1086400084F84500FFF72CFFA06B28B904F1240043
:1086500031462A4600F014F92046FFF739FC70BD78
:1086600010B5D8B1044647F2F840C2F200000068E5
:1086700048B14FF0500080F31188BFF36F8FBFF304
:108680004F8F00BFFEE700F06DF920460021FEF796
:10869000A3FF01F0EFF8002818BF10BD4EF60450FC
:1086A000CEF200004FF080510160BFF34F8FBFF357
:1086B0006F8F10BDB0B590B10D46D1B1044647F2F1
:1086C000F840C2F200000068E8B14FF0500080F3BB
:1086D0001188BFF36F8FBFF34F8F00BFFEE74FF0DE
:1086E000500080F31188BFF36F8FBFF34F8F00BF2F
:1086F000FEE74FF0500080F31188BFF36F8FBFF398
:108700004F8F00BFFEE700F02DF947F6B840C2F2E8
:10871000000000682268904202EB050102D29142FB
:1087200002D309E0914201D3814205D92160081AA0
:108730000021FEF751FF00E0216001F09BF80028C6
:1087400018BFB0BD4EF60450CEF200004FF080517D
:108750000160BFF34F8FBFF36F8FB0BD70B504469C
:10876000FFF77AFE40F68416002CC2F2000608BF1E
:108770003468251D2846FFF7F9FDA06A18B104F1F9
:108780001800FFF7F3FD47F2FC40C2F20000016859
:1087900001310160306884420CD047F2F040C2F2EF
:1087A00000000168013901602046FFF763F8FFF718
:1087B000F7FA0DE047F6A440C2F200002946FFF7A1
:1087C00033FE47F2F440C2F200000168013101605B
:1087D000FFF766FE47F68440C2F200000068E8B189
:1087E0003068844218BF70BD47F2F840C2F2000002
:1087F000006840B14FF0500080F31188BFF36F8FD5
:10880000BFF34F8FFEE74EF60450CEF200004FF05C
:1088100080510160BFF34F8FBFF36F8F70BD0000B9
:1088200047F62041C2F200010968016047F6B841ED
:10883000C2F20001096841607047000047F6C44079
:10884000C2F20000012101607047000010B568B15C
:108850000C4640F68411C2F2000109681831FFF796
:10886000C5FD20460121FEF7B7FE10BD4FF05000B8
:1088700080F31188BFF36F8FBFF34F8FFEE70000C7
:10888000B0B590B10D4640F68411C2F200010968FE
:1088900014461831FFF7C8FD002C18BF4FF0FF3504
:1088A00028462146FEF798FEB0BD4FF0500080F3F9
:1088B0001188BFF36F8FBFF34F8F00BFFEE700003B
:1088C00010B586B0002405A804A903AACDE9044484
:1088D000FFF75EFDDDE9032005990023CDE90101E5
:1088E00047F64110C0F600001CA1009400F0C4FC43
:1088F00047F61441C2F20001086010B101F044F8DB
:108900000446601C20D0012C1CD14FF0500080F395
:108910001188BFF36F8FBFF34F8F47F61C40C2F231
:1089200000004FF0FF31016047F68440C2F20000C2
:108930000121016047F6B840C2F200000021016049
:1089400000F07EF806B010BD4FF0500080F31188A3
:10895000BFF36F8FBFF34F8FFEE700BF49444C4515
:108960000000000047F2F840C2F200000168013147
:108970000160704710B547F2F840C2F2000000688D
:1089800030B147F6C440C2F200000121016010BDC1
:1089900047F6C440C2F20000002140F68414016092
:1089A000C2F200042068006B0168B1F1A53F0BD151
:1089B0004168B1F1A53F07D18168B1F1A53F03D16D
:1089C000C068B0F1A53F04D0206821683431FFF7BA
:1089D000FBFC47F2005CC2F2000CDCF8001040F631
:1089E0009C1201EB8103C2F2000252F8230048B945
:1089F00002EB8300A0F11403B9B153F81409013953
:108A00000028F9D001EB810002EB800252F8040F3C
:108A10004368101D8342136001D1586810601068CC
:108A2000C0682060CCF8001010BD4FF0500080F3FB
:108A30001188BFF36F8FBFF34F8F00BFFEE70000B9
:108A400080B582B04EF20040CEF200004CF27021B0
:108A5000C4F20F11D0F800294B1C9A4209D14FF0F3
:108A6000500080F31188BFF36F8FBFF34F8F00BFAB
:108A7000FEE7D0F800298A4209D14FF0500080F378
:108A80001188BFF36F8FBFF34F8F00BFFEE70178F0
:108A900047F2E4420191FF2101700178C2F2000225
:108AA0008DF803109DF8031001F05001117047F28A
:108AB000E841C2F2000107220A609DF90320B2F1E9
:108AC000FF3F0CDC0A6800BF9DF80330013A5B00F1
:108AD0008DF803309DF90330002BF5D40A600A6845
:108AE000032A2DD14FF4E06303EA02220A600199C0
:108AF0000170D0F8201941F47001C0F82019D0F8A5
:108B0000201941F07041C0F82019FFF727FD40F20D
:108B10003C10C2F2000000210160FFF793FC4EF60A
:108B20003470CEF20000016841F040410160FFF76F
:108B300019F8FFF71FFFFFF7A5F9002002B080BD6D
:108B40004FF0500080F31188BFF36F8FBFF34F8F4A
:108B5000FEE7000080B54FF0500080F31188BFF3AE
:108B60006F8FBFF34F8F00F001FD30B14EF6045010
:108B7000CEF200004FF080510160002080F3118898
:108B800080BD0000F0B581B0B0B10546484350301B
:108B900014460E46FFF7D6F9074650B1002007F1FC
:108BA000500287F846002846314623460097FEF7D4
:108BB000DDFE384601B0F0BD4FF0500080F3118863
:108BC000BFF36F8FBFF34F8FFEE70000B0B582B0E9
:108BD00068B11D46ABB1F1B9EAB14FF0500080F376
:108BE0001188BFF36F8FBFF34F8F00BFFEE74FF0C9
:108BF000500080F31188BFF36F8FBFF34F8F00BF1A
:108C0000FEE74FF0500080F31188BFF36F8FBFF382
:108C10004F8F00BFFEE751B14AB94FF0500080F3CB
:108C20001188BFF36F8FBFF34F8F00BFFEE7502354
:108C30000193019B502B0AD1069B019C012485F8CE
:108C400046400095FEF792FE284602B0B0BD4FF0B8
:108C5000500080F31188BFF36F8FBFF34F8F00BFB9
:108C6000FEE7000070B5F8B104460E46FFF7F4FBCE
:108C70002068D4E90F12002502FB0103013901FB32
:108C80000201A563C4E90103FF20E16084F8440008
:108C900084F8450004F110007EB1FFF797FB04F162
:108CA0002400FFF793FB18E04FF0500080F3118889
:108CB000BFF36F8FBFF34F8FFEE7016869B100F01C
:108CC00091FD50B14EF60450CEF200004FF08051AD
:108CD0000160BFF34F8FBFF36F8FFFF7E1FB012000
:108CE00070BD00002DE9F04F83B00292B8B11D466F
:108CF0000E460446E9B1022D03D1E06B012840F095
:108D00009A8000F00FFC00BB0298F0B14FF05000C9
:108D100080F31188BFF36F8FBFF34F8FFEE74FF0E3
:108D2000500080F31188BFF36F8FBFF34F8F00BFE8
:108D3000FEE7206C0028DED04FF0500080F3118851
:108D4000BFF36F8FBFF34F8FFEE7FFF785FBA06B7D
:108D5000022D58D0E16B884255D304F11008012050
:108D60006F464FF0000B0DF108094FF0805A00BF1D
:108D70000299002900F07B80C00702D03846FFF737
:108D80004FFDFFF78DFBFFF7EDFDFFF765FB94F857
:108D90004400FF2808BF84F844B094F84500FF2839
:108DA00008BF84F845B0FFF77BFB3846494600F022
:108DB000EBF900285ED12046FEF7C6FEA0B102996D
:108DC0004046FFF743FD2046FFF782F800F052FDD2
:108DD00078B94EF60450CEF20000C0F800A0BFF300
:108DE0004F8FBFF36F8F04E02046FFF771F800F05C
:108DF00041FDFFF731FBA06B022D04D0E16B8842EF
:108E00004FF00000B4D2204631462A46FEF7F4FC6B
:108E100054F8241FC9B1204600F0E4FC08B34EF614
:108E20000450CEF200004FF080510160BFF34F8F2D
:108E3000BFF36F8F15E04FF0500080F31188BFF340
:108E40006F8FBFF34F8F00BFFEE750B14EF6045057
:108E5000CEF200004FF080510160BFF34F8FBFF39F
:108E60006F8FFFF71DFB012003B0BDE8F08FFFF708
:108E700017FB04E02046FFF72BF800F0FBFC002076
:108E800003B0BDE8F08F00002DE9F04381B0E8B1F8
:108E90001E46914605460F4609B3022E02D1E86BE5
:108EA000012837D1FFF774FBEFF311884FF0500022
:108EB00080F31188BFF36F8FBFF34F8FA86B022E23
:108EC00019D0E96B884216D300203FE04FF05000E4
:108ED00080F31188BFF36F8FBFF34F8FFEE7286CCD
:108EE0000028DAD04FF0500080F31188BFF36F8F65
:108EF000BFF34F8FFEE795F84540A86B28463946EB
:108F00003246FEF779FCFF2C0DD0601C85F8450039
:108F100001201BE04FF0500080F31188BFF36F8FEA
:108F2000BFF34F8FFEE755F8240F70B1284600F0CD
:108F300059FC0146B9F1000F4FF0010006D000299D
:108F40001CBF0120C9F8000000E0012088F311884F
:108F500001B0BDE8F08300002DE9F04F85B0049228
:108F600098B10C460546002900F0A58000F0DAFA19
:108F7000A8B9049898B14FF0500080F31188BFF35E
:108F80006F8FBFF34F8F00BFFEE74FF0500080F3AD
:108F90001188BFF36F8FBFF34F8F00BFFEE705F15E
:108FA000240005F11009019002AF0DF1100A4FF0F5
:108FB00000080AE02846FEF78BFF00F05BFC28461D
:108FC000FEF7B6FD002840F08480FFF745FAD5F89B
:108FD00038B0BBF1000F1DD028462146FEF7F8FB44
:108FE000ABF10100A863286970B1484600F0FAFBB4
:108FF00050B14EF60450CEF200004FF080510160A7
:10900000BFF34F8FBFF36F8FFFF74AFA002001269F
:10901000A0B95FE0049850B1B8F1000F02D1384612
:10902000FFF7FEFB4FF00108012038B952E0FFF7CF
:1090300037FA0026002000284CD000BFFFF730FA96
:10904000FFF790FCFFF708FA95F84400FF2804BFEB
:10905000002085F8440095F84500FF2804BF002053
:1090600085F84500FFF71CFA3846514600F08CF8A9
:1090700000289FD12846FEF75BFDB0B10499019806
:10908000FFF7E4FB2846FEF723FF00F0F3FB002880
:109090009BD14EF60450CEF200004FF0805101609B
:1090A000BFF34F8FBFF36F8F8FE72846FEF710FF98
:1090B00000F0E0FB89E7286C00283FF457AF4FF041
:1090C000500080F31188BFF36F8FBFF34F8F00BF45
:1090D000FEE70026304605B0BDE8F08F2DE9F043ED
:1090E00081B000B3914605460E4631B3FFF750FA02
:1090F000EFF311884FF0500080F31188BFF36F8FAA
:10910000BFF34F8FAC6B24B395F8447028463146BB
:10911000FEF75EFB601EFF2FA8631CD0781C85F84D
:10912000440001202AE04FF0500080F31188BFF383
:109130006F8FBFF34F8F00BFFEE7286C0028D5D09C
:109140004FF0500080F31188BFF36F8FBFF34F8F44
:10915000FEE7002012E055F8100F70B1284600F02D
:1091600041FB0146B9F1000F4FF0010006D0002984
:109170001CBF0120C9F8000000E0012088F311881D
:1091800001B0BDE8F0830000B0B5D0B10D4611B319
:109190000446FFF761F947F6B840C2F200000168E3
:1091A0002868421C21D047F620436268C2F20003BF
:1091B000D3F800C091421AD323689C4517D00124EC
:1091C00022E04FF0500080F31188BFF36F8FBFF3A0
:1091D0004F8F00BFFEE74FF0500080F31188BFF3C0
:1091E0006F8FBFF34F8F00BFFEE700240CE0891A9A
:1091F000884206D9401A28602046FFF711FB002458
:1092000002E0002001242860FFF74AF92046B0BDA3
:109210002DE9F04383B007469000984615468946ED
:10922000FEF790FE78B106465C20FEF78BFE38B163
:109230000446066354B94FF0FF3003B0BDE8F08335
:109240003046FFF745F90024002CF4D0DDE90A1080
:10925000002284F85920CDE90010384649462A46B4
:1092600043460294FEF792FB2046FEF7F5F90120F3
:1092700003B0BDE8F083000070B586B00B9CCCB1A4
:109280000C9E06B35C250495049D5C2D25D1049DA0
:10929000DDF828C0022586F8595005AD3463CDE9C4
:1092A00000C50296FEF772FB3046FEF7D5F9059829
:1092B00006B070BD4FF0500080F31188BFF36F8F80
:1092C000BFF34F8FFEE74FF0500080F31188BFF3DC
:1092D0006F8FBFF34F8F00BFFEE74FF0500080F35A
:1092E0001188BFF36F8FBFF34F8F00BFFEE7000001
:1092F000F0B581B0D0B11D46174604460E46FFF7C3
:10930000ABF8002D1CBF606D286094F85800022156
:10931000042F84F8581012D80125DFE807F0230342
:109320001C262000616D314361651FE04FF0500045
:1093300080F31188BFF36F8FBFF34F8FFEE7616D2E
:10934000013113D04FF0500080F31188BFF36F8FBD
:10935000BFF34F8FFEE7616D0131616506E00228C2
:1093600003D1002501283CD103E0666501250128D1
:1093700037D1261D3046FEF7F9FF47F20051C2F201
:109380000001E06A0A68904288BF086040F69C11BC
:1093900000EB8000C2F2000101EB80003146FFF7D4
:1093A00043F8A06A48B14FF0500080F31188BFF332
:1093B0006F8FBFF34F8F00BFFEE740F68411C2F2FC
:1093C0000001E06A0968C96A88420AD94EF6045069
:1093D000CEF200004FF080510160BFF34F8FBFF31A
:1093E0006F8FFFF75DF8284601B0F0BD2DE9F04121
:1093F00020B31D46174604460E46FFF7C9F8EFF3A3
:1094000011884FF0500080F31188BFF36F8FBFF3C6
:109410004F8F002D1CBF606D286094F8580002210A
:10942000042F84F8581012D80125DFE807F0230331
:109430001C262000616D314361651FE04FF0500034
:1094400080F31188BFF36F8FBFF34F8FFEE7616D1D
:10945000013113D04FF0500080F31188BFF36F8FAC
:10946000BFF34F8FFEE7616D0131616506E00228B1
:1094700003D10025012849D103E0666501250128B3
:1094800044D1A06A48B14FF0500080F31188BFF377
:109490006F8FBFF34F8F00BFFEE747F2F840C2F275
:1094A0000000006830B147F6304004F11801C2F204
:1094B000000015E0261D3046FEF758FF47F2005128
:1094C000C2F20001E06A0A68904288BF086040F674
:1094D0009C1100EB8000C2F2000101EB80003146DC
:1094E000FEF7A2FF40F68411C2F20001E06A0968AB
:1094F000C96A88420AD9069800281CBF0121016068
:1095000047F6C440C2F200000121016088F31188CF
:109510002846BDE8F081000040F68410C2F2000049
:109520000068704747F68440C2F2000000680028D7
:1095300004BF0120704747F2F840C2F20000006803
:10954000B0FA80F0400940007047000047F6B8408C
:10955000C2F200000068704780B5FFF719F847F6BF
:10956000B840C2F20000006880BD00002DE9F04F55
:1095700081B047F2F840C2F20000006840B147F6FF
:109580002C40C2F20000016800240131016092E029
:1095900047F6B840C2F2000001684E1C066021D3B5
:1095A00040F68C10C2F200000168096849B14FF022
:1095B000500080F31188BFF36F8FBFF34F8F00BF50
:1095C000FEE740F69412C2F20002016813680360DD
:1095D00047F620401160C2F20000016801310160CD
:1095E000FEF7DEFB47F61C41C2F20001086840F6B8
:1095F000841A40F69C188642C2F2000AC2F20008A1
:1096000001D2002445E040F68C17C2F2000738680A
:109610000024006898B347F2005BC2F2000B19E027
:10962000D9F82C00DBF80010884288BFCBF8000086
:1096300000EB800008EB80002946FEF7F5FED9F824
:109640002C00DAF80010C96A3A68884228BF012461
:109650001068B8B13868C068D0F80C904D4655F81D
:10966000040F864210D32846FEF780FED9F8280062
:109670000028D5D009F11800FEF778FED0E74FF0AA
:10968000FF3005E04FF0FF3047F61C41C2F2000109
:109690000860DAF80000C06A00EB800058F820008B
:1096A000012847F6C440C2F2000088BF01240068C8
:1096B000002818BF0124204601B0BDE8F08F00004B
:1096C0002DE9F0411E46154688460746FEF7C4FEC2
:1096D00040F68414C2F20004206890F85800022872
:1096E00019D02068416D21EA0701416520684FF0DB
:1096F000010180F8581076B130460121FDF76CFF6A
:109700004EF60450CEF200004FF080510160BFF3DE
:109710004F8FBFF36F8FFEF7C3FEFEF79DFE15B1AF
:109720002068406D28602068002590F858100020BF
:10973000022905D1216801254A6D22EA08024A65FD
:10974000216881F85800FEF7ABFE2846BDE8F0819D
:10975000B0B580B1044640F68410C2F20000006843
:10976000A0420AD04FF0500080F31188BFF36F8FF2
:10977000BFF34F8FFEE70020B0BD206D38B3013836
:1097800020654FF0000018BFB0BDE16AE26C914265
:109790001CD0251D2846FEF7E9FDE06CC0F138011C
:1097A000A16147F20051E062C2F200010A689042F2
:1097B00088BF086040F69C1100EB8000C2F20001F7
:1097C00001EB80002946FEF72FFE0120B0BD4FF0CF
:1097D000500080F31188BFF36F8FBFF34F8F00BF2E
:1097E000FEE70000B0B5C068C5687DB105F118049A
:1097F0002046FEF7BBFD47F2F840C2F200000068C9
:1098000068B147F63040C2F200001DE04FF0500052
:1098100080F31188BFF36F8FBFF34F8FFEE72C1DCE
:109820002046FEF7A3FD47F20051C2F20001E86AAC
:109830000A68904288BF086040F69C1100EB8000E7
:10984000C2F2000101EB80002146FEF7EDFD40F67B
:109850008411C2F20001E86A0968C96A884291BFAE
:10986000002047F6C441C2F20001012088BF086011
:10987000B0BD00002DE9F04F81B047F2F844C2F2CC
:109880000004206868B1FEF7E7FD20680138206019
:10989000206880B10024FEF703FE204601B0BDE839
:1098A000F08F4FF0500080F31188BFF36F8FBFF33C
:1098B0004F8F00BFFEE747F2F040C2F200000068A1
:1098C00000285DD047F63046C2F20006306847F601
:1098D000C448C2F2000890B347F2005740F69C1902
:1098E00040F6841BC2F20007C2F20009C2F2000B6C
:1098F0004FF0010AF068C56805F11800FEF736FD63
:109900002C1D2046FEF732FDE86A3968884288BF80
:10991000386000EB800009EB80002146FEF784FDF3
:10992000E86ADBF80010C96A884228BFC8F800A0BE
:1099300030680028DED1002D18BFFEF731FA47F657
:109940002C44C2F20004256855B10126FFF70EFE33
:10995000002818BFC8F80060013DF7D10020206042
:10996000D8F8000070B14EF60450CEF200004FF06F
:1099700080510160BFF34F8F0124BFF36F8F8AE7DF
:10998000002488E7002486E780B586B0FDF7BAFE9C
:1099900047F6BC40C2F20000006808B30020CDE9E1
:1099A000040005A804A903AAFEF700FDDDE90320D1
:1099B0000221DDF814C0CDE9001047F6B960C0F609
:1099C00000000CA10023CDF808C0FFF755FC47F6B6
:1099D000C041C2F20001086010B1012006B080BD94
:1099E0004FF0500080F31188BFF36F8FBFF34F8F9C
:1099F000FEE700BF546D72205376630010B584B04B
:109A0000A8B147F6BC44C2F2000484462068C0B145
:109A10000529CDE90012CDF808C015DCFFF782FD5D
:109A200001462068022916D1069A694615E04FF0D2
:109A3000500080F31188BFF36F8FBFF34F8F00BFCB
:109A4000FEE7002004B010BD69461A460023FFF768
:109A50001BFA04B010BD694600220023FFF742F94B
:109A600004B010BD03B401984100009850EAC12031
:109A700018BF04204A0D18BF40F0010040F2FF72E9
:109A8000B2EB515F08BF40F00200012808BF05207B
:109A900002B070474100080218BF04200A0E18BF28
:109AA00040F001004FF07F4232EA010108BF40F070
:109AB0000200012808BF05207047000010B54FF0D4
:109AC0000E402DED028BB0EE408A18EE104A00EBEE
:109AD0004400B0F1506F4AD84FF0FC40B0EB440F57
:109AE00022D2B0EEC80AF7EE000A30EEC00AF6EE57
:109AF000000A60EE208A18EE900A01F0D4FD01EE13
:109B0000100A14F0004F1DBFDFED2D0A9FED2D0A46
:109B1000B1EE411ADFED2C0A08BF9FED2C0AF8EEDA
:109B2000001A21EE218A05E0DFED290A68EE088A95
:109B3000B0EE600A9FED271ADFED271A30EE080A13
:109B400048EE811A9FED251A08EEA11ADFED241ABE
:109B500048EE811A9FED231A08EEA11A68EE281A22
:109B6000BDEC028B01EE810A30EE200A10BD4FF0F1
:109B7000E440B0EB440F0CD918EE100AFFF78AFF4F
:109B8000042808BF01F092FCB0EE480ABDEC028B3D
:109B900010BD4FF07F40B0EB440F07D2B0EE480A43
:109BA000BDEC028BBDE8104001F072BC0120F6F75D
:109BB000A1FCBDEC028BBDE8104001F06FBC0000C1
:109BC0000000C9BF22AAFDB90000C93F22AAFD3981
:109BD0000000000024FE1C3DC78AD83C1E67383DAB
:109BE0001B93993DAFAA2A3E70B59B482DED020B01
:109BF0002DED068B079D25F00044A04218DC974808
:109C0000844202DC0AD1069840B19DED060BBDEC02
:109C1000068B02B0BDE8704001F0F6BB002DCCBF52
:109C20009FED8F0B9FED900BBDEC068B02B070BDCE
:109C30008F48A04215DD8F48A042D8BF4FF0FF34B7
:109C400058DD9DED060B51EC100BFFF70BFF0428C0
:109C500008BF01F00DFC9DED060BBDEC068B02B0BC
:109C600070BD9DED060B51EC100B01F0D9FCCDE958
:109C7000060181489FED828BA0423CDD8248A042D4
:109C80001FDD00249FED82AB9DED060B53EC1A2BDC
:109C900051EC100B01F064FD9DED060B41EC190B2E
:109CA00053EC1A2B51EC100B02F070F853EC182BFC
:109CB00002F078FA53EC192B01F00EFECDE9060103
:109CC00049E09DED060B012453EC182B51EC100BD1
:109CD00001F046FD9DED060B41EC190B53EC182BE2
:109CE00051EC100B02F05EFA53EC192B01F0F4FD6D
:109CF000CDE906012FE06848A0421FDD02249FED58
:109D0000689B9DED060B53EC192B51EC100B02F0E8
:109D10003DF853EC182B01F023FD9DED060B41ECB3
:109D2000180B53EC192B51EC100B02F03BFA53ECCF
:109D3000182B01F0D1FDCDE906010CE09DED060BDD
:109D4000032453EC102B9FED580B51EC100B01F03A
:109D5000C3FDCDE906019DED060B53EC102B51EC34
:109D6000100B02F013F841EC180B53EC182B02F017
:109D70000DF841EC190B4E480621B0EE490AF0EE01
:109D8000690A784401F0AAFA53EC182B51EC100B35
:109D900001F0FCFF41EC180B4648B0EE490AF0EE2A
:109DA000690A0521784401F099FA53EC192B51EC1A
:109DB000100B01F0EBFF41EC100B51EC180B53ECC6
:109DC000102B002C0EDA01F0CBFC9DED061B53ECA2
:109DD000112B01F0DBFF9DED061B53EC112B02F064
:109DE00009F935E001F0BCFC9DED061B53EC112B8D
:109DF00001F0CCFF41EC100B2F48784400EBC4007D
:109E000090ED001B51EC100B53EC112B02F0CAF932
:109E10009DED061B53EC112B02F0C4F941EC100B25
:109E20002648784400EBC40090ED001B51EC100B69
:109E300053EC112B02F0DEF841EC100B002DA2BF09
:109E4000BDEC068B02B070BD51EC100B01F04AFC6A
:109E500041EC100B01E70000000010440000F07F0F
:109E6000182D4454FB21F93F182D4454FB21F9BF10
:109E70000000DC3F0000203E0000F33F0000000037
:109E8000000000000000F03F0000E63F000000007E
:109E900000000000000000400080034000000000BF
:109EA000000000000000F83F000000000000F0BFCC
:109EB0002A2A0000E02900006A2900002229000067
:109EC00070B56F4E2DED040B2DED048B82B0DDF8D7
:109ED00024C0DDE907235C422CF000411C4341EA29
:109EE000D474069D22F00040B44205D86C422C4345
:109EF00040EAD474B4420BD99DED081B9DED060BCE
:109F000002B0BDEC048B04B0BDE8704001F086BA2D
:109F1000ACF14054A4F17F641C430BD0022404EA4A
:109F2000AC7444EAD27405439FED578B9FED582BD8
:109F300007D015E09DED060B51EC100B01F068FB0E
:109F400042E0002C11BF012C9DED060B02B0BDECD0
:109F5000048B04BF04B070BD022C38D0032C3BD05E
:109F60000B439FED4D1B9FED4E0B0AD0B14218D114
:109F7000B04209D121F0804120F080400991079042
:109F80000FE0002A15DA10E0474B7B44002C08BF95
:109F900093ED000B0DD0012C10D0022C17D0032C08
:109FA0001AD0B0421DD1002A03DAB0EE410AF0EE19
:109FB000610A02B0BDEC048B04B070BD93ED000BE0
:109FC00051EC100B01F08EFB41EC100BF1E7B0EE01
:109FD000480AF0EE680AECE7B0EE420AF0EE620AD8
:109FE000E7E7401A00159FED329B3C28C8BF8DED76
:109FF000000B17DCBCF1000FBCBF10F13C0F8DED66
:10A00000009B0FDB9DED080B53EC102B9DED060B19
:10A0100051EC100B01F060FC01F002FB01F0F8FACA
:10A02000CDE90001B4B1012C10D0022C9FED220B20
:10A0300053EC102B9DED000B51EC100B19D002F0DE
:10A04000B1F853EC182B02F0ADF8BDE7019880F0A1
:10A05000004001909DED000B53EC192B51EC100BBF
:10A0600001F094FD04BF0220F6F744FA9DED000BC9
:10A070009FE702F097F853EC182B01F0BBFFA3E722
:10A080000000F07F00000000182D4454FB2109401F
:10A09000182D4454FB2109C0182D4454FB21F9BF4D
:10A0A000182D4454FB21F93F522800000000000005
:10A0B0000000000000000000075C143326A6A13C4D
:10A0C00070B54FF068422DED048BF0EE408A18EE2B
:10A0D000900AB0EE608A18EE101A02EB4003B3F15A
:10A0E000654F3CBF02EB4102B2F1654F7DD200BF2C
:10A0F000C0F3C753C1F3C7529A1A1B2A09DD10F0E7
:10A10000004F14BF9FED830A9FED830ABDEC048BC3
:10A1100070BD12F11A0F36DA11F0004F09D010F0AD
:10A12000004F0CBF9FED7D0A9FED7D0ABDEC048BB7
:10A1300070BD88EE889A19EE100AFFF7ABFC042870
:10A1400008BF01F0B3F918EE900AFFF7A3FC05462B
:10A1500018EE100AFFF79EFC044619EE100AFFF7EE
:10A1600099FC042D18BF052D08D1042C18BF052C0F
:10A1700004D1002804BF0220F6F7BCF9B0EE490A6A
:10A18000BDEC048B70BD4200B2EB410F3AD910F028
:10A19000004F19BFDFED630A9FED630ADFED630A2D
:10A1A0009FED630AB0EE481A0A46B1EE688A80F065
:10A1B0000041F0EE418A10460A1A5200B2F1807F47
:10A1C00034D2484010F0004FDFED5A1A9FED5A2A62
:10A1D0001DBFBEEE001A70EEE10A30EE420AB6EE86
:10A1E000001A08BF70EEA10A00E040E008BF30EEA0
:10A1F000020AB0EE682A01EE482A08EE818AC2EE11
:10A20000081A15E011F0004F04BF9FED4C0AF0EE64
:10A21000400AD1D010F0004F19BFDFED490A9FED81
:10A22000490ADFED490A9FED490AC5E7C8EE881AD9
:10A2300021EEA11A9FED462ADFED462A41EE022AC1
:10A240009FED452A01EE222ADFED442A41EE022A43
:10A250009FED432ABDEC048B01EE222A21EE811AE8
:10A2600001EE020A30EE210A30EE200A70BD4FF0F6
:10A270007F42B2EB400F28BFB2EB410F09D2F0EEA4
:10A28000480AB0EE680ABDEC048BBDE8704001F0EE
:10A2900002B940EA01035B0008BF41F0FF410BD067
:10A2A000B2EB400F08BFB2EB410F08D120F0804065
:10A2B00008EE900A21F0804108EE101A18E7B2EB80
:10A2C000400F12BF5FEA410340F0FF4001F0004140
:10A2D0003FF40EAFB2EB410F12BF5FEA400200F055
:10A2E000004041F0FF413FF403AF4A0092EA4003CF
:10A2F0003FF5FEAE002AACBF9FED1A0A9FED1A0A89
:10A3000068EE808A28EE008A18EE900A18EE101A7D
:10A31000EEE60000DB0FC9BFDB0FC93FDB0F494092
:10A32000DB0F49C00000C9BF22AAFDB90000C93F28
:10A3300022AAFD390060ED3EC30ACE3700000000BE
:10A34000000049C022AA7DBA0000494022AA7D3AF5
:10A350002DAD65BD8FB8D53D0FB511BE61C84C3E62
:10A36000A8AAAABE0000804F0000802F00000000B5
:10A370002DE9F04D2DED040B2DED0E8B94B0DDE9A4
:10A380002350259CDDF888A025F0004624F00048E5
:10A39000BAF1000F14BF0121002101EB4502FC4975
:10A3A00053184A1093422AD3002814BF01230023D4
:10A3B00003EB44030B44F7498B4220D358EA0001D6
:10A3C0009FEDF5AB76D0DFF8D8B35D4503D1BAF198
:10A3D000000F05D188E0BAF1000F08BF002100D0BE
:10A3E000012101EB450111F5001F08D8002814BF19
:10A3F0000121002101EB440111F5001F0BD99DED56
:10A40000241B9DED220B14B0BDEC0E8B04B0BDE8F7
:10A41000F04D01F003B80027002DBCBFE14988458D
:10A4200021DAE1498845A8BF02271CDAC3451ADCB6
:10A43000DE4901EB2851142908DDC1F1340220FA6C
:10A4400002F101FA02F282420DD108E058B9C1F1DD
:10A45000140228FA02F101FA02F2424503D101F096
:10A460000101C1F1020756EA0A0124D1002C22DAC7
:10A47000002D18BF022F01D0012F0AD00220F6F7BD
:10A4800039F814B0BDEC0E8B04B0BDE8F04D00F00F
:10A49000A3BF0220F6F72EF800F09EFF51EC100B40
:10A4A00001F020F941EC100B14B0BDEC0E8B04B0A0
:10A4B000BDE8F08D18E09FEDBE9B9FEDBF8B00289F
:10A4C00071D1B848804522D105F1804010F5801047
:10A4D00008BFBAF1000F07D0B3450ADC002CA8BFB3
:10A4E0009DED240BE0DA0DE0B0EE4A0AF0EE6A0AC8
:10A4F000DAE7002C06DA9DED240B51EC100B01F08D
:10A50000F1F86FE0AE48784490ED000BCCE7D84509
:10A510004DD1002C48DA2EB186423AD1BAF1000F63
:10A5200042D126E0BAF1000F13D00220F5F7E2FF86
:10A5300000F08EFF8DED020B9DED220B8DED000BDB
:10A5400010EE900A039961F31E0003909DED020B3B
:10A55000AAE78DED029B9DED220B19EE901A10EEED
:10A56000900A8DED000B61F31E0003909DED020B30
:10A570009AE78DED028B9DED220B18EE901A10EEEE
:10A58000900A8DED000B61F31E0003909DED020B10
:10A590008AE709DA9DED220B51EC1A0B53EC102BD4
:10A5A00001F09AF91EE020E09DED220B7CE7864247
:10A5B0001BDAB4F1804F0DD0A4F10050B0F1FF5080
:10A5C00013D1002D11DB9DED220B51EC100B01F08E
:10A5D00033F807E09DED220B53EC102B51EC100BE0
:10A5E00000F0CABC41EC100B5EE79DED220B51EC74
:10A5F000100B01F015F8BAF1000FCDE90A0142D1B4
:10A600009FED710B46B3A6F1E040B0F17F600CD036
:10A610005E4538D1002D00DAA7B3022F0CBF012010
:10A620004FF0FF3001F04BFBDCE7002D01DD002C8B
:10A630000DDA002D01DD002C1FDB002D16DA002CB9
:10A6400014DB012F08BF9FED620B3FF42DAFB0EE7E
:10A65000490AF0EE690A27E7022F18BF002D0CD037
:10A66000012F0AD1002DFFF61FAF06E0002DB8BF65
:10A67000002C08DA012F3FF417AFB0EE480AF0EED5
:10A68000680A11E71BE0012000EBE57050EA0701C2
:10A6900015D0791EB0EE4A8AF0EE6A8A084308BFE8
:10A6A0009FED4D8B4E480025804570DD4D494E484D
:10A6B000884514DDB0420DDB002C19DB2FE00120B2
:10A6C000F5F718FF14B0BDEC0E8B04B0BDE8F04DEB
:10A6D00000F0AEBEB34502DC002C09DC1FE0864270
:10A6E00002DA002C1BDA03E05E452BDD002C16DDC0
:10A6F0000220F5F7FFFE00F0ABFE8DED020B53ECF0
:10A70000192B51EC180B01F041FBCDE90001039925
:10A71000019861F31E0003909DED020BC4E6022038
:10A72000F5F7E8FE00F0A4FE10EE901A18EE900A7D
:10A730008DED020B8DED008B61F31E0003909DEDFE
:10A74000020BB1E69DED0A0B53EC1A2B51EC100BEA
:10A7500001F028FD9FED260BCDE90A0153EC102BEB
:10A760009DED0A0B51EC100B01F010FB9FED221B2D
:10A7700053EC112B01F03EFC9DED0A1B53EC112B09
:10A7800001F004FB9FED1E1B53EC112B3CE08CE011
:10A79000FFFF1F00FFFF0F00000000000000F03F60
:10A7A0000000F03F0000F07F0000404301FCFFFF8D
:10A7B000000000000000F07F00000000000000002A
:10A7C000D622000000000000000000000000008011
:10A7D000000000000000F0FF000000000000F0BFDB
:10A7E0000000E0410000F043FFFFEF3F00000000E9
:10A7F000000000000000D03F555555555555D53F38
:10A80000000000000000E03F01F0F4FB9DED0A0BAA
:10A8100041EC190B53EC102B51EC100B01F0B6FA74
:10A8200053EC192B01F0B2FA9DED0A0B41EC1B0B16
:10A8300053EC102B9FEDFE0B51EC100B01F0A6FA20
:10A8400041EC190B9FEDFC0B51EC1B0B53EC102B47
:10A8500001F09CFA41EC1B0B9FEDF90B53EC102B14
:10A860009DED0A0B51EC100B01F090FA53EC1B2BF1
:10A8700001F098FC41EC1B0B51EC190B53EC1B2B1A
:10A8800000F06EFF0490CDE904519DED040B53ECF4
:10A89000192B51EC100B01F085FC53EC1B2B01F034
:10A8A000A9FB41EC100B00F0A9B90020B6F5801F00
:10A8B0000EDA9FEDE50B53EC102B9DED0A0B51ECDE
:10A8C000100B01F063FACDE90A016FF034000E4677
:10A8D00000EB2650A0F2FF37C6F31300DC4940F02E
:10A8E0007F6646F040568842D8BF002408DDD9492B
:10A8F0008142C8BF012403DC0024A6F580167F1C1A
:10A90000D548784400EBC4080B9698ED000B53EC47
:10A91000102B9DED0A0B51EC100B01F043FC98ED50
:10A92000000B41EC1B0B53EC102B9DED0A0B51EC73
:10A93000100B00F015FF41EC100B51EC1A0B53EC0F
:10A94000102B00F0C9FF41EC1C0B51EC1B0B53EC1E
:10A950001C2B01F01BFA41EC190BC0488DED0E9B2E
:10A9600078440E9590ED000B4FF0005040EA6600E1
:10A9700000EB84408DED120B00F50020139098ED54
:10A98000000B53EC102B9DED120B51EC100B01F052
:10A9900009FC9DED0A1B53EC112B01F02BFB41EC44
:10A9A000100B53EC102B9DED0E0B51EC100B01F026
:10A9B000EDF99DED120B41EC1D0B53EC102B9DEDB1
:10A9C0000E0B51EC100B01F0E1F953EC1B2B01F0D5
:10A9D00011FB53EC1D2B01F0E5FB53EC1C2B01F09C
:10A9E000D5F941EC1C0B53EC192B51EC190B01F070
:10A9F000CDF941EC1B0B9A480621B0EE4B0AF0EE64
:10AA00006B0A784400F06AFCB0EE401AF0EE601A6F
:10AA1000B0EE41DAF0EE61DA53EC1B2B51EC1B0B7C
:10AA200001F0B4F953EC1D2B01F0B0F99DED0E0BC4
:10AA300041EC1B0B53EC192B51EC100B00F090FE6A
:10AA400053EC1C2B01F0A2F953EC1B2B00F088FEF9
:10AA50009DED0E0B41EC1B0B53EC102B51EC100B2E
:10AA600001F094F941EC1D0B53EC1D2B9FED7EEB97
:10AA700051EC1E0B00F074FE53EC1B2B00F070FE2B
:10AA80001290CDE912519DED120B53EC1E2B51EC9F
:10AA9000100B01F087FB53EC1D2B01F083FB53ECF3
:10AAA0001B2B01F0A7FA9DED120B41EC1D0B53EC93
:10AAB000102B9DED0E0B51EC100B01F067F941ECE2
:10AAC0001B0B53EC192B51EC1D0B01F05FF99DEDA5
:10AAD000120B41EC190B53EC102B51EC1C0B01F039
:10AAE00055F953EC192B00F03BFE41EC190B51ECDE
:10AAF0001B0B53EC192B00F033FE0490CDE90451ED
:10AB00009DED040B53EC1B2B51EC100B01F04AFB99
:10AB100053EC192B01F06EFA9DED040B41EC190B6F
:10AB200053EC102B9FED520B51EC100B01F02EF952
:10AB300041EC1B0B9FED500B51EC190B53EC102B00
:10AB400001F024F99DED040B41EC190B53EC102B93
:10AB50009FED4B0B51EC100B01F018F953EC192B36
:10AB600000F0FEFD41EC100B4748784400EBC400B8
:10AB700090ED001B51EC100B53EC112B00F0F0FD8D
:10AB800041EC190B384601F09AF8CDE90A0153EC73
:10AB9000192B51EC1B0B00F0E3FD41EC100B3B4873
:10ABA000784400EBC40451EC100B94ED001B53EC03
:10ABB000112B00F0D5FD9DED0A1B53EC112B00F07D
:10ABC000CFFD0490CDE904519DED0A0B53EC102B01
:10ABD0009DED040B51EC100B01F0E4FA94ED001B19
:10ABE00053EC112B01F0DEFA53EC1B2B01F0DAFAD7
:10ABF00053EC192B01F0FEF941EC100B9DED241BD9
:10AC000053EC102B8DED001B00959DED240B51ECAA
:10AC1000100B01F0BBF89DED000B41EC190B53EC50
:10AC2000102B9DED240B51EC100B01F0BBFA2FE023
:10AC3000000000604715F73FFE822B654715F73F80
:10AC400044DF5DF80BAE543E0000000000004043BE
:10AC50008E9803007AB60B00BA1D00007C1E00001F
:10AC6000EA1C000000000000000000000000084096
:10AC7000000000E009C7EE3FFD033ADC09C7EE3FE4
:10AC8000F5015B14E02F3EBE721B00002C1B000080
:10AC90009DED041B53EC112B01F078F853EC192BAC
:10ACA00000F05EFD9DED040B41EC190B53EC102BF5
:10ACB0009DED000B51EC100B01F068F8CDE904019B
:10ACC0009DED040B51EC190B53EC102B00F048FDDB
:10ACD000CDE902010C46AA498C422FDB611A0843D8
:10ACE00018D19DED040B53EC102B9DED020B51EC94
:10ACF000100B01F057FA41EC1B0B9FEDA30B51EC2D
:10AD0000190B53EC102B00F02BFD53EC1B2B01F017
:10AD10003BF92DD20220F5F7EDFB00F099FB10EE88
:10AD2000901A18EE900A8DED020B8DED008B61F3F9
:10AD30001E0003909DED020BFFF7B6BB944A24F072
:10AD40000041914214D39349214408437FF4E7AC76
:10AD50009DED040B53EC102B9DED020B51EC100BF1
:10AD600001F020FA53EC192B01F00EF97FF6D7AC65
:10AD700024F000408849894A002601EB2051824294
:10AD80002BDA481C4FF4801121FA00F02044844A49
:10AD9000C0F30A517A44A1F2FF3192ED000B814ACF
:10ADA0008DED0A0BCA4020EA0202C0F3130040F402
:10ADB0008010C1F1140120FA01F60B92002CB8BFEB
:10ADC00076429DED0A0B53EC102B9DED040B51ECDC
:10ADD000100B01F0E7F9CDE904019DED040B51ECF6
:10ADE000190B53EC102B00F0BBFC9FED6F0B0A907E
:10ADF000CDE90A5153EC102B9DED0A0B51EC100BD1
:10AE000000F0C4FF41EC1B0B9FED690B53EC102BC2
:10AE10009DED0A0B51EC100B00F0B8FF9DED040BFB
:10AE200041EC1C0B53EC102B9DED0A0B51EC100B5D
:10AE300001F0B8F953EC192B01F0DCF89FED5E1B23
:10AE400053EC112B00F0A2FF53EC1C2B00F088FCFC
:10AE500041EC190B51EC1B0B53EC192B00F080FC4F
:10AE6000CDE902019DED020B53EC1B2B51EC100BB5
:10AE700001F098F953EC192B01F0BCF89DED020B91
:10AE800041EC190B53EC102B51EC100B00F07EFF32
:10AE9000CDE90A014A489DED0A0B0521784400F0EE
:10AEA0001DFA9DED0A1B51EC100B53EC112B00F019
:10AEB0006DFF9DED021B53EC112B01F09BF8CDE9CA
:10AEC00004019DED020B53EC192B51EC100B00F01B
:10AED0005DFF53EC192B00F043FC9FED3B0B41EC65
:10AEE000190B53EC102B9DED040B51EC100B01F0E2
:10AEF00059F99DED040B41EC1B0B53EC102B9DED10
:10AF0000020B51EC100B00F041FF53EC1B2B00F037
:10AF1000E3FC53EC192B01F045F99DED021B53ECBA
:10AF2000112B01F03FF953EC1A2B01F063F8CDE936
:10AF3000020101EB065001150029C8BF039015DC82
:10AF40009DED020B324651EC100B01F071FBFEF748
:10AF500089FD042808BF00F08BFA32469DED020BF4
:10AF600051EC100B01F064FBCDE902019DED020BE9
:10AF700051EC180B53EC102B00F008FFFFF732BB1D
:10AF80000000904000000000FE822B654715973CB2
:10AF900000CC904000346F3F01FCFFFF0000E03F19
:10AFA000481A0000FFFF0F0000000000432EE63F9C
:10AFB000396CA80C615C20BEEF39FAFE422EE63FE8
:10AFC00080180000000000000000000000000040A9
:10AFD00000B510EE101A2DED028B81B0524A684672
:10AFE000B2EB410F2ED94FF0E640B0EB410F94BFCA
:10AFF00000204FF0FF3000900098B0EE408A00280B
:10B000006ADB10F0010F4BD068EE080A9FED471A7B
:10B010009FED470A00EE810A9FED461A10F0020FDD
:10B0200000EE801AB7EE000A00EE810A02BF01B0FE
:10B03000BDEC028B00BD00BF01B0B1EE400ABDEC1B
:10B04000028B00BD3C4B21F00042934241D911F0EC
:10B05000004FDFED3A0A20EE201ADFED390A19BF62
:10B0600031EE601A71EE200A31EE201A71EE600A9C
:10B07000BDEEE01A11EE100A9FED321A00F0030047
:10B0800000EEC10A9FED301A009000EEC10A9FED5C
:10B090002F1A00EEC10A9FED2E1A00EEC10AABE78F
:10B0A00028EE080A9FED2B1ADFED2B0A10F0020F95
:10B0B00040EE010A9FED291A00EE201A61EE000A07
:10B0C000B0EE480A08EE200AB6D101B0BDEC028B02
:10B0D00000BD00F0F3F98FE718EE100A4000B0F160
:10B0E0007F4F0DD218EE100AFEF7D4FC042808BFDB
:10B0F00000F0DCF9B0EE480A01B0BDEC028B00BDF7
:10B1000009D10120F5F7F6F901B0BDEC028B5DF82D
:10B1100004EB00F0C3B901B0B0EE480ABDEC028BFD
:10B120005DF804EB00F0B4B9B61F927EB93AB2BA3A
:10B13000CA9F2A3DDDFFFFBE490E494683F9223FE3
:10B140000000004B0000C93F00A0FD390020A233E1
:10B150001A61342C336D4CB9DA82083CA0AA2ABE9D
:10B1600000B510EE101A2DED028B81B04D4A6846E5
:10B17000B2EB410F3CD94FF0E640B0EB410F94BF2A
:10B1800000204FF0FF3000900098B0EE408A002879
:10B190005FDB28EE080ADFED440A9FED441A00EE5B
:10B1A000201ADFED430A40EE010A9FED421A00EE3D
:10B1B000201ADFED410A10F0010F40EE010A9FED69
:10B1C0003F1A00EE201A61EE000AB0EE480A08EEBF
:10B1D000200A02BF01B0BDEC028B00BDBFEE001A19
:10B1E00001B0C1EE000ABDEC028BB0EE600A00BDFA
:10B1F000334B21F00042934228D911F0004FDFED8C
:10B20000310A20EE201ADFED300A19BF31EE601A44
:10B2100071EE200A31EE201A71EE600ABDEEE01ADE
:10B2200011EE100A9FED291A00F0030000EEC10A8A
:10B230009FED271A009000EEC10A9FED261A00EE3E
:10B24000C10A9FED251A00EEC10A9DE700F036F90C
:10B250009AE718EE100A4000B0F17F4F0DD218EEB9
:10B26000100AFEF717FC042808BF00F01FF9B0EE23
:10B27000480A01B0BDEC028B00BD09D10120F5F7F1
:10B2800039F901B0BDEC028B5DF804EB00F006B9B2
:10B2900001B0B0EE480ABDEC028B5DF804EB00F0A3
:10B2A000F7B80000B61F927EBCE9223C0B6D063B4E
:10B2B0008A76CE3CACB5593D35A1083E29AAAA3EB6
:10B2C000490E494683F9223F0000004B0000C93F68
:10B2D00000A0FD390020A2331A61342C70B5044659
:10B2E0002DED028B4D1E00EBC500B0EE408AF0EE56
:10B2F000608A90ED000B35F0060017D053EC182B48
:10B3000051EC100B00F042FD41EC100B6D1E04EBF4
:10B31000C50090ED001B51EC100B53EC112B00F00D
:10B320001FFA41EC100B35F00600E7D1022D36D0A4
:10B33000042D1CD0062D1CBFBDEC028B70BD53EC40
:10B34000182B51EC100B00F021FD94ED0A1B53EC6F
:10B35000112B00F005FA53EC182B00F017FD94EDBB
:10B36000081B53EC112B00F0FBF941EC100B53ECD4
:10B37000182B51EC100B00F009FD94ED061B53EC5B
:10B38000112B00F0EDF953EC182B00F0FFFC94EDBD
:10B39000040B53EC102B00F0E3F941EC100B53ECD1
:10B3A000182B51EC100B00F0F1FC94ED021B53EC48
:10B3B000112B00F0D5F953EC182B00F0E7FC94EDBD
:10B3C000001B53EC112B00F0CBF9BDEC028B41ECD0
:10B3D000100B70BD000000009FED070B10B553EC83
:10B3E000102B9FED070B51EC100B00F075FA41ECA0
:10B3F000100B10BD00000000000000000000000065
:10B40000000000000000F03F10B553EC102B51EC91
:10B41000100B00F0A5F941EC100B10BD10B553EC6A
:10B42000112B51EC100B00F09BF941EC100B10BDEF
:10B430009FED050B10B553EC102B51EC100B00F0E9
:10B440004BFA41EC100B10BD0000000000000000A2
:10B450009FED050B10B553EC102B51EC100B00F0C9
:10B4600095FC41EC100B10BD0000000000000070C6
:10B470009FED050B10B553EC102B51EC100B00F0A9
:10B4800085FC41EC100B10BD000000000000001016
:10B4900030EE000A704730EE200A7047DFED020AF6
:10B4A00080EEA00A70470000000000009FED020A35
:10B4B00020EE000A70470000000000102DE9F001A6
:10B4C0004FF07F42B2EB410F9FBF4FF0FF31016061
:10B4D000BDE8F00170474FF0004242EA0123C1F39A
:10B4E000C752783A551112F01F0C434CCCF120068C
:10B4F0007C44C1F3C752A2F178024FEA621204EB16
:10B50000820254F8254008BFD2E9015612D055688E
:10B5100004FA0CF425FA06F73C43976805FA0CF593
:10B5200027FA06F8D26807FA0CFCF24045EA08054B
:10B530004CEA0206A4FB034CA5FB0352A6FB0363E3
:10B540001D449D4234BF012600261319334416B111
:10B55000934202D903E0934201D2012200E000228B
:10B56000624402F1200C9206DC0C42EA443200EE06
:10B57000102A5B03DFED210AF8EEC01A00EE103A44
:10B580004FEA9C1C11F0004FB8EE400AC0F800C012
:10B5900020EE201A00EE105ADFED190AB8EE400A2C
:10B5A00020EE200A71EE810A70EE800A10EE902AD9
:10B5B00002F500626FF30B0200EE902A70EEE11AC2
:10B5C00031EEC11ADFED101A30EE411A9FED0D0A6F
:10B5D00020EE800A01EE210A9FED0C1A00EE810A8E
:10B5E00004BFBDE8F0017047CCF180510160BDE8B7
:10B5F000F001B1EE400A7047F4120000000000367E
:10B600000000802C22AAFD29DB0FC92F0000C92FC2
:10B6100010B541EC100BFEF7E7FA51EC100B10BD22
:10B6200082B0CDE9000121F0004001909DED000BBA
:10B6300002B051EC100B704700B52DED048B83B0B8
:10B6400041EC190B00F0E2FC41EC180B18EE100A6B
:10B6500018EE901A8DED008B002818BF01200843CA
:10B6600020F00040C0F17F6000F1E040C00F14D036
:10B6700019EE101A19EE900A8DED009B002918BFE3
:10B680000121084320F00040C0F17F6000F1E0405C
:10B69000C00F04BF0120F4F72DFF51EC180B03B0CD
:10B6A000BDEC048B00BD10B500EE100A2DED028B31
:10B6B000B1EEC08A18EE100A20F00040C0F1FF4041
:10B6C000C00F0AD010EE100A20F00040C0F1FF4079
:10B6D000C00F04BF0120F4F70DFF18EE100ABDECF7
:10B6E000028B10BD81F00041704780F00040704730
:10B6F00021F00041704720F00040704721F00042E7
:10B7000001F00043A2F16052B2F5801F28BFD2F1D0
:10B710007F6C0BD95FEA001C43EAC20242EB507017
:10B7200018BF704728BF20F001007047B2F5801F96
:10B73000BCBF184670474FEA410C1CF5001F02D2EF
:10B74000084600F0CBBE70B500F0CAFB00000089CF
:10B75000FFF7F6BF4FF00040A0F5800070470000F3
:10B7600010B591EA030F48BF83F0004300F1228532
:10B77000841A71EB030C05D2121943EB0C03001B66
:10B7800061EB0C014FEA1154A4EB135CDFF81CE1F0
:10B790001EEA430F18BF9EEA445F00F0748021EA5E
:10B7A000045123EA0E0343F48013DCF1200E32D35C
:10B7B00022FA0CFE10EB0E0023FA0CFE41EB0E01F8
:10B7C000CCF1200E03FA0EFE10EB0E00CCF1200E91
:10B7D00051F10001B1F5801F32D201EB045112FA90
:10B7E0000EF2BDE8104058BF7047401C38BF5FEAFA
:10B7F000420218BF7047002814BF20F0010041F139
:10B8000000014FEA410313F5001F38BF7047A1F153
:10B81000C04100F0B3BB012A43EB0302ACF1200CA2
:10B82000DCF11F0E32BF4FF0000E23FA0CF310EBC9
:10B83000030041EB0451B4EB115FD0D0A1EB0451F4
:10B8400001F58011490801EB04515FEA30000ED385
:10B8500050F1000038BF12FA0EFE08D1BDE81040CA
:10B86000C9E7401C38BF5FEA4202CAD1C3E7BDE85E
:10B8700010404FEA410313F5001F38BF7047A1F194
:10B88000C04100F07BBB9EEA445F08D011EA5E0F26
:10B89000BDE8104004BF01F0004100207047BDE842
:10B8A000104070B500F01CFB64FBBE3E0000E0FFE2
:10B8B00002494FF0000000F089BE00BF0000F87F91
:10B8C000491058BFC1F140415B1058BFC3F140431C
:10B8D0008B42EFF3008070472DE9C04130B4DFF8B0
:10B8E000A4C23CEA111418BF3CEA131400F0ED8026
:10B8F0001CEA111481EA030544EAD57418BF1CEA56
:10B90000131500F0C880A4EB050404F17F7404F55E
:10B9100000344FF0004545EAC12145EAC32341EA1E
:10B92000505143EA52534FEAC0204FEAC222994293
:10B9300008BF904200F09D804FEA13650FF2441655
:10B94000765D4FEA134506FB05F7C7F1807706FBE6
:10B9500007F74FEAD737A7FB03687642A7FB06CE67
:10B96000C8F5803838BFA8F1010807FB08E6A6FB38
:10B97000028C4FF0000EE6FB03CEDCF1000CCEF1A2
:10B98000004E38BFAEF1010EA6FB0C584FF0000779
:10B99000E6FB0E87A1FB08C6A0FB07CE16EB0E0642
:10B9A0004FF0000545F10005E1FB076515F1E04E9C
:10B9B0007EBFA4F580345FEA46066D4116F180072C
:10B9C00045F100054FEA172747EA05674FEA1525B5
:10B9D0004FEA0666A6F1DE46B6F1805F20D938460A
:10B9E00005EBC47124F0010C01EB0C11BCF1FE6FEE
:10B9F00002D8F0BCBDE8008124425CBF01F5801E86
:10BA00009EEAC47F02D4F0BCBDE80081244200F16C
:10BA10003980A1F1C041F0BCBDE8004100F0AEBAF0
:10BA20004FEAD02040EA41504FEAD1214FEAD222DA
:10BA300042EA43524FEAD323A7FB028607FB036681
:10BA400005FB02661EEA0E0F58BFA6EB0056B6EBCA
:10BA500000564FEA520E4EEAC37E18EB0E0E56EB1E
:10BA6000530EBCD518EB02085E417F1C55F1000552
:10BA7000B5E74FF480154FF000074FF000064FF088
:10BA80000008ACE701F1C04101F000414FF00000B7
:10BA9000F0BCBDE800810CEA131511EA0C1F00D0C0
:10BAA0000CE013EA0C1F00F026804FF0000081EA42
:10BAB000030101F00041F0BCBDE80081F0BCBDE82D
:10BAC000004181EA030100F059BAF0BCBDE8004131
:10BAD00070B500F005FA00BF097EFC3E00F007B823
:10BAE0004FF0000081EA030101F00041704781EA54
:10BAF000030100F043BAF0BCBDE8004122494FF019
:10BB000000007047FFFDFBF9F7F5F4F2F0EEEDEB06
:10BB1000E9E8E6E4E3E1E0DEDDDBDAD8D7D5D4D34B
:10BB2000D1D0CFCDCCCBCAC8C7C6C5C4C2C1C0BF97
:10BB3000BEBDBCBBBAB9B8B7B6B5B4B3B2B1B0AF9D
:10BB4000AEADACABAAA9A8A8A7A6A5A4A3A3A2A181
:10BB5000A09F9F9E9D9C9C9B9A999998979796953C
:10BB600095949393929191908F8F8E8E8D8C8C8BD8
:10BB70008B8A898988888787868585848483838260
:10BB8000828181800000FF070000F87F51EA030CEA
:10BB900017D41CF5801F58BFBCF5801F00F106802C
:10BBA000994218BF704708BF9042704707D711F5F8
:10BBB000801F58BF13F5801F19D4994270478942DE
:10BBC00070471CF5801F08D5BCF5801FF7D58B4248
:10BBD00018BF704708BF824270474FF4001C1CEB2F
:10BBE000410F38BF1CEB430F01D28B42704770B539
:10BBF00000F076F9922449004FF000514FF0805345
:10BC0000FFF75EBE4FEA41034FEA5353A3F580634B
:10BC1000D3F11E03C8BFD3F1210C0CDD4FF000425D
:10BC200042EAC12242EA505232FA03FC8CEAE17C39
:10BC3000ACEBE1707047102BC4BF0020704703F5D8
:10BC4000787CBCF1FF3F04D06FF0004282EA210013
:10BC5000704770B500F044F9499224800020704785
:10BC6000F2E700004FEA1153A3F58063D3F11E03FE
:10BC7000A8BFD3F1200C08DB4FF0004242EAC122FA
:10BC800052EA505232FA03F0704709420BD4102B9B
:10BC9000C4BF0020704703F5787CBCF1FF3F05D09E
:10BCA0004FF0FF3070474FF00000704770B500F064
:10BCB00017F900BF4992248000207047F0E710F088
:10BCC000004248BF4042B0FA80F310FA03F10AD0B4
:10BCD000C3F11D0303F5806302EB03524FEA4150A9
:10BCE00002EBD12170474FF000007047B0FA80F3AB
:10BCF00010FA03F10AD0C3F11D0303F580634FEA84
:10BD000003524FEA415002EBD12170474FF000003F
:10BD10007047000051EA030C17D41CF5801F58BF70
:10BD2000BCF5801F00F10680994218BF704708BF1C
:10BD30009042704707D711F5801F58BF13F5801F39
:10BD400019D499427047894270471CF5801F08D565
:10BD5000BCF5801FF7D58B4218BF704708BF8242E1
:10BD600070474FF4001C1CEB410F38BF1CEB430F16
:10BD700001D28B42704770B500F0B2F892244900AE
:10BD80004FF000514FF08053FFF79ABD70B5DFF8C8
:10BD900048C11CEA111E1EBF1CEA13159EEA0C0FB7
:10BDA00095EA0C0F00F06F8081EA03044EEAD47E1E
:10BDB000AE4421EA4C1123EA4C1341F4801143F4C0
:10BDC0008013AEF17F7EA1FB024CA0FB0365361908
:10BDD00055EB0C05A1FB034C4CF10003A0FB021C2E
:10BDE00016EB0C06654153F10003094218BF46F0FB
:10BDF000010613F4007F0BD14FEA03314FEA0530FF
:10BE000041EA155140EA165034036FF003020AE08C
:10BE10004FEAC3214FEAC52041EA555140EA565046
:10BE2000F4026FF0020202EB2E4201EB025585EAAA
:10BE3000CE710AD05FEA440C18BF24F0004450F1E0
:10BE4000000041F1000120EAD47040F2FE7C62451E
:10BE500000D270BDA84214BF4FF080444FF0404460
:10BE6000002E08BF0024BEF1806FA8BFA1F1C04121
:10BE7000BDE8704080F2828001F1C04101F00041D4
:10BE80004FF0000070470CEA13159EEA0C0F18BF24
:10BE900095EA0C0F06D081EA030E4FF000000EF079
:10BEA000004170BD00F01CF88900013E00F007B8A9
:10BEB00000F009B84FEA430C5FEA5C5C08D081EA05
:10BEC000030100F05BB84FEA410C5FEA5C5CF6D11D
:10BED00002494FF0000070470000FF070000F87FA4
:10BEE0000EF1020E2EF0030E5EF8046B364205D4FE
:10BEF000012A43EB030515F5001F12D8012841EB79
:10BF0000010C1CF5001F0CD80ED14FEAD17C0CEBB4
:10BF10004C0C0CF1020C15F5001F08BF4CEBD37C48
:10BF200004E04FF0080C01E04FEAD37C0CEB4C0529
:10BF300026FA05F606F00706B6F1040C06D20EEB5B
:10BF4000860CBDE870404CF0010C6047DFE80CF057
:10BF5000090B02024FF00041A1F500214FF0000053
:10BF600070BD19461046012851EB010418BFD4F5E5
:10BF7000001484BF002001F0004170BD0808A0F546
:10BF800000114FEA3101704753EA010C17D41CF538
:10BF9000801F58BFBCF5801F00F106808B4218BF80
:10BFA000704708BF8242704707D713F5801F58BFFC
:10BFB00011F5801F19D48B4270479B4270471CF5C6
:10BFC000801F08D5BCF5801FF7D5994218BF704770
:10BFD00008BF904270474FF4001C1CEB430F38BF62
:10BFE0001CEB410F01D2994270470FB40CBC03BC4B
:10BFF000FFF7C1BE10B591EA030F81F000413FF594
:10C00000B7AB83F0004300F0D5B800002DE9F04154
:10C0100001F5801CBCF5001FC0F2A9804FEA115C3D
:10C0200021EA0C5141F480110CF1FD0C5FEA5C0C2B
:10C030000CF5C07C01D340004941890241EA90518E
:10C0400087022EA48E0EA45D0A0C04FB04F602FBEC
:10C0500006F6C6F14046A4FB0662F60D46EA422605
:10C0600006FB06F4A4FB01235242C3F1404338BF50
:10C070005B1EA6FB02420024E6FB0324D20B42EA2D
:10C080004446A6FB0623A1FB02E2A3FB07E4E3FB75
:10C0900061426442C2F1404E38BFAEF1010EA6FBD0
:10C0A00004234FF00002E6FB0E32A2FB03463400ED
:10C0B000E2FB6264A1FB06E6A4FB07E8E4FB61681F
:10C0C0007642C8F1405838BFA8F10108A2FB06E447
:10C0D000A3FB08E5E2FB6854A1FB05E6A7FB04E827
:10C0E000E1FB648618F1200556F10006A80940EA34
:10C0F0008660B109A8F11B0808F03F08B8F10A0FE3
:10C100001CD901EB0C51BDE8F08100BFFCF5EEE855
:10C11000E2DDD8D3CFCBC7C3C0BDB9B6B4B1AEACE6
:10C12000A9A7A5A3A19F9D9B9A9896959392908F5E
:10C130008D8C8B898887868584838281A0FB0068AB
:10C1400000FB01F208EB4208B8EB872807D534184A
:10C1500058EB0104D5D5401C51F10001D1E7341A48
:10C1600078EB0104CDD4401E71F10001C9E75FEA0C
:10C170004C0C5FEA9C5C0DD105D301F000414FF0FF
:10C180000000BDE8F081BDE8F04170B5FFF7A8FE02
:10C190006DDBFFBEBDE8F04101494FF00000704784
:10C1A0000000F87F10B591EA030F48BF83F0004309
:10C1B0003FF5DEAA841A71EB030C07D28CF0004C19
:10C1C000121943EB0C03001B61EB0C014FEA1154F5
:10C1D000A4EB135CDFF8A4E11EEA430F18BF9EEA4C
:10C1E000445F00F0B48021EA045123EA6E03524216
:10C1F000C3EB6E0338BF5B1EDCF1200E25D322FAA1
:10C200000CFE10EB0E0043FA0CFE41EB0E01CCF1DC
:10C21000200E03FA0EFE10EB0E00CCF1200E51F1B1
:10C22000000129D401EB045112FA0EF2BDE81040CE
:10C2300058BF7047401C1CBFB2F1004F7047002828
:10C240000CBF491C20F00100704712EB020E43EBBB
:10C25000030218BF4FF0010E4EEA4202ACF1200C6F
:10C26000DCF11E0E56D943FA0CFE10EB0E00CCF199
:10C270001E0E51F1FF31D5D50EF1010E12FA0EFE50
:10C28000404141EB010101EB445C5FEA5C5C10D989
:10C2900001EB045110EBDE7038BFBEF1004FBDE87A
:10C2A000104018BF704700280CBF491C20F0010047
:10C2B000704734D24FEAD42C24F4006411F50011F5
:10C2C0001BD0B1FA81F20B3AA41AA41ED2F12003BA
:10C2D000914030FA03F31943904001EBCC7101EB2C
:10C2E0000451002CBDE81040A8BF704701F1C041C7
:10C2F00001F000414FF000007047B0FA80F310FAEF
:10C3000003F102D1BDE810407047E41A173C48051C
:10C31000C90AE2E701EB0451BDE81040704749103B
:10C320004FEA300001EB0451BDE8104002E04FF04D
:10C33000000170474A0008BF0042F8D0B2F5001F64
:10C3400028BF704701F000414FF0000070479EEA9F
:10C35000445F07D011EA5E0FBDE8104004BF002122
:10C3600000207047BDE8104070B5FFF7B9FD00BF71
:10C3700040DFF63E104683F0004170470000E0FFCA
:10C3800043004FEAD30C4FEA3C0C43401FBF400729
:10C390000CF1605113F0FE4F70471CF0006F03D199
:10C3A0000CF00041002070470CF0004343EA50704D
:10C3B00040EACC0010B500F03EF800BF000000924B
:10C3C0004FEA0001FFF7DABD4FF00041A1F500216F
:10C3D0004FF0000070474FF07E5209E011F000422C
:10C3E00004D54042C1F1000138BF491E42F07E52DF
:10C3F00002F170620B0012BF20235FEA0001704758
:10C40000B1FA81FC01FA0CF1A3EB0C0320FA03FC56
:10C4100041EA0C0102EBC352C3F1200310FA03FC02
:10C420005CEA416C42EB112018BF5FF0806C28BFC2
:10C4300020F0010070470EF1020E2EF0030E5EF8A0
:10C44000044B244204D44FEA4102B2F17F4F11D889
:10C450004FEA4003B3F17F4F0CD80ED14FEAD07CA6
:10C460000CEB4C0C0CF1020CB2F17F4F08BF4CEB03
:10C47000D17C04E04FF0080C01E04FEAD17C0CEBDA
:10C480004C0324FA03F404F00704B4F1040C06D2BC
:10C490000EEB840CBDE810404CF0010C6047DFE867
:10C4A0000CF0070802024FF00040A0F5800010BD1C
:10C4B0000846420018BFD2F1807288BF00F00040E9
:10C4C00010BDF1EE100A4FF6FF71C0F2C03120EA44
:10C4D000010040F04070E1EE100A7047FF2141EA90
:10C4E000D050C00570470000C2154FEA002318BFA6
:10C4F00043F0004300F11080D2F1BE0240F22880E8
:10C5000023FA02F1B2F1200C2EBF23FA0CF0C2F193
:10C51000200C03FA0CF07047B0F15F4F00F2188066
:10C5200012F0FF0208BF23F00043C2F1BE0223FA5B
:10C5300002F1B2F1200C2EBF23FA0CF0C2F1200C54
:10C5400003FA0CF04042C1F1000138BF491E7047A8
:10C5500010B5FFF770FF00BF922449804FF0000133
:10C56000002070476FEAE07080F0004170470000E3
:10C57000C2154FEA002318BF43F000430ED4D2F196
:10C58000BE0215D323FA02F1B2F1200C2EBF23FA1A
:10C590000CF0C2F1200C03FA0CF070474FEA400C8B
:10C5A000BCF1FE4F04D24FF000004FF00001704785
:10C5B00010B5FFF740FF00BF922449804FF0000103
:10C5C000002070476FEAE070014670470CF00F03DF
:10C5D000092B08BF082000F059800A2B0BD0082B2C
:10C5E00018BF704708BF1CF0400F0AD04FF0000082
:10C5F0004FF0000170471CF0400F18BF4FF0004093
:10C6000070471CF0100F08D000F07F4220F07043FC
:10C6100042EAD3014FEA4370704700F0604021F0D6
:10C620007F4242EA000201F07F4040EA72707047A8
:10C630004FF0FF0C4CF4E06C1CEA11531CBF9CEA59
:10C64000030C9445C2BFDA4201EB02517047002B44
:10C650000DD0BCF1000F0FD001F00041002AA4BFA3
:10C6600041F0E04141F07F614FF00000704701F080
:10C6700000414FF00000704750EA01334FF09B0C2F
:10C6800018BF4CF0806C7FF413A970471CF4801F16
:10C6900011D01CF4E02F03D06FEACC314900704771
:10C6A0004FF04050EFF3008222F0704242EA000265
:10C6B00082F3008870474FF00000704700000000D0
:10C6C000000000000000F03F000000000000F83F04
:10C6D00000000000000000000000004003B8E23F3E
:10C6E000000000000000000006D0CF43EBFD4C3EF0
:10C6F000033333333333E33FFFAB6FDBB66DDB3FE5
:10C700004D268F515555D53F01411DA96074D13F2C
:10C7100065DBC9934A86CD3FEF4E454A287ECA3F26
:10C720003E5555555555C53F93BDBE166CC166BFA8
:10C730002CDE25AF6A56113FF16BD2C541BDBBBEA1
:10C74000D0A4BE726937663E4FBB610567ACDD3F62
:10C75000182D4454FB21E93F9BF681D20B73EF3F28
:10C76000182D4454FB21F93FE2652F227F2B7A3CA0
:10C77000075C143326A6813CBDCBF07A8807703C59
:10C78000075C143326A6913CC4EB98999999C9BFCC
:10C79000711623FEC671BCBF6D9A74AFF2B0B3BF01
:10C7A0009AFDDE522DDEADBF2F6C6A2C44B4A2BFC1
:10C7B0000D5555555555D53FFF8300922449C23F2D
:10C7C0006E204CC5CD45B73F513DD0A0660DB13F61
:10C7D000EB0D76244B7BA93F11DA22E33AAD903F73
:10C7E0000000000000000000000000006E83F9A2BD
:10C7F0002915444ED15727FCC0DD34F5999562DBED
:10C800004190433CAB6351FE00000000000000007B
:10C8100001020304060708090000000001020304E6
:10C82000100000000000024001000000000402406F
:10C830001000000000080240200000000008024034
:10C8400008000000001802404000000000180240EC
:10C8500018070020080000008806002004000000DF
:10C860008806002008000000880600200C00000058
:10C870008806002000000000D00600200000000014
:10C880006007002000000000600700200400000096
:10C890006007002008000000C4C900080000000074
:10C8A0000000000000000000000000000004000084
:10C8B000180000000000000000000000CEC90008C1
:10C8C0000000000000000000000000000000000068
:10C8D000000400001800000000000000000000003C
:10C8E000C0C90008000000000000000000000000B7
:10C8F000000000000004000018000000000000001C
:10C9000000000000D4C90008000000000000000082
:10C9100000000000000000000004000018000000FB
:10C920000000000000000000E9C90008000000004D
:10C9300000000000000000000000000000040000F3
:10C94000300000000000000000000000DFC9000807
:10C9500000000000000000000000000000000000D7
:10C9600000080000180000000000000000000000A7
:10C97000B4C9000800000000000000000000000032
:10C98000000000000002000018000000000000008D
:10C99000000000009A99993E0000803F0AD7233C8E
:10C9A000000000000000803F0000803F0000000009
:10C9B0000000000064656661756C745461736B00FF
:10C9C000636D6400617474695F6573746900626C9F
:10C9D000696E6B006865696768745F63616C00719C
:10C9E0007561645F6374726C005461736B5F496E50
:10C9F0006974000018CA000800000020400100000F
:10CA0000C401000890CA000840010020888100008D
:10CA10002002000800000000111324F41012022B61
:10CA2000073D63ADC1BA503A33BBD3F2C93A641281
:10CA30006412FA27E8039A99993E2E803FCDCC4C98
:10CA400004423D6914A109402019042A3E202D0A00
:10CA5000D7233C08190419240B45F0412069C43937
:10CA6000803119308340401C0AD7A3300B100C4092
:10CA7000406B80BF602DC1B8323E04300ACDCCCCB3
:10CA80003D6666663F0132101AAA010000000000F0
:040000050800018965
:00000001FF
